
Temp_Control.elf:     file format elf32-littlearm

Sections:
Idx Name          Size      VMA       LMA       File off  Algn
  0 .isr_vector   000001ac  08000000  08000000  00010000  2**0
                  CONTENTS, ALLOC, LOAD, READONLY, DATA
  1 .text         00008ba4  080001b0  080001b0  000101b0  2**4
                  CONTENTS, ALLOC, LOAD, READONLY, CODE
  2 .rodata       0000050c  08008d58  08008d58  00018d58  2**3
                  CONTENTS, ALLOC, LOAD, READONLY, DATA
  3 .ARM.extab    00000000  08009264  08009264  000201dc  2**0
                  CONTENTS
  4 .ARM          00000008  08009264  08009264  00019264  2**2
                  CONTENTS, ALLOC, LOAD, READONLY, DATA
  5 .preinit_array 00000000  0800926c  0800926c  000201dc  2**0
                  CONTENTS, ALLOC, LOAD, DATA
  6 .init_array   00000004  0800926c  0800926c  0001926c  2**2
                  CONTENTS, ALLOC, LOAD, DATA
  7 .fini_array   00000004  08009270  08009270  00019270  2**2
                  CONTENTS, ALLOC, LOAD, DATA
  8 .data         000001dc  20000000  08009274  00020000  2**2
                  CONTENTS, ALLOC, LOAD, DATA
  9 .ccmram       00000000  10000000  10000000  000201dc  2**0
                  CONTENTS
 10 .bss          000001c4  200001dc  200001dc  000201dc  2**2
                  ALLOC
 11 ._user_heap_stack 00000600  200003a0  200003a0  000201dc  2**0
                  ALLOC
 12 .ARM.attributes 00000030  00000000  00000000  000201dc  2**0
                  CONTENTS, READONLY
 13 .debug_info   00010f9d  00000000  00000000  0002020c  2**0
                  CONTENTS, READONLY, DEBUGGING, OCTETS
 14 .debug_abbrev 0000228f  00000000  00000000  000311a9  2**0
                  CONTENTS, READONLY, DEBUGGING, OCTETS
 15 .debug_aranges 00000fe8  00000000  00000000  00033438  2**3
                  CONTENTS, READONLY, DEBUGGING, OCTETS
 16 .debug_ranges 00000f10  00000000  00000000  00034420  2**3
                  CONTENTS, READONLY, DEBUGGING, OCTETS
 17 .debug_macro  00025c9f  00000000  00000000  00035330  2**0
                  CONTENTS, READONLY, DEBUGGING, OCTETS
 18 .debug_line   00011cff  00000000  00000000  0005afcf  2**0
                  CONTENTS, READONLY, DEBUGGING, OCTETS
 19 .debug_str    000e9c01  00000000  00000000  0006ccce  2**0
                  CONTENTS, READONLY, DEBUGGING, OCTETS
 20 .comment      00000050  00000000  00000000  001568cf  2**0
                  CONTENTS, READONLY
 21 .debug_frame  000054b8  00000000  00000000  00156920  2**2
                  CONTENTS, READONLY, DEBUGGING, OCTETS

Disassembly of section .text:

080001b0 <__do_global_dtors_aux>:
 80001b0:	b510      	push	{r4, lr}
 80001b2:	4c05      	ldr	r4, [pc, #20]	; (80001c8 <__do_global_dtors_aux+0x18>)
 80001b4:	7823      	ldrb	r3, [r4, #0]
 80001b6:	b933      	cbnz	r3, 80001c6 <__do_global_dtors_aux+0x16>
 80001b8:	4b04      	ldr	r3, [pc, #16]	; (80001cc <__do_global_dtors_aux+0x1c>)
 80001ba:	b113      	cbz	r3, 80001c2 <__do_global_dtors_aux+0x12>
 80001bc:	4804      	ldr	r0, [pc, #16]	; (80001d0 <__do_global_dtors_aux+0x20>)
 80001be:	f3af 8000 	nop.w
 80001c2:	2301      	movs	r3, #1
 80001c4:	7023      	strb	r3, [r4, #0]
 80001c6:	bd10      	pop	{r4, pc}
 80001c8:	200001dc 	.word	0x200001dc
 80001cc:	00000000 	.word	0x00000000
 80001d0:	08008d3c 	.word	0x08008d3c

080001d4 <frame_dummy>:
 80001d4:	b508      	push	{r3, lr}
 80001d6:	4b03      	ldr	r3, [pc, #12]	; (80001e4 <frame_dummy+0x10>)
 80001d8:	b11b      	cbz	r3, 80001e2 <frame_dummy+0xe>
 80001da:	4903      	ldr	r1, [pc, #12]	; (80001e8 <frame_dummy+0x14>)
 80001dc:	4803      	ldr	r0, [pc, #12]	; (80001ec <frame_dummy+0x18>)
 80001de:	f3af 8000 	nop.w
 80001e2:	bd08      	pop	{r3, pc}
 80001e4:	00000000 	.word	0x00000000
 80001e8:	200001e0 	.word	0x200001e0
 80001ec:	08008d3c 	.word	0x08008d3c

080001f0 <strlen>:
 80001f0:	4603      	mov	r3, r0
 80001f2:	f813 2b01 	ldrb.w	r2, [r3], #1
 80001f6:	2a00      	cmp	r2, #0
 80001f8:	d1fb      	bne.n	80001f2 <strlen+0x2>
 80001fa:	1a18      	subs	r0, r3, r0
 80001fc:	3801      	subs	r0, #1
 80001fe:	4770      	bx	lr

08000200 <memchr>:
 8000200:	f001 01ff 	and.w	r1, r1, #255	; 0xff
 8000204:	2a10      	cmp	r2, #16
 8000206:	db2b      	blt.n	8000260 <memchr+0x60>
 8000208:	f010 0f07 	tst.w	r0, #7
 800020c:	d008      	beq.n	8000220 <memchr+0x20>
 800020e:	f810 3b01 	ldrb.w	r3, [r0], #1
 8000212:	3a01      	subs	r2, #1
 8000214:	428b      	cmp	r3, r1
 8000216:	d02d      	beq.n	8000274 <memchr+0x74>
 8000218:	f010 0f07 	tst.w	r0, #7
 800021c:	b342      	cbz	r2, 8000270 <memchr+0x70>
 800021e:	d1f6      	bne.n	800020e <memchr+0xe>
 8000220:	b4f0      	push	{r4, r5, r6, r7}
 8000222:	ea41 2101 	orr.w	r1, r1, r1, lsl #8
 8000226:	ea41 4101 	orr.w	r1, r1, r1, lsl #16
 800022a:	f022 0407 	bic.w	r4, r2, #7
 800022e:	f07f 0700 	mvns.w	r7, #0
 8000232:	2300      	movs	r3, #0
 8000234:	e8f0 5602 	ldrd	r5, r6, [r0], #8
 8000238:	3c08      	subs	r4, #8
 800023a:	ea85 0501 	eor.w	r5, r5, r1
 800023e:	ea86 0601 	eor.w	r6, r6, r1
 8000242:	fa85 f547 	uadd8	r5, r5, r7
 8000246:	faa3 f587 	sel	r5, r3, r7
 800024a:	fa86 f647 	uadd8	r6, r6, r7
 800024e:	faa5 f687 	sel	r6, r5, r7
 8000252:	b98e      	cbnz	r6, 8000278 <memchr+0x78>
 8000254:	d1ee      	bne.n	8000234 <memchr+0x34>
 8000256:	bcf0      	pop	{r4, r5, r6, r7}
 8000258:	f001 01ff 	and.w	r1, r1, #255	; 0xff
 800025c:	f002 0207 	and.w	r2, r2, #7
 8000260:	b132      	cbz	r2, 8000270 <memchr+0x70>
 8000262:	f810 3b01 	ldrb.w	r3, [r0], #1
 8000266:	3a01      	subs	r2, #1
 8000268:	ea83 0301 	eor.w	r3, r3, r1
 800026c:	b113      	cbz	r3, 8000274 <memchr+0x74>
 800026e:	d1f8      	bne.n	8000262 <memchr+0x62>
 8000270:	2000      	movs	r0, #0
 8000272:	4770      	bx	lr
 8000274:	3801      	subs	r0, #1
 8000276:	4770      	bx	lr
 8000278:	2d00      	cmp	r5, #0
 800027a:	bf06      	itte	eq
 800027c:	4635      	moveq	r5, r6
 800027e:	3803      	subeq	r0, #3
 8000280:	3807      	subne	r0, #7
 8000282:	f015 0f01 	tst.w	r5, #1
 8000286:	d107      	bne.n	8000298 <memchr+0x98>
 8000288:	3001      	adds	r0, #1
 800028a:	f415 7f80 	tst.w	r5, #256	; 0x100
 800028e:	bf02      	ittt	eq
 8000290:	3001      	addeq	r0, #1
 8000292:	f415 3fc0 	tsteq.w	r5, #98304	; 0x18000
 8000296:	3001      	addeq	r0, #1
 8000298:	bcf0      	pop	{r4, r5, r6, r7}
 800029a:	3801      	subs	r0, #1
 800029c:	4770      	bx	lr
 800029e:	bf00      	nop

080002a0 <__aeabi_drsub>:
 80002a0:	f081 4100 	eor.w	r1, r1, #2147483648	; 0x80000000
 80002a4:	e002      	b.n	80002ac <__adddf3>
 80002a6:	bf00      	nop

080002a8 <__aeabi_dsub>:
 80002a8:	f083 4300 	eor.w	r3, r3, #2147483648	; 0x80000000

080002ac <__adddf3>:
 80002ac:	b530      	push	{r4, r5, lr}
 80002ae:	ea4f 0441 	mov.w	r4, r1, lsl #1
 80002b2:	ea4f 0543 	mov.w	r5, r3, lsl #1
 80002b6:	ea94 0f05 	teq	r4, r5
 80002ba:	bf08      	it	eq
 80002bc:	ea90 0f02 	teqeq	r0, r2
 80002c0:	bf1f      	itttt	ne
 80002c2:	ea54 0c00 	orrsne.w	ip, r4, r0
 80002c6:	ea55 0c02 	orrsne.w	ip, r5, r2
 80002ca:	ea7f 5c64 	mvnsne.w	ip, r4, asr #21
 80002ce:	ea7f 5c65 	mvnsne.w	ip, r5, asr #21
 80002d2:	f000 80e2 	beq.w	800049a <__adddf3+0x1ee>
 80002d6:	ea4f 5454 	mov.w	r4, r4, lsr #21
 80002da:	ebd4 5555 	rsbs	r5, r4, r5, lsr #21
 80002de:	bfb8      	it	lt
 80002e0:	426d      	neglt	r5, r5
 80002e2:	dd0c      	ble.n	80002fe <__adddf3+0x52>
 80002e4:	442c      	add	r4, r5
 80002e6:	ea80 0202 	eor.w	r2, r0, r2
 80002ea:	ea81 0303 	eor.w	r3, r1, r3
 80002ee:	ea82 0000 	eor.w	r0, r2, r0
 80002f2:	ea83 0101 	eor.w	r1, r3, r1
 80002f6:	ea80 0202 	eor.w	r2, r0, r2
 80002fa:	ea81 0303 	eor.w	r3, r1, r3
 80002fe:	2d36      	cmp	r5, #54	; 0x36
 8000300:	bf88      	it	hi
 8000302:	bd30      	pophi	{r4, r5, pc}
 8000304:	f011 4f00 	tst.w	r1, #2147483648	; 0x80000000
 8000308:	ea4f 3101 	mov.w	r1, r1, lsl #12
 800030c:	f44f 1c80 	mov.w	ip, #1048576	; 0x100000
 8000310:	ea4c 3111 	orr.w	r1, ip, r1, lsr #12
 8000314:	d002      	beq.n	800031c <__adddf3+0x70>
 8000316:	4240      	negs	r0, r0
 8000318:	eb61 0141 	sbc.w	r1, r1, r1, lsl #1
 800031c:	f013 4f00 	tst.w	r3, #2147483648	; 0x80000000
 8000320:	ea4f 3303 	mov.w	r3, r3, lsl #12
 8000324:	ea4c 3313 	orr.w	r3, ip, r3, lsr #12
 8000328:	d002      	beq.n	8000330 <__adddf3+0x84>
 800032a:	4252      	negs	r2, r2
 800032c:	eb63 0343 	sbc.w	r3, r3, r3, lsl #1
 8000330:	ea94 0f05 	teq	r4, r5
 8000334:	f000 80a7 	beq.w	8000486 <__adddf3+0x1da>
 8000338:	f1a4 0401 	sub.w	r4, r4, #1
 800033c:	f1d5 0e20 	rsbs	lr, r5, #32
 8000340:	db0d      	blt.n	800035e <__adddf3+0xb2>
 8000342:	fa02 fc0e 	lsl.w	ip, r2, lr
 8000346:	fa22 f205 	lsr.w	r2, r2, r5
 800034a:	1880      	adds	r0, r0, r2
 800034c:	f141 0100 	adc.w	r1, r1, #0
 8000350:	fa03 f20e 	lsl.w	r2, r3, lr
 8000354:	1880      	adds	r0, r0, r2
 8000356:	fa43 f305 	asr.w	r3, r3, r5
 800035a:	4159      	adcs	r1, r3
 800035c:	e00e      	b.n	800037c <__adddf3+0xd0>
 800035e:	f1a5 0520 	sub.w	r5, r5, #32
 8000362:	f10e 0e20 	add.w	lr, lr, #32
 8000366:	2a01      	cmp	r2, #1
 8000368:	fa03 fc0e 	lsl.w	ip, r3, lr
 800036c:	bf28      	it	cs
 800036e:	f04c 0c02 	orrcs.w	ip, ip, #2
 8000372:	fa43 f305 	asr.w	r3, r3, r5
 8000376:	18c0      	adds	r0, r0, r3
 8000378:	eb51 71e3 	adcs.w	r1, r1, r3, asr #31
 800037c:	f001 4500 	and.w	r5, r1, #2147483648	; 0x80000000
 8000380:	d507      	bpl.n	8000392 <__adddf3+0xe6>
 8000382:	f04f 0e00 	mov.w	lr, #0
 8000386:	f1dc 0c00 	rsbs	ip, ip, #0
 800038a:	eb7e 0000 	sbcs.w	r0, lr, r0
 800038e:	eb6e 0101 	sbc.w	r1, lr, r1
 8000392:	f5b1 1f80 	cmp.w	r1, #1048576	; 0x100000
 8000396:	d31b      	bcc.n	80003d0 <__adddf3+0x124>
 8000398:	f5b1 1f00 	cmp.w	r1, #2097152	; 0x200000
 800039c:	d30c      	bcc.n	80003b8 <__adddf3+0x10c>
 800039e:	0849      	lsrs	r1, r1, #1
 80003a0:	ea5f 0030 	movs.w	r0, r0, rrx
 80003a4:	ea4f 0c3c 	mov.w	ip, ip, rrx
 80003a8:	f104 0401 	add.w	r4, r4, #1
 80003ac:	ea4f 5244 	mov.w	r2, r4, lsl #21
 80003b0:	f512 0f80 	cmn.w	r2, #4194304	; 0x400000
 80003b4:	f080 809a 	bcs.w	80004ec <__adddf3+0x240>
 80003b8:	f1bc 4f00 	cmp.w	ip, #2147483648	; 0x80000000
 80003bc:	bf08      	it	eq
 80003be:	ea5f 0c50 	movseq.w	ip, r0, lsr #1
 80003c2:	f150 0000 	adcs.w	r0, r0, #0
 80003c6:	eb41 5104 	adc.w	r1, r1, r4, lsl #20
 80003ca:	ea41 0105 	orr.w	r1, r1, r5
 80003ce:	bd30      	pop	{r4, r5, pc}
 80003d0:	ea5f 0c4c 	movs.w	ip, ip, lsl #1
 80003d4:	4140      	adcs	r0, r0
 80003d6:	eb41 0101 	adc.w	r1, r1, r1
 80003da:	3c01      	subs	r4, #1
 80003dc:	bf28      	it	cs
 80003de:	f5b1 1f80 	cmpcs.w	r1, #1048576	; 0x100000
 80003e2:	d2e9      	bcs.n	80003b8 <__adddf3+0x10c>
 80003e4:	f091 0f00 	teq	r1, #0
 80003e8:	bf04      	itt	eq
 80003ea:	4601      	moveq	r1, r0
 80003ec:	2000      	moveq	r0, #0
 80003ee:	fab1 f381 	clz	r3, r1
 80003f2:	bf08      	it	eq
 80003f4:	3320      	addeq	r3, #32
 80003f6:	f1a3 030b 	sub.w	r3, r3, #11
 80003fa:	f1b3 0220 	subs.w	r2, r3, #32
 80003fe:	da0c      	bge.n	800041a <__adddf3+0x16e>
 8000400:	320c      	adds	r2, #12
 8000402:	dd08      	ble.n	8000416 <__adddf3+0x16a>
 8000404:	f102 0c14 	add.w	ip, r2, #20
 8000408:	f1c2 020c 	rsb	r2, r2, #12
 800040c:	fa01 f00c 	lsl.w	r0, r1, ip
 8000410:	fa21 f102 	lsr.w	r1, r1, r2
 8000414:	e00c      	b.n	8000430 <__adddf3+0x184>
 8000416:	f102 0214 	add.w	r2, r2, #20
 800041a:	bfd8      	it	le
 800041c:	f1c2 0c20 	rsble	ip, r2, #32
 8000420:	fa01 f102 	lsl.w	r1, r1, r2
 8000424:	fa20 fc0c 	lsr.w	ip, r0, ip
 8000428:	bfdc      	itt	le
 800042a:	ea41 010c 	orrle.w	r1, r1, ip
 800042e:	4090      	lslle	r0, r2
 8000430:	1ae4      	subs	r4, r4, r3
 8000432:	bfa2      	ittt	ge
 8000434:	eb01 5104 	addge.w	r1, r1, r4, lsl #20
 8000438:	4329      	orrge	r1, r5
 800043a:	bd30      	popge	{r4, r5, pc}
 800043c:	ea6f 0404 	mvn.w	r4, r4
 8000440:	3c1f      	subs	r4, #31
 8000442:	da1c      	bge.n	800047e <__adddf3+0x1d2>
 8000444:	340c      	adds	r4, #12
 8000446:	dc0e      	bgt.n	8000466 <__adddf3+0x1ba>
 8000448:	f104 0414 	add.w	r4, r4, #20
 800044c:	f1c4 0220 	rsb	r2, r4, #32
 8000450:	fa20 f004 	lsr.w	r0, r0, r4
 8000454:	fa01 f302 	lsl.w	r3, r1, r2
 8000458:	ea40 0003 	orr.w	r0, r0, r3
 800045c:	fa21 f304 	lsr.w	r3, r1, r4
 8000460:	ea45 0103 	orr.w	r1, r5, r3
 8000464:	bd30      	pop	{r4, r5, pc}
 8000466:	f1c4 040c 	rsb	r4, r4, #12
 800046a:	f1c4 0220 	rsb	r2, r4, #32
 800046e:	fa20 f002 	lsr.w	r0, r0, r2
 8000472:	fa01 f304 	lsl.w	r3, r1, r4
 8000476:	ea40 0003 	orr.w	r0, r0, r3
 800047a:	4629      	mov	r1, r5
 800047c:	bd30      	pop	{r4, r5, pc}
 800047e:	fa21 f004 	lsr.w	r0, r1, r4
 8000482:	4629      	mov	r1, r5
 8000484:	bd30      	pop	{r4, r5, pc}
 8000486:	f094 0f00 	teq	r4, #0
 800048a:	f483 1380 	eor.w	r3, r3, #1048576	; 0x100000
 800048e:	bf06      	itte	eq
 8000490:	f481 1180 	eoreq.w	r1, r1, #1048576	; 0x100000
 8000494:	3401      	addeq	r4, #1
 8000496:	3d01      	subne	r5, #1
 8000498:	e74e      	b.n	8000338 <__adddf3+0x8c>
 800049a:	ea7f 5c64 	mvns.w	ip, r4, asr #21
 800049e:	bf18      	it	ne
 80004a0:	ea7f 5c65 	mvnsne.w	ip, r5, asr #21
 80004a4:	d029      	beq.n	80004fa <__adddf3+0x24e>
 80004a6:	ea94 0f05 	teq	r4, r5
 80004aa:	bf08      	it	eq
 80004ac:	ea90 0f02 	teqeq	r0, r2
 80004b0:	d005      	beq.n	80004be <__adddf3+0x212>
 80004b2:	ea54 0c00 	orrs.w	ip, r4, r0
 80004b6:	bf04      	itt	eq
 80004b8:	4619      	moveq	r1, r3
 80004ba:	4610      	moveq	r0, r2
 80004bc:	bd30      	pop	{r4, r5, pc}
 80004be:	ea91 0f03 	teq	r1, r3
 80004c2:	bf1e      	ittt	ne
 80004c4:	2100      	movne	r1, #0
 80004c6:	2000      	movne	r0, #0
 80004c8:	bd30      	popne	{r4, r5, pc}
 80004ca:	ea5f 5c54 	movs.w	ip, r4, lsr #21
 80004ce:	d105      	bne.n	80004dc <__adddf3+0x230>
 80004d0:	0040      	lsls	r0, r0, #1
 80004d2:	4149      	adcs	r1, r1
 80004d4:	bf28      	it	cs
 80004d6:	f041 4100 	orrcs.w	r1, r1, #2147483648	; 0x80000000
 80004da:	bd30      	pop	{r4, r5, pc}
 80004dc:	f514 0480 	adds.w	r4, r4, #4194304	; 0x400000
 80004e0:	bf3c      	itt	cc
 80004e2:	f501 1180 	addcc.w	r1, r1, #1048576	; 0x100000
 80004e6:	bd30      	popcc	{r4, r5, pc}
 80004e8:	f001 4500 	and.w	r5, r1, #2147483648	; 0x80000000
 80004ec:	f045 41fe 	orr.w	r1, r5, #2130706432	; 0x7f000000
 80004f0:	f441 0170 	orr.w	r1, r1, #15728640	; 0xf00000
 80004f4:	f04f 0000 	mov.w	r0, #0
 80004f8:	bd30      	pop	{r4, r5, pc}
 80004fa:	ea7f 5c64 	mvns.w	ip, r4, asr #21
 80004fe:	bf1a      	itte	ne
 8000500:	4619      	movne	r1, r3
 8000502:	4610      	movne	r0, r2
 8000504:	ea7f 5c65 	mvnseq.w	ip, r5, asr #21
 8000508:	bf1c      	itt	ne
 800050a:	460b      	movne	r3, r1
 800050c:	4602      	movne	r2, r0
 800050e:	ea50 3401 	orrs.w	r4, r0, r1, lsl #12
 8000512:	bf06      	itte	eq
 8000514:	ea52 3503 	orrseq.w	r5, r2, r3, lsl #12
 8000518:	ea91 0f03 	teqeq	r1, r3
 800051c:	f441 2100 	orrne.w	r1, r1, #524288	; 0x80000
 8000520:	bd30      	pop	{r4, r5, pc}
 8000522:	bf00      	nop

08000524 <__aeabi_ui2d>:
 8000524:	f090 0f00 	teq	r0, #0
 8000528:	bf04      	itt	eq
 800052a:	2100      	moveq	r1, #0
 800052c:	4770      	bxeq	lr
 800052e:	b530      	push	{r4, r5, lr}
 8000530:	f44f 6480 	mov.w	r4, #1024	; 0x400
 8000534:	f104 0432 	add.w	r4, r4, #50	; 0x32
 8000538:	f04f 0500 	mov.w	r5, #0
 800053c:	f04f 0100 	mov.w	r1, #0
 8000540:	e750      	b.n	80003e4 <__adddf3+0x138>
 8000542:	bf00      	nop

08000544 <__aeabi_i2d>:
 8000544:	f090 0f00 	teq	r0, #0
 8000548:	bf04      	itt	eq
 800054a:	2100      	moveq	r1, #0
 800054c:	4770      	bxeq	lr
 800054e:	b530      	push	{r4, r5, lr}
 8000550:	f44f 6480 	mov.w	r4, #1024	; 0x400
 8000554:	f104 0432 	add.w	r4, r4, #50	; 0x32
 8000558:	f010 4500 	ands.w	r5, r0, #2147483648	; 0x80000000
 800055c:	bf48      	it	mi
 800055e:	4240      	negmi	r0, r0
 8000560:	f04f 0100 	mov.w	r1, #0
 8000564:	e73e      	b.n	80003e4 <__adddf3+0x138>
 8000566:	bf00      	nop

08000568 <__aeabi_f2d>:
 8000568:	0042      	lsls	r2, r0, #1
 800056a:	ea4f 01e2 	mov.w	r1, r2, asr #3
 800056e:	ea4f 0131 	mov.w	r1, r1, rrx
 8000572:	ea4f 7002 	mov.w	r0, r2, lsl #28
 8000576:	bf1f      	itttt	ne
 8000578:	f012 437f 	andsne.w	r3, r2, #4278190080	; 0xff000000
 800057c:	f093 4f7f 	teqne	r3, #4278190080	; 0xff000000
 8000580:	f081 5160 	eorne.w	r1, r1, #939524096	; 0x38000000
 8000584:	4770      	bxne	lr
 8000586:	f032 427f 	bics.w	r2, r2, #4278190080	; 0xff000000
 800058a:	bf08      	it	eq
 800058c:	4770      	bxeq	lr
 800058e:	f093 4f7f 	teq	r3, #4278190080	; 0xff000000
 8000592:	bf04      	itt	eq
 8000594:	f441 2100 	orreq.w	r1, r1, #524288	; 0x80000
 8000598:	4770      	bxeq	lr
 800059a:	b530      	push	{r4, r5, lr}
 800059c:	f44f 7460 	mov.w	r4, #896	; 0x380
 80005a0:	f001 4500 	and.w	r5, r1, #2147483648	; 0x80000000
 80005a4:	f021 4100 	bic.w	r1, r1, #2147483648	; 0x80000000
 80005a8:	e71c      	b.n	80003e4 <__adddf3+0x138>
 80005aa:	bf00      	nop

080005ac <__aeabi_ul2d>:
 80005ac:	ea50 0201 	orrs.w	r2, r0, r1
 80005b0:	bf08      	it	eq
 80005b2:	4770      	bxeq	lr
 80005b4:	b530      	push	{r4, r5, lr}
 80005b6:	f04f 0500 	mov.w	r5, #0
 80005ba:	e00a      	b.n	80005d2 <__aeabi_l2d+0x16>

080005bc <__aeabi_l2d>:
 80005bc:	ea50 0201 	orrs.w	r2, r0, r1
 80005c0:	bf08      	it	eq
 80005c2:	4770      	bxeq	lr
 80005c4:	b530      	push	{r4, r5, lr}
 80005c6:	f011 4500 	ands.w	r5, r1, #2147483648	; 0x80000000
 80005ca:	d502      	bpl.n	80005d2 <__aeabi_l2d+0x16>
 80005cc:	4240      	negs	r0, r0
 80005ce:	eb61 0141 	sbc.w	r1, r1, r1, lsl #1
 80005d2:	f44f 6480 	mov.w	r4, #1024	; 0x400
 80005d6:	f104 0432 	add.w	r4, r4, #50	; 0x32
 80005da:	ea5f 5c91 	movs.w	ip, r1, lsr #22
 80005de:	f43f aed8 	beq.w	8000392 <__adddf3+0xe6>
 80005e2:	f04f 0203 	mov.w	r2, #3
 80005e6:	ea5f 0cdc 	movs.w	ip, ip, lsr #3
 80005ea:	bf18      	it	ne
 80005ec:	3203      	addne	r2, #3
 80005ee:	ea5f 0cdc 	movs.w	ip, ip, lsr #3
 80005f2:	bf18      	it	ne
 80005f4:	3203      	addne	r2, #3
 80005f6:	eb02 02dc 	add.w	r2, r2, ip, lsr #3
 80005fa:	f1c2 0320 	rsb	r3, r2, #32
 80005fe:	fa00 fc03 	lsl.w	ip, r0, r3
 8000602:	fa20 f002 	lsr.w	r0, r0, r2
 8000606:	fa01 fe03 	lsl.w	lr, r1, r3
 800060a:	ea40 000e 	orr.w	r0, r0, lr
 800060e:	fa21 f102 	lsr.w	r1, r1, r2
 8000612:	4414      	add	r4, r2
 8000614:	e6bd      	b.n	8000392 <__adddf3+0xe6>
 8000616:	bf00      	nop

08000618 <__aeabi_dmul>:
 8000618:	b570      	push	{r4, r5, r6, lr}
 800061a:	f04f 0cff 	mov.w	ip, #255	; 0xff
 800061e:	f44c 6ce0 	orr.w	ip, ip, #1792	; 0x700
 8000622:	ea1c 5411 	ands.w	r4, ip, r1, lsr #20
 8000626:	bf1d      	ittte	ne
 8000628:	ea1c 5513 	andsne.w	r5, ip, r3, lsr #20
 800062c:	ea94 0f0c 	teqne	r4, ip
 8000630:	ea95 0f0c 	teqne	r5, ip
 8000634:	f000 f8de 	bleq	80007f4 <__aeabi_dmul+0x1dc>
 8000638:	442c      	add	r4, r5
 800063a:	ea81 0603 	eor.w	r6, r1, r3
 800063e:	ea21 514c 	bic.w	r1, r1, ip, lsl #21
 8000642:	ea23 534c 	bic.w	r3, r3, ip, lsl #21
 8000646:	ea50 3501 	orrs.w	r5, r0, r1, lsl #12
 800064a:	bf18      	it	ne
 800064c:	ea52 3503 	orrsne.w	r5, r2, r3, lsl #12
 8000650:	f441 1180 	orr.w	r1, r1, #1048576	; 0x100000
 8000654:	f443 1380 	orr.w	r3, r3, #1048576	; 0x100000
 8000658:	d038      	beq.n	80006cc <__aeabi_dmul+0xb4>
 800065a:	fba0 ce02 	umull	ip, lr, r0, r2
 800065e:	f04f 0500 	mov.w	r5, #0
 8000662:	fbe1 e502 	umlal	lr, r5, r1, r2
 8000666:	f006 4200 	and.w	r2, r6, #2147483648	; 0x80000000
 800066a:	fbe0 e503 	umlal	lr, r5, r0, r3
 800066e:	f04f 0600 	mov.w	r6, #0
 8000672:	fbe1 5603 	umlal	r5, r6, r1, r3
 8000676:	f09c 0f00 	teq	ip, #0
 800067a:	bf18      	it	ne
 800067c:	f04e 0e01 	orrne.w	lr, lr, #1
 8000680:	f1a4 04ff 	sub.w	r4, r4, #255	; 0xff
 8000684:	f5b6 7f00 	cmp.w	r6, #512	; 0x200
 8000688:	f564 7440 	sbc.w	r4, r4, #768	; 0x300
 800068c:	d204      	bcs.n	8000698 <__aeabi_dmul+0x80>
 800068e:	ea5f 0e4e 	movs.w	lr, lr, lsl #1
 8000692:	416d      	adcs	r5, r5
 8000694:	eb46 0606 	adc.w	r6, r6, r6
 8000698:	ea42 21c6 	orr.w	r1, r2, r6, lsl #11
 800069c:	ea41 5155 	orr.w	r1, r1, r5, lsr #21
 80006a0:	ea4f 20c5 	mov.w	r0, r5, lsl #11
 80006a4:	ea40 505e 	orr.w	r0, r0, lr, lsr #21
 80006a8:	ea4f 2ece 	mov.w	lr, lr, lsl #11
 80006ac:	f1b4 0cfd 	subs.w	ip, r4, #253	; 0xfd
 80006b0:	bf88      	it	hi
 80006b2:	f5bc 6fe0 	cmphi.w	ip, #1792	; 0x700
 80006b6:	d81e      	bhi.n	80006f6 <__aeabi_dmul+0xde>
 80006b8:	f1be 4f00 	cmp.w	lr, #2147483648	; 0x80000000
 80006bc:	bf08      	it	eq
 80006be:	ea5f 0e50 	movseq.w	lr, r0, lsr #1
 80006c2:	f150 0000 	adcs.w	r0, r0, #0
 80006c6:	eb41 5104 	adc.w	r1, r1, r4, lsl #20
 80006ca:	bd70      	pop	{r4, r5, r6, pc}
 80006cc:	f006 4600 	and.w	r6, r6, #2147483648	; 0x80000000
 80006d0:	ea46 0101 	orr.w	r1, r6, r1
 80006d4:	ea40 0002 	orr.w	r0, r0, r2
 80006d8:	ea81 0103 	eor.w	r1, r1, r3
 80006dc:	ebb4 045c 	subs.w	r4, r4, ip, lsr #1
 80006e0:	bfc2      	ittt	gt
 80006e2:	ebd4 050c 	rsbsgt	r5, r4, ip
 80006e6:	ea41 5104 	orrgt.w	r1, r1, r4, lsl #20
 80006ea:	bd70      	popgt	{r4, r5, r6, pc}
 80006ec:	f441 1180 	orr.w	r1, r1, #1048576	; 0x100000
 80006f0:	f04f 0e00 	mov.w	lr, #0
 80006f4:	3c01      	subs	r4, #1
 80006f6:	f300 80ab 	bgt.w	8000850 <__aeabi_dmul+0x238>
 80006fa:	f114 0f36 	cmn.w	r4, #54	; 0x36
 80006fe:	bfde      	ittt	le
 8000700:	2000      	movle	r0, #0
 8000702:	f001 4100 	andle.w	r1, r1, #2147483648	; 0x80000000
 8000706:	bd70      	pople	{r4, r5, r6, pc}
 8000708:	f1c4 0400 	rsb	r4, r4, #0
 800070c:	3c20      	subs	r4, #32
 800070e:	da35      	bge.n	800077c <__aeabi_dmul+0x164>
 8000710:	340c      	adds	r4, #12
 8000712:	dc1b      	bgt.n	800074c <__aeabi_dmul+0x134>
 8000714:	f104 0414 	add.w	r4, r4, #20
 8000718:	f1c4 0520 	rsb	r5, r4, #32
 800071c:	fa00 f305 	lsl.w	r3, r0, r5
 8000720:	fa20 f004 	lsr.w	r0, r0, r4
 8000724:	fa01 f205 	lsl.w	r2, r1, r5
 8000728:	ea40 0002 	orr.w	r0, r0, r2
 800072c:	f001 4200 	and.w	r2, r1, #2147483648	; 0x80000000
 8000730:	f021 4100 	bic.w	r1, r1, #2147483648	; 0x80000000
 8000734:	eb10 70d3 	adds.w	r0, r0, r3, lsr #31
 8000738:	fa21 f604 	lsr.w	r6, r1, r4
 800073c:	eb42 0106 	adc.w	r1, r2, r6
 8000740:	ea5e 0e43 	orrs.w	lr, lr, r3, lsl #1
 8000744:	bf08      	it	eq
 8000746:	ea20 70d3 	biceq.w	r0, r0, r3, lsr #31
 800074a:	bd70      	pop	{r4, r5, r6, pc}
 800074c:	f1c4 040c 	rsb	r4, r4, #12
 8000750:	f1c4 0520 	rsb	r5, r4, #32
 8000754:	fa00 f304 	lsl.w	r3, r0, r4
 8000758:	fa20 f005 	lsr.w	r0, r0, r5
 800075c:	fa01 f204 	lsl.w	r2, r1, r4
 8000760:	ea40 0002 	orr.w	r0, r0, r2
 8000764:	f001 4100 	and.w	r1, r1, #2147483648	; 0x80000000
 8000768:	eb10 70d3 	adds.w	r0, r0, r3, lsr #31
 800076c:	f141 0100 	adc.w	r1, r1, #0
 8000770:	ea5e 0e43 	orrs.w	lr, lr, r3, lsl #1
 8000774:	bf08      	it	eq
 8000776:	ea20 70d3 	biceq.w	r0, r0, r3, lsr #31
 800077a:	bd70      	pop	{r4, r5, r6, pc}
 800077c:	f1c4 0520 	rsb	r5, r4, #32
 8000780:	fa00 f205 	lsl.w	r2, r0, r5
 8000784:	ea4e 0e02 	orr.w	lr, lr, r2
 8000788:	fa20 f304 	lsr.w	r3, r0, r4
 800078c:	fa01 f205 	lsl.w	r2, r1, r5
 8000790:	ea43 0302 	orr.w	r3, r3, r2
 8000794:	fa21 f004 	lsr.w	r0, r1, r4
 8000798:	f001 4100 	and.w	r1, r1, #2147483648	; 0x80000000
 800079c:	fa21 f204 	lsr.w	r2, r1, r4
 80007a0:	ea20 0002 	bic.w	r0, r0, r2
 80007a4:	eb00 70d3 	add.w	r0, r0, r3, lsr #31
 80007a8:	ea5e 0e43 	orrs.w	lr, lr, r3, lsl #1
 80007ac:	bf08      	it	eq
 80007ae:	ea20 70d3 	biceq.w	r0, r0, r3, lsr #31
 80007b2:	bd70      	pop	{r4, r5, r6, pc}
 80007b4:	f094 0f00 	teq	r4, #0
 80007b8:	d10f      	bne.n	80007da <__aeabi_dmul+0x1c2>
 80007ba:	f001 4600 	and.w	r6, r1, #2147483648	; 0x80000000
 80007be:	0040      	lsls	r0, r0, #1
 80007c0:	eb41 0101 	adc.w	r1, r1, r1
 80007c4:	f411 1f80 	tst.w	r1, #1048576	; 0x100000
 80007c8:	bf08      	it	eq
 80007ca:	3c01      	subeq	r4, #1
 80007cc:	d0f7      	beq.n	80007be <__aeabi_dmul+0x1a6>
 80007ce:	ea41 0106 	orr.w	r1, r1, r6
 80007d2:	f095 0f00 	teq	r5, #0
 80007d6:	bf18      	it	ne
 80007d8:	4770      	bxne	lr
 80007da:	f003 4600 	and.w	r6, r3, #2147483648	; 0x80000000
 80007de:	0052      	lsls	r2, r2, #1
 80007e0:	eb43 0303 	adc.w	r3, r3, r3
 80007e4:	f413 1f80 	tst.w	r3, #1048576	; 0x100000
 80007e8:	bf08      	it	eq
 80007ea:	3d01      	subeq	r5, #1
 80007ec:	d0f7      	beq.n	80007de <__aeabi_dmul+0x1c6>
 80007ee:	ea43 0306 	orr.w	r3, r3, r6
 80007f2:	4770      	bx	lr
 80007f4:	ea94 0f0c 	teq	r4, ip
 80007f8:	ea0c 5513 	and.w	r5, ip, r3, lsr #20
 80007fc:	bf18      	it	ne
 80007fe:	ea95 0f0c 	teqne	r5, ip
 8000802:	d00c      	beq.n	800081e <__aeabi_dmul+0x206>
 8000804:	ea50 0641 	orrs.w	r6, r0, r1, lsl #1
 8000808:	bf18      	it	ne
 800080a:	ea52 0643 	orrsne.w	r6, r2, r3, lsl #1
 800080e:	d1d1      	bne.n	80007b4 <__aeabi_dmul+0x19c>
 8000810:	ea81 0103 	eor.w	r1, r1, r3
 8000814:	f001 4100 	and.w	r1, r1, #2147483648	; 0x80000000
 8000818:	f04f 0000 	mov.w	r0, #0
 800081c:	bd70      	pop	{r4, r5, r6, pc}
 800081e:	ea50 0641 	orrs.w	r6, r0, r1, lsl #1
 8000822:	bf06      	itte	eq
 8000824:	4610      	moveq	r0, r2
 8000826:	4619      	moveq	r1, r3
 8000828:	ea52 0643 	orrsne.w	r6, r2, r3, lsl #1
 800082c:	d019      	beq.n	8000862 <__aeabi_dmul+0x24a>
 800082e:	ea94 0f0c 	teq	r4, ip
 8000832:	d102      	bne.n	800083a <__aeabi_dmul+0x222>
 8000834:	ea50 3601 	orrs.w	r6, r0, r1, lsl #12
 8000838:	d113      	bne.n	8000862 <__aeabi_dmul+0x24a>
 800083a:	ea95 0f0c 	teq	r5, ip
 800083e:	d105      	bne.n	800084c <__aeabi_dmul+0x234>
 8000840:	ea52 3603 	orrs.w	r6, r2, r3, lsl #12
 8000844:	bf1c      	itt	ne
 8000846:	4610      	movne	r0, r2
 8000848:	4619      	movne	r1, r3
 800084a:	d10a      	bne.n	8000862 <__aeabi_dmul+0x24a>
 800084c:	ea81 0103 	eor.w	r1, r1, r3
 8000850:	f001 4100 	and.w	r1, r1, #2147483648	; 0x80000000
 8000854:	f041 41fe 	orr.w	r1, r1, #2130706432	; 0x7f000000
 8000858:	f441 0170 	orr.w	r1, r1, #15728640	; 0xf00000
 800085c:	f04f 0000 	mov.w	r0, #0
 8000860:	bd70      	pop	{r4, r5, r6, pc}
 8000862:	f041 41fe 	orr.w	r1, r1, #2130706432	; 0x7f000000
 8000866:	f441 0178 	orr.w	r1, r1, #16252928	; 0xf80000
 800086a:	bd70      	pop	{r4, r5, r6, pc}

0800086c <__aeabi_ddiv>:
 800086c:	b570      	push	{r4, r5, r6, lr}
 800086e:	f04f 0cff 	mov.w	ip, #255	; 0xff
 8000872:	f44c 6ce0 	orr.w	ip, ip, #1792	; 0x700
 8000876:	ea1c 5411 	ands.w	r4, ip, r1, lsr #20
 800087a:	bf1d      	ittte	ne
 800087c:	ea1c 5513 	andsne.w	r5, ip, r3, lsr #20
 8000880:	ea94 0f0c 	teqne	r4, ip
 8000884:	ea95 0f0c 	teqne	r5, ip
 8000888:	f000 f8a7 	bleq	80009da <__aeabi_ddiv+0x16e>
 800088c:	eba4 0405 	sub.w	r4, r4, r5
 8000890:	ea81 0e03 	eor.w	lr, r1, r3
 8000894:	ea52 3503 	orrs.w	r5, r2, r3, lsl #12
 8000898:	ea4f 3101 	mov.w	r1, r1, lsl #12
 800089c:	f000 8088 	beq.w	80009b0 <__aeabi_ddiv+0x144>
 80008a0:	ea4f 3303 	mov.w	r3, r3, lsl #12
 80008a4:	f04f 5580 	mov.w	r5, #268435456	; 0x10000000
 80008a8:	ea45 1313 	orr.w	r3, r5, r3, lsr #4
 80008ac:	ea43 6312 	orr.w	r3, r3, r2, lsr #24
 80008b0:	ea4f 2202 	mov.w	r2, r2, lsl #8
 80008b4:	ea45 1511 	orr.w	r5, r5, r1, lsr #4
 80008b8:	ea45 6510 	orr.w	r5, r5, r0, lsr #24
 80008bc:	ea4f 2600 	mov.w	r6, r0, lsl #8
 80008c0:	f00e 4100 	and.w	r1, lr, #2147483648	; 0x80000000
 80008c4:	429d      	cmp	r5, r3
 80008c6:	bf08      	it	eq
 80008c8:	4296      	cmpeq	r6, r2
 80008ca:	f144 04fd 	adc.w	r4, r4, #253	; 0xfd
 80008ce:	f504 7440 	add.w	r4, r4, #768	; 0x300
 80008d2:	d202      	bcs.n	80008da <__aeabi_ddiv+0x6e>
 80008d4:	085b      	lsrs	r3, r3, #1
 80008d6:	ea4f 0232 	mov.w	r2, r2, rrx
 80008da:	1ab6      	subs	r6, r6, r2
 80008dc:	eb65 0503 	sbc.w	r5, r5, r3
 80008e0:	085b      	lsrs	r3, r3, #1
 80008e2:	ea4f 0232 	mov.w	r2, r2, rrx
 80008e6:	f44f 1080 	mov.w	r0, #1048576	; 0x100000
 80008ea:	f44f 2c00 	mov.w	ip, #524288	; 0x80000
 80008ee:	ebb6 0e02 	subs.w	lr, r6, r2
 80008f2:	eb75 0e03 	sbcs.w	lr, r5, r3
 80008f6:	bf22      	ittt	cs
 80008f8:	1ab6      	subcs	r6, r6, r2
 80008fa:	4675      	movcs	r5, lr
 80008fc:	ea40 000c 	orrcs.w	r0, r0, ip
 8000900:	085b      	lsrs	r3, r3, #1
 8000902:	ea4f 0232 	mov.w	r2, r2, rrx
 8000906:	ebb6 0e02 	subs.w	lr, r6, r2
 800090a:	eb75 0e03 	sbcs.w	lr, r5, r3
 800090e:	bf22      	ittt	cs
 8000910:	1ab6      	subcs	r6, r6, r2
 8000912:	4675      	movcs	r5, lr
 8000914:	ea40 005c 	orrcs.w	r0, r0, ip, lsr #1
 8000918:	085b      	lsrs	r3, r3, #1
 800091a:	ea4f 0232 	mov.w	r2, r2, rrx
 800091e:	ebb6 0e02 	subs.w	lr, r6, r2
 8000922:	eb75 0e03 	sbcs.w	lr, r5, r3
 8000926:	bf22      	ittt	cs
 8000928:	1ab6      	subcs	r6, r6, r2
 800092a:	4675      	movcs	r5, lr
 800092c:	ea40 009c 	orrcs.w	r0, r0, ip, lsr #2
 8000930:	085b      	lsrs	r3, r3, #1
 8000932:	ea4f 0232 	mov.w	r2, r2, rrx
 8000936:	ebb6 0e02 	subs.w	lr, r6, r2
 800093a:	eb75 0e03 	sbcs.w	lr, r5, r3
 800093e:	bf22      	ittt	cs
 8000940:	1ab6      	subcs	r6, r6, r2
 8000942:	4675      	movcs	r5, lr
 8000944:	ea40 00dc 	orrcs.w	r0, r0, ip, lsr #3
 8000948:	ea55 0e06 	orrs.w	lr, r5, r6
 800094c:	d018      	beq.n	8000980 <__aeabi_ddiv+0x114>
 800094e:	ea4f 1505 	mov.w	r5, r5, lsl #4
 8000952:	ea45 7516 	orr.w	r5, r5, r6, lsr #28
 8000956:	ea4f 1606 	mov.w	r6, r6, lsl #4
 800095a:	ea4f 03c3 	mov.w	r3, r3, lsl #3
 800095e:	ea43 7352 	orr.w	r3, r3, r2, lsr #29
 8000962:	ea4f 02c2 	mov.w	r2, r2, lsl #3
 8000966:	ea5f 1c1c 	movs.w	ip, ip, lsr #4
 800096a:	d1c0      	bne.n	80008ee <__aeabi_ddiv+0x82>
 800096c:	f411 1f80 	tst.w	r1, #1048576	; 0x100000
 8000970:	d10b      	bne.n	800098a <__aeabi_ddiv+0x11e>
 8000972:	ea41 0100 	orr.w	r1, r1, r0
 8000976:	f04f 0000 	mov.w	r0, #0
 800097a:	f04f 4c00 	mov.w	ip, #2147483648	; 0x80000000
 800097e:	e7b6      	b.n	80008ee <__aeabi_ddiv+0x82>
 8000980:	f411 1f80 	tst.w	r1, #1048576	; 0x100000
 8000984:	bf04      	itt	eq
 8000986:	4301      	orreq	r1, r0
 8000988:	2000      	moveq	r0, #0
 800098a:	f1b4 0cfd 	subs.w	ip, r4, #253	; 0xfd
 800098e:	bf88      	it	hi
 8000990:	f5bc 6fe0 	cmphi.w	ip, #1792	; 0x700
 8000994:	f63f aeaf 	bhi.w	80006f6 <__aeabi_dmul+0xde>
 8000998:	ebb5 0c03 	subs.w	ip, r5, r3
 800099c:	bf04      	itt	eq
 800099e:	ebb6 0c02 	subseq.w	ip, r6, r2
 80009a2:	ea5f 0c50 	movseq.w	ip, r0, lsr #1
 80009a6:	f150 0000 	adcs.w	r0, r0, #0
 80009aa:	eb41 5104 	adc.w	r1, r1, r4, lsl #20
 80009ae:	bd70      	pop	{r4, r5, r6, pc}
 80009b0:	f00e 4e00 	and.w	lr, lr, #2147483648	; 0x80000000
 80009b4:	ea4e 3111 	orr.w	r1, lr, r1, lsr #12
 80009b8:	eb14 045c 	adds.w	r4, r4, ip, lsr #1
 80009bc:	bfc2      	ittt	gt
 80009be:	ebd4 050c 	rsbsgt	r5, r4, ip
 80009c2:	ea41 5104 	orrgt.w	r1, r1, r4, lsl #20
 80009c6:	bd70      	popgt	{r4, r5, r6, pc}
 80009c8:	f441 1180 	orr.w	r1, r1, #1048576	; 0x100000
 80009cc:	f04f 0e00 	mov.w	lr, #0
 80009d0:	3c01      	subs	r4, #1
 80009d2:	e690      	b.n	80006f6 <__aeabi_dmul+0xde>
 80009d4:	ea45 0e06 	orr.w	lr, r5, r6
 80009d8:	e68d      	b.n	80006f6 <__aeabi_dmul+0xde>
 80009da:	ea0c 5513 	and.w	r5, ip, r3, lsr #20
 80009de:	ea94 0f0c 	teq	r4, ip
 80009e2:	bf08      	it	eq
 80009e4:	ea95 0f0c 	teqeq	r5, ip
 80009e8:	f43f af3b 	beq.w	8000862 <__aeabi_dmul+0x24a>
 80009ec:	ea94 0f0c 	teq	r4, ip
 80009f0:	d10a      	bne.n	8000a08 <__aeabi_ddiv+0x19c>
 80009f2:	ea50 3401 	orrs.w	r4, r0, r1, lsl #12
 80009f6:	f47f af34 	bne.w	8000862 <__aeabi_dmul+0x24a>
 80009fa:	ea95 0f0c 	teq	r5, ip
 80009fe:	f47f af25 	bne.w	800084c <__aeabi_dmul+0x234>
 8000a02:	4610      	mov	r0, r2
 8000a04:	4619      	mov	r1, r3
 8000a06:	e72c      	b.n	8000862 <__aeabi_dmul+0x24a>
 8000a08:	ea95 0f0c 	teq	r5, ip
 8000a0c:	d106      	bne.n	8000a1c <__aeabi_ddiv+0x1b0>
 8000a0e:	ea52 3503 	orrs.w	r5, r2, r3, lsl #12
 8000a12:	f43f aefd 	beq.w	8000810 <__aeabi_dmul+0x1f8>
 8000a16:	4610      	mov	r0, r2
 8000a18:	4619      	mov	r1, r3
 8000a1a:	e722      	b.n	8000862 <__aeabi_dmul+0x24a>
 8000a1c:	ea50 0641 	orrs.w	r6, r0, r1, lsl #1
 8000a20:	bf18      	it	ne
 8000a22:	ea52 0643 	orrsne.w	r6, r2, r3, lsl #1
 8000a26:	f47f aec5 	bne.w	80007b4 <__aeabi_dmul+0x19c>
 8000a2a:	ea50 0441 	orrs.w	r4, r0, r1, lsl #1
 8000a2e:	f47f af0d 	bne.w	800084c <__aeabi_dmul+0x234>
 8000a32:	ea52 0543 	orrs.w	r5, r2, r3, lsl #1
 8000a36:	f47f aeeb 	bne.w	8000810 <__aeabi_dmul+0x1f8>
 8000a3a:	e712      	b.n	8000862 <__aeabi_dmul+0x24a>

08000a3c <__gedf2>:
 8000a3c:	f04f 3cff 	mov.w	ip, #4294967295
 8000a40:	e006      	b.n	8000a50 <__cmpdf2+0x4>
 8000a42:	bf00      	nop

08000a44 <__ledf2>:
 8000a44:	f04f 0c01 	mov.w	ip, #1
 8000a48:	e002      	b.n	8000a50 <__cmpdf2+0x4>
 8000a4a:	bf00      	nop

08000a4c <__cmpdf2>:
 8000a4c:	f04f 0c01 	mov.w	ip, #1
 8000a50:	f84d cd04 	str.w	ip, [sp, #-4]!
 8000a54:	ea4f 0c41 	mov.w	ip, r1, lsl #1
 8000a58:	ea7f 5c6c 	mvns.w	ip, ip, asr #21
 8000a5c:	ea4f 0c43 	mov.w	ip, r3, lsl #1
 8000a60:	bf18      	it	ne
 8000a62:	ea7f 5c6c 	mvnsne.w	ip, ip, asr #21
 8000a66:	d01b      	beq.n	8000aa0 <__cmpdf2+0x54>
 8000a68:	b001      	add	sp, #4
 8000a6a:	ea50 0c41 	orrs.w	ip, r0, r1, lsl #1
 8000a6e:	bf0c      	ite	eq
 8000a70:	ea52 0c43 	orrseq.w	ip, r2, r3, lsl #1
 8000a74:	ea91 0f03 	teqne	r1, r3
 8000a78:	bf02      	ittt	eq
 8000a7a:	ea90 0f02 	teqeq	r0, r2
 8000a7e:	2000      	moveq	r0, #0
 8000a80:	4770      	bxeq	lr
 8000a82:	f110 0f00 	cmn.w	r0, #0
 8000a86:	ea91 0f03 	teq	r1, r3
 8000a8a:	bf58      	it	pl
 8000a8c:	4299      	cmppl	r1, r3
 8000a8e:	bf08      	it	eq
 8000a90:	4290      	cmpeq	r0, r2
 8000a92:	bf2c      	ite	cs
 8000a94:	17d8      	asrcs	r0, r3, #31
 8000a96:	ea6f 70e3 	mvncc.w	r0, r3, asr #31
 8000a9a:	f040 0001 	orr.w	r0, r0, #1
 8000a9e:	4770      	bx	lr
 8000aa0:	ea4f 0c41 	mov.w	ip, r1, lsl #1
 8000aa4:	ea7f 5c6c 	mvns.w	ip, ip, asr #21
 8000aa8:	d102      	bne.n	8000ab0 <__cmpdf2+0x64>
 8000aaa:	ea50 3c01 	orrs.w	ip, r0, r1, lsl #12
 8000aae:	d107      	bne.n	8000ac0 <__cmpdf2+0x74>
 8000ab0:	ea4f 0c43 	mov.w	ip, r3, lsl #1
 8000ab4:	ea7f 5c6c 	mvns.w	ip, ip, asr #21
 8000ab8:	d1d6      	bne.n	8000a68 <__cmpdf2+0x1c>
 8000aba:	ea52 3c03 	orrs.w	ip, r2, r3, lsl #12
 8000abe:	d0d3      	beq.n	8000a68 <__cmpdf2+0x1c>
 8000ac0:	f85d 0b04 	ldr.w	r0, [sp], #4
 8000ac4:	4770      	bx	lr
 8000ac6:	bf00      	nop

08000ac8 <__aeabi_cdrcmple>:
 8000ac8:	4684      	mov	ip, r0
 8000aca:	4610      	mov	r0, r2
 8000acc:	4662      	mov	r2, ip
 8000ace:	468c      	mov	ip, r1
 8000ad0:	4619      	mov	r1, r3
 8000ad2:	4663      	mov	r3, ip
 8000ad4:	e000      	b.n	8000ad8 <__aeabi_cdcmpeq>
 8000ad6:	bf00      	nop

08000ad8 <__aeabi_cdcmpeq>:
 8000ad8:	b501      	push	{r0, lr}
 8000ada:	f7ff ffb7 	bl	8000a4c <__cmpdf2>
 8000ade:	2800      	cmp	r0, #0
 8000ae0:	bf48      	it	mi
 8000ae2:	f110 0f00 	cmnmi.w	r0, #0
 8000ae6:	bd01      	pop	{r0, pc}

08000ae8 <__aeabi_dcmpeq>:
 8000ae8:	f84d ed08 	str.w	lr, [sp, #-8]!
 8000aec:	f7ff fff4 	bl	8000ad8 <__aeabi_cdcmpeq>
 8000af0:	bf0c      	ite	eq
 8000af2:	2001      	moveq	r0, #1
 8000af4:	2000      	movne	r0, #0
 8000af6:	f85d fb08 	ldr.w	pc, [sp], #8
 8000afa:	bf00      	nop

08000afc <__aeabi_dcmplt>:
 8000afc:	f84d ed08 	str.w	lr, [sp, #-8]!
 8000b00:	f7ff ffea 	bl	8000ad8 <__aeabi_cdcmpeq>
 8000b04:	bf34      	ite	cc
 8000b06:	2001      	movcc	r0, #1
 8000b08:	2000      	movcs	r0, #0
 8000b0a:	f85d fb08 	ldr.w	pc, [sp], #8
 8000b0e:	bf00      	nop

08000b10 <__aeabi_dcmple>:
 8000b10:	f84d ed08 	str.w	lr, [sp, #-8]!
 8000b14:	f7ff ffe0 	bl	8000ad8 <__aeabi_cdcmpeq>
 8000b18:	bf94      	ite	ls
 8000b1a:	2001      	movls	r0, #1
 8000b1c:	2000      	movhi	r0, #0
 8000b1e:	f85d fb08 	ldr.w	pc, [sp], #8
 8000b22:	bf00      	nop

08000b24 <__aeabi_dcmpge>:
 8000b24:	f84d ed08 	str.w	lr, [sp, #-8]!
 8000b28:	f7ff ffce 	bl	8000ac8 <__aeabi_cdrcmple>
 8000b2c:	bf94      	ite	ls
 8000b2e:	2001      	movls	r0, #1
 8000b30:	2000      	movhi	r0, #0
 8000b32:	f85d fb08 	ldr.w	pc, [sp], #8
 8000b36:	bf00      	nop

08000b38 <__aeabi_dcmpgt>:
 8000b38:	f84d ed08 	str.w	lr, [sp, #-8]!
 8000b3c:	f7ff ffc4 	bl	8000ac8 <__aeabi_cdrcmple>
 8000b40:	bf34      	ite	cc
 8000b42:	2001      	movcc	r0, #1
 8000b44:	2000      	movcs	r0, #0
 8000b46:	f85d fb08 	ldr.w	pc, [sp], #8
 8000b4a:	bf00      	nop

08000b4c <__aeabi_dcmpun>:
 8000b4c:	ea4f 0c41 	mov.w	ip, r1, lsl #1
 8000b50:	ea7f 5c6c 	mvns.w	ip, ip, asr #21
 8000b54:	d102      	bne.n	8000b5c <__aeabi_dcmpun+0x10>
 8000b56:	ea50 3c01 	orrs.w	ip, r0, r1, lsl #12
 8000b5a:	d10a      	bne.n	8000b72 <__aeabi_dcmpun+0x26>
 8000b5c:	ea4f 0c43 	mov.w	ip, r3, lsl #1
 8000b60:	ea7f 5c6c 	mvns.w	ip, ip, asr #21
 8000b64:	d102      	bne.n	8000b6c <__aeabi_dcmpun+0x20>
 8000b66:	ea52 3c03 	orrs.w	ip, r2, r3, lsl #12
 8000b6a:	d102      	bne.n	8000b72 <__aeabi_dcmpun+0x26>
 8000b6c:	f04f 0000 	mov.w	r0, #0
 8000b70:	4770      	bx	lr
 8000b72:	f04f 0001 	mov.w	r0, #1
 8000b76:	4770      	bx	lr

08000b78 <__aeabi_d2iz>:
 8000b78:	ea4f 0241 	mov.w	r2, r1, lsl #1
 8000b7c:	f512 1200 	adds.w	r2, r2, #2097152	; 0x200000
 8000b80:	d215      	bcs.n	8000bae <__aeabi_d2iz+0x36>
 8000b82:	d511      	bpl.n	8000ba8 <__aeabi_d2iz+0x30>
 8000b84:	f46f 7378 	mvn.w	r3, #992	; 0x3e0
 8000b88:	ebb3 5262 	subs.w	r2, r3, r2, asr #21
 8000b8c:	d912      	bls.n	8000bb4 <__aeabi_d2iz+0x3c>
 8000b8e:	ea4f 23c1 	mov.w	r3, r1, lsl #11
 8000b92:	f043 4300 	orr.w	r3, r3, #2147483648	; 0x80000000
 8000b96:	ea43 5350 	orr.w	r3, r3, r0, lsr #21
 8000b9a:	f011 4f00 	tst.w	r1, #2147483648	; 0x80000000
 8000b9e:	fa23 f002 	lsr.w	r0, r3, r2
 8000ba2:	bf18      	it	ne
 8000ba4:	4240      	negne	r0, r0
 8000ba6:	4770      	bx	lr
 8000ba8:	f04f 0000 	mov.w	r0, #0
 8000bac:	4770      	bx	lr
 8000bae:	ea50 3001 	orrs.w	r0, r0, r1, lsl #12
 8000bb2:	d105      	bne.n	8000bc0 <__aeabi_d2iz+0x48>
 8000bb4:	f011 4000 	ands.w	r0, r1, #2147483648	; 0x80000000
 8000bb8:	bf08      	it	eq
 8000bba:	f06f 4000 	mvneq.w	r0, #2147483648	; 0x80000000
 8000bbe:	4770      	bx	lr
 8000bc0:	f04f 0000 	mov.w	r0, #0
 8000bc4:	4770      	bx	lr
 8000bc6:	bf00      	nop

08000bc8 <__aeabi_d2f>:
 8000bc8:	ea4f 0241 	mov.w	r2, r1, lsl #1
 8000bcc:	f1b2 43e0 	subs.w	r3, r2, #1879048192	; 0x70000000
 8000bd0:	bf24      	itt	cs
 8000bd2:	f5b3 1c00 	subscs.w	ip, r3, #2097152	; 0x200000
 8000bd6:	f1dc 5cfe 	rsbscs	ip, ip, #532676608	; 0x1fc00000
 8000bda:	d90d      	bls.n	8000bf8 <__aeabi_d2f+0x30>
 8000bdc:	f001 4c00 	and.w	ip, r1, #2147483648	; 0x80000000
 8000be0:	ea4f 02c0 	mov.w	r2, r0, lsl #3
 8000be4:	ea4c 7050 	orr.w	r0, ip, r0, lsr #29
 8000be8:	f1b2 4f00 	cmp.w	r2, #2147483648	; 0x80000000
 8000bec:	eb40 0083 	adc.w	r0, r0, r3, lsl #2
 8000bf0:	bf08      	it	eq
 8000bf2:	f020 0001 	biceq.w	r0, r0, #1
 8000bf6:	4770      	bx	lr
 8000bf8:	f011 4f80 	tst.w	r1, #1073741824	; 0x40000000
 8000bfc:	d121      	bne.n	8000c42 <__aeabi_d2f+0x7a>
 8000bfe:	f113 7238 	adds.w	r2, r3, #48234496	; 0x2e00000
 8000c02:	bfbc      	itt	lt
 8000c04:	f001 4000 	andlt.w	r0, r1, #2147483648	; 0x80000000
 8000c08:	4770      	bxlt	lr
 8000c0a:	f441 1180 	orr.w	r1, r1, #1048576	; 0x100000
 8000c0e:	ea4f 5252 	mov.w	r2, r2, lsr #21
 8000c12:	f1c2 0218 	rsb	r2, r2, #24
 8000c16:	f1c2 0c20 	rsb	ip, r2, #32
 8000c1a:	fa10 f30c 	lsls.w	r3, r0, ip
 8000c1e:	fa20 f002 	lsr.w	r0, r0, r2
 8000c22:	bf18      	it	ne
 8000c24:	f040 0001 	orrne.w	r0, r0, #1
 8000c28:	ea4f 23c1 	mov.w	r3, r1, lsl #11
 8000c2c:	ea4f 23d3 	mov.w	r3, r3, lsr #11
 8000c30:	fa03 fc0c 	lsl.w	ip, r3, ip
 8000c34:	ea40 000c 	orr.w	r0, r0, ip
 8000c38:	fa23 f302 	lsr.w	r3, r3, r2
 8000c3c:	ea4f 0343 	mov.w	r3, r3, lsl #1
 8000c40:	e7cc      	b.n	8000bdc <__aeabi_d2f+0x14>
 8000c42:	ea7f 5362 	mvns.w	r3, r2, asr #21
 8000c46:	d107      	bne.n	8000c58 <__aeabi_d2f+0x90>
 8000c48:	ea50 3301 	orrs.w	r3, r0, r1, lsl #12
 8000c4c:	bf1e      	ittt	ne
 8000c4e:	f04f 40fe 	movne.w	r0, #2130706432	; 0x7f000000
 8000c52:	f440 0040 	orrne.w	r0, r0, #12582912	; 0xc00000
 8000c56:	4770      	bxne	lr
 8000c58:	f001 4000 	and.w	r0, r1, #2147483648	; 0x80000000
 8000c5c:	f040 40fe 	orr.w	r0, r0, #2130706432	; 0x7f000000
 8000c60:	f440 0000 	orr.w	r0, r0, #8388608	; 0x800000
 8000c64:	4770      	bx	lr
 8000c66:	bf00      	nop

08000c68 <__aeabi_uldivmod>:
 8000c68:	b953      	cbnz	r3, 8000c80 <__aeabi_uldivmod+0x18>
 8000c6a:	b94a      	cbnz	r2, 8000c80 <__aeabi_uldivmod+0x18>
 8000c6c:	2900      	cmp	r1, #0
 8000c6e:	bf08      	it	eq
 8000c70:	2800      	cmpeq	r0, #0
 8000c72:	bf1c      	itt	ne
 8000c74:	f04f 31ff 	movne.w	r1, #4294967295
 8000c78:	f04f 30ff 	movne.w	r0, #4294967295
 8000c7c:	f000 b974 	b.w	8000f68 <__aeabi_idiv0>
 8000c80:	f1ad 0c08 	sub.w	ip, sp, #8
 8000c84:	e96d ce04 	strd	ip, lr, [sp, #-16]!
 8000c88:	f000 f806 	bl	8000c98 <__udivmoddi4>
 8000c8c:	f8dd e004 	ldr.w	lr, [sp, #4]
 8000c90:	e9dd 2302 	ldrd	r2, r3, [sp, #8]
 8000c94:	b004      	add	sp, #16
 8000c96:	4770      	bx	lr

08000c98 <__udivmoddi4>:
 8000c98:	e92d 47f0 	stmdb	sp!, {r4, r5, r6, r7, r8, r9, sl, lr}
 8000c9c:	9d08      	ldr	r5, [sp, #32]
 8000c9e:	4604      	mov	r4, r0
 8000ca0:	468e      	mov	lr, r1
 8000ca2:	2b00      	cmp	r3, #0
 8000ca4:	d14d      	bne.n	8000d42 <__udivmoddi4+0xaa>
 8000ca6:	428a      	cmp	r2, r1
 8000ca8:	4694      	mov	ip, r2
 8000caa:	d969      	bls.n	8000d80 <__udivmoddi4+0xe8>
 8000cac:	fab2 f282 	clz	r2, r2
 8000cb0:	b152      	cbz	r2, 8000cc8 <__udivmoddi4+0x30>
 8000cb2:	fa01 f302 	lsl.w	r3, r1, r2
 8000cb6:	f1c2 0120 	rsb	r1, r2, #32
 8000cba:	fa20 f101 	lsr.w	r1, r0, r1
 8000cbe:	fa0c fc02 	lsl.w	ip, ip, r2
 8000cc2:	ea41 0e03 	orr.w	lr, r1, r3
 8000cc6:	4094      	lsls	r4, r2
 8000cc8:	ea4f 481c 	mov.w	r8, ip, lsr #16
 8000ccc:	0c21      	lsrs	r1, r4, #16
 8000cce:	fbbe f6f8 	udiv	r6, lr, r8
 8000cd2:	fa1f f78c 	uxth.w	r7, ip
 8000cd6:	fb08 e316 	mls	r3, r8, r6, lr
 8000cda:	ea41 4303 	orr.w	r3, r1, r3, lsl #16
 8000cde:	fb06 f107 	mul.w	r1, r6, r7
 8000ce2:	4299      	cmp	r1, r3
 8000ce4:	d90a      	bls.n	8000cfc <__udivmoddi4+0x64>
 8000ce6:	eb1c 0303 	adds.w	r3, ip, r3
 8000cea:	f106 30ff 	add.w	r0, r6, #4294967295
 8000cee:	f080 811f 	bcs.w	8000f30 <__udivmoddi4+0x298>
 8000cf2:	4299      	cmp	r1, r3
 8000cf4:	f240 811c 	bls.w	8000f30 <__udivmoddi4+0x298>
 8000cf8:	3e02      	subs	r6, #2
 8000cfa:	4463      	add	r3, ip
 8000cfc:	1a5b      	subs	r3, r3, r1
 8000cfe:	b2a4      	uxth	r4, r4
 8000d00:	fbb3 f0f8 	udiv	r0, r3, r8
 8000d04:	fb08 3310 	mls	r3, r8, r0, r3
 8000d08:	ea44 4403 	orr.w	r4, r4, r3, lsl #16
 8000d0c:	fb00 f707 	mul.w	r7, r0, r7
 8000d10:	42a7      	cmp	r7, r4
 8000d12:	d90a      	bls.n	8000d2a <__udivmoddi4+0x92>
 8000d14:	eb1c 0404 	adds.w	r4, ip, r4
 8000d18:	f100 33ff 	add.w	r3, r0, #4294967295
 8000d1c:	f080 810a 	bcs.w	8000f34 <__udivmoddi4+0x29c>
 8000d20:	42a7      	cmp	r7, r4
 8000d22:	f240 8107 	bls.w	8000f34 <__udivmoddi4+0x29c>
 8000d26:	4464      	add	r4, ip
 8000d28:	3802      	subs	r0, #2
 8000d2a:	ea40 4006 	orr.w	r0, r0, r6, lsl #16
 8000d2e:	1be4      	subs	r4, r4, r7
 8000d30:	2600      	movs	r6, #0
 8000d32:	b11d      	cbz	r5, 8000d3c <__udivmoddi4+0xa4>
 8000d34:	40d4      	lsrs	r4, r2
 8000d36:	2300      	movs	r3, #0
 8000d38:	e9c5 4300 	strd	r4, r3, [r5]
 8000d3c:	4631      	mov	r1, r6
 8000d3e:	e8bd 87f0 	ldmia.w	sp!, {r4, r5, r6, r7, r8, r9, sl, pc}
 8000d42:	428b      	cmp	r3, r1
 8000d44:	d909      	bls.n	8000d5a <__udivmoddi4+0xc2>
 8000d46:	2d00      	cmp	r5, #0
 8000d48:	f000 80ef 	beq.w	8000f2a <__udivmoddi4+0x292>
 8000d4c:	2600      	movs	r6, #0
 8000d4e:	e9c5 0100 	strd	r0, r1, [r5]
 8000d52:	4630      	mov	r0, r6
 8000d54:	4631      	mov	r1, r6
 8000d56:	e8bd 87f0 	ldmia.w	sp!, {r4, r5, r6, r7, r8, r9, sl, pc}
 8000d5a:	fab3 f683 	clz	r6, r3
 8000d5e:	2e00      	cmp	r6, #0
 8000d60:	d14a      	bne.n	8000df8 <__udivmoddi4+0x160>
 8000d62:	428b      	cmp	r3, r1
 8000d64:	d302      	bcc.n	8000d6c <__udivmoddi4+0xd4>
 8000d66:	4282      	cmp	r2, r0
 8000d68:	f200 80f9 	bhi.w	8000f5e <__udivmoddi4+0x2c6>
 8000d6c:	1a84      	subs	r4, r0, r2
 8000d6e:	eb61 0303 	sbc.w	r3, r1, r3
 8000d72:	2001      	movs	r0, #1
 8000d74:	469e      	mov	lr, r3
 8000d76:	2d00      	cmp	r5, #0
 8000d78:	d0e0      	beq.n	8000d3c <__udivmoddi4+0xa4>
 8000d7a:	e9c5 4e00 	strd	r4, lr, [r5]
 8000d7e:	e7dd      	b.n	8000d3c <__udivmoddi4+0xa4>
 8000d80:	b902      	cbnz	r2, 8000d84 <__udivmoddi4+0xec>
 8000d82:	deff      	udf	#255	; 0xff
 8000d84:	fab2 f282 	clz	r2, r2
 8000d88:	2a00      	cmp	r2, #0
 8000d8a:	f040 8092 	bne.w	8000eb2 <__udivmoddi4+0x21a>
 8000d8e:	eba1 010c 	sub.w	r1, r1, ip
 8000d92:	ea4f 471c 	mov.w	r7, ip, lsr #16
 8000d96:	fa1f fe8c 	uxth.w	lr, ip
 8000d9a:	2601      	movs	r6, #1
 8000d9c:	0c20      	lsrs	r0, r4, #16
 8000d9e:	fbb1 f3f7 	udiv	r3, r1, r7
 8000da2:	fb07 1113 	mls	r1, r7, r3, r1
 8000da6:	ea40 4101 	orr.w	r1, r0, r1, lsl #16
 8000daa:	fb0e f003 	mul.w	r0, lr, r3
 8000dae:	4288      	cmp	r0, r1
 8000db0:	d908      	bls.n	8000dc4 <__udivmoddi4+0x12c>
 8000db2:	eb1c 0101 	adds.w	r1, ip, r1
 8000db6:	f103 38ff 	add.w	r8, r3, #4294967295
 8000dba:	d202      	bcs.n	8000dc2 <__udivmoddi4+0x12a>
 8000dbc:	4288      	cmp	r0, r1
 8000dbe:	f200 80cb 	bhi.w	8000f58 <__udivmoddi4+0x2c0>
 8000dc2:	4643      	mov	r3, r8
 8000dc4:	1a09      	subs	r1, r1, r0
 8000dc6:	b2a4      	uxth	r4, r4
 8000dc8:	fbb1 f0f7 	udiv	r0, r1, r7
 8000dcc:	fb07 1110 	mls	r1, r7, r0, r1
 8000dd0:	ea44 4401 	orr.w	r4, r4, r1, lsl #16
 8000dd4:	fb0e fe00 	mul.w	lr, lr, r0
 8000dd8:	45a6      	cmp	lr, r4
 8000dda:	d908      	bls.n	8000dee <__udivmoddi4+0x156>
 8000ddc:	eb1c 0404 	adds.w	r4, ip, r4
 8000de0:	f100 31ff 	add.w	r1, r0, #4294967295
 8000de4:	d202      	bcs.n	8000dec <__udivmoddi4+0x154>
 8000de6:	45a6      	cmp	lr, r4
 8000de8:	f200 80bb 	bhi.w	8000f62 <__udivmoddi4+0x2ca>
 8000dec:	4608      	mov	r0, r1
 8000dee:	eba4 040e 	sub.w	r4, r4, lr
 8000df2:	ea40 4003 	orr.w	r0, r0, r3, lsl #16
 8000df6:	e79c      	b.n	8000d32 <__udivmoddi4+0x9a>
 8000df8:	f1c6 0720 	rsb	r7, r6, #32
 8000dfc:	40b3      	lsls	r3, r6
 8000dfe:	fa22 fc07 	lsr.w	ip, r2, r7
 8000e02:	ea4c 0c03 	orr.w	ip, ip, r3
 8000e06:	fa20 f407 	lsr.w	r4, r0, r7
 8000e0a:	fa01 f306 	lsl.w	r3, r1, r6
 8000e0e:	431c      	orrs	r4, r3
 8000e10:	40f9      	lsrs	r1, r7
 8000e12:	ea4f 491c 	mov.w	r9, ip, lsr #16
 8000e16:	fa00 f306 	lsl.w	r3, r0, r6
 8000e1a:	fbb1 f8f9 	udiv	r8, r1, r9
 8000e1e:	0c20      	lsrs	r0, r4, #16
 8000e20:	fa1f fe8c 	uxth.w	lr, ip
 8000e24:	fb09 1118 	mls	r1, r9, r8, r1
 8000e28:	ea40 4101 	orr.w	r1, r0, r1, lsl #16
 8000e2c:	fb08 f00e 	mul.w	r0, r8, lr
 8000e30:	4288      	cmp	r0, r1
 8000e32:	fa02 f206 	lsl.w	r2, r2, r6
 8000e36:	d90b      	bls.n	8000e50 <__udivmoddi4+0x1b8>
 8000e38:	eb1c 0101 	adds.w	r1, ip, r1
 8000e3c:	f108 3aff 	add.w	sl, r8, #4294967295
 8000e40:	f080 8088 	bcs.w	8000f54 <__udivmoddi4+0x2bc>
 8000e44:	4288      	cmp	r0, r1
 8000e46:	f240 8085 	bls.w	8000f54 <__udivmoddi4+0x2bc>
 8000e4a:	f1a8 0802 	sub.w	r8, r8, #2
 8000e4e:	4461      	add	r1, ip
 8000e50:	1a09      	subs	r1, r1, r0
 8000e52:	b2a4      	uxth	r4, r4
 8000e54:	fbb1 f0f9 	udiv	r0, r1, r9
 8000e58:	fb09 1110 	mls	r1, r9, r0, r1
 8000e5c:	ea44 4101 	orr.w	r1, r4, r1, lsl #16
 8000e60:	fb00 fe0e 	mul.w	lr, r0, lr
 8000e64:	458e      	cmp	lr, r1
 8000e66:	d908      	bls.n	8000e7a <__udivmoddi4+0x1e2>
 8000e68:	eb1c 0101 	adds.w	r1, ip, r1
 8000e6c:	f100 34ff 	add.w	r4, r0, #4294967295
 8000e70:	d26c      	bcs.n	8000f4c <__udivmoddi4+0x2b4>
 8000e72:	458e      	cmp	lr, r1
 8000e74:	d96a      	bls.n	8000f4c <__udivmoddi4+0x2b4>
 8000e76:	3802      	subs	r0, #2
 8000e78:	4461      	add	r1, ip
 8000e7a:	ea40 4008 	orr.w	r0, r0, r8, lsl #16
 8000e7e:	fba0 9402 	umull	r9, r4, r0, r2
 8000e82:	eba1 010e 	sub.w	r1, r1, lr
 8000e86:	42a1      	cmp	r1, r4
 8000e88:	46c8      	mov	r8, r9
 8000e8a:	46a6      	mov	lr, r4
 8000e8c:	d356      	bcc.n	8000f3c <__udivmoddi4+0x2a4>
 8000e8e:	d053      	beq.n	8000f38 <__udivmoddi4+0x2a0>
 8000e90:	b15d      	cbz	r5, 8000eaa <__udivmoddi4+0x212>
 8000e92:	ebb3 0208 	subs.w	r2, r3, r8
 8000e96:	eb61 010e 	sbc.w	r1, r1, lr
 8000e9a:	fa01 f707 	lsl.w	r7, r1, r7
 8000e9e:	fa22 f306 	lsr.w	r3, r2, r6
 8000ea2:	40f1      	lsrs	r1, r6
 8000ea4:	431f      	orrs	r7, r3
 8000ea6:	e9c5 7100 	strd	r7, r1, [r5]
 8000eaa:	2600      	movs	r6, #0
 8000eac:	4631      	mov	r1, r6
 8000eae:	e8bd 87f0 	ldmia.w	sp!, {r4, r5, r6, r7, r8, r9, sl, pc}
 8000eb2:	f1c2 0320 	rsb	r3, r2, #32
 8000eb6:	40d8      	lsrs	r0, r3
 8000eb8:	fa0c fc02 	lsl.w	ip, ip, r2
 8000ebc:	fa21 f303 	lsr.w	r3, r1, r3
 8000ec0:	4091      	lsls	r1, r2
 8000ec2:	4301      	orrs	r1, r0
 8000ec4:	ea4f 471c 	mov.w	r7, ip, lsr #16
 8000ec8:	fa1f fe8c 	uxth.w	lr, ip
 8000ecc:	fbb3 f0f7 	udiv	r0, r3, r7
 8000ed0:	fb07 3610 	mls	r6, r7, r0, r3
 8000ed4:	0c0b      	lsrs	r3, r1, #16
 8000ed6:	ea43 4306 	orr.w	r3, r3, r6, lsl #16
 8000eda:	fb00 f60e 	mul.w	r6, r0, lr
 8000ede:	429e      	cmp	r6, r3
 8000ee0:	fa04 f402 	lsl.w	r4, r4, r2
 8000ee4:	d908      	bls.n	8000ef8 <__udivmoddi4+0x260>
 8000ee6:	eb1c 0303 	adds.w	r3, ip, r3
 8000eea:	f100 38ff 	add.w	r8, r0, #4294967295
 8000eee:	d22f      	bcs.n	8000f50 <__udivmoddi4+0x2b8>
 8000ef0:	429e      	cmp	r6, r3
 8000ef2:	d92d      	bls.n	8000f50 <__udivmoddi4+0x2b8>
 8000ef4:	3802      	subs	r0, #2
 8000ef6:	4463      	add	r3, ip
 8000ef8:	1b9b      	subs	r3, r3, r6
 8000efa:	b289      	uxth	r1, r1
 8000efc:	fbb3 f6f7 	udiv	r6, r3, r7
 8000f00:	fb07 3316 	mls	r3, r7, r6, r3
 8000f04:	ea41 4103 	orr.w	r1, r1, r3, lsl #16
 8000f08:	fb06 f30e 	mul.w	r3, r6, lr
 8000f0c:	428b      	cmp	r3, r1
 8000f0e:	d908      	bls.n	8000f22 <__udivmoddi4+0x28a>
 8000f10:	eb1c 0101 	adds.w	r1, ip, r1
 8000f14:	f106 38ff 	add.w	r8, r6, #4294967295
 8000f18:	d216      	bcs.n	8000f48 <__udivmoddi4+0x2b0>
 8000f1a:	428b      	cmp	r3, r1
 8000f1c:	d914      	bls.n	8000f48 <__udivmoddi4+0x2b0>
 8000f1e:	3e02      	subs	r6, #2
 8000f20:	4461      	add	r1, ip
 8000f22:	1ac9      	subs	r1, r1, r3
 8000f24:	ea46 4600 	orr.w	r6, r6, r0, lsl #16
 8000f28:	e738      	b.n	8000d9c <__udivmoddi4+0x104>
 8000f2a:	462e      	mov	r6, r5
 8000f2c:	4628      	mov	r0, r5
 8000f2e:	e705      	b.n	8000d3c <__udivmoddi4+0xa4>
 8000f30:	4606      	mov	r6, r0
 8000f32:	e6e3      	b.n	8000cfc <__udivmoddi4+0x64>
 8000f34:	4618      	mov	r0, r3
 8000f36:	e6f8      	b.n	8000d2a <__udivmoddi4+0x92>
 8000f38:	454b      	cmp	r3, r9
 8000f3a:	d2a9      	bcs.n	8000e90 <__udivmoddi4+0x1f8>
 8000f3c:	ebb9 0802 	subs.w	r8, r9, r2
 8000f40:	eb64 0e0c 	sbc.w	lr, r4, ip
 8000f44:	3801      	subs	r0, #1
 8000f46:	e7a3      	b.n	8000e90 <__udivmoddi4+0x1f8>
 8000f48:	4646      	mov	r6, r8
 8000f4a:	e7ea      	b.n	8000f22 <__udivmoddi4+0x28a>
 8000f4c:	4620      	mov	r0, r4
 8000f4e:	e794      	b.n	8000e7a <__udivmoddi4+0x1e2>
 8000f50:	4640      	mov	r0, r8
 8000f52:	e7d1      	b.n	8000ef8 <__udivmoddi4+0x260>
 8000f54:	46d0      	mov	r8, sl
 8000f56:	e77b      	b.n	8000e50 <__udivmoddi4+0x1b8>
 8000f58:	3b02      	subs	r3, #2
 8000f5a:	4461      	add	r1, ip
 8000f5c:	e732      	b.n	8000dc4 <__udivmoddi4+0x12c>
 8000f5e:	4630      	mov	r0, r6
 8000f60:	e709      	b.n	8000d76 <__udivmoddi4+0xde>
 8000f62:	4464      	add	r4, ip
 8000f64:	3802      	subs	r0, #2
 8000f66:	e742      	b.n	8000dee <__udivmoddi4+0x156>

08000f68 <__aeabi_idiv0>:
 8000f68:	4770      	bx	lr
 8000f6a:	bf00      	nop

08000f6c <door>:

/* Private user code ---------------------------------------------------------*/
/* USER CODE BEGIN 0 */

void door(void)	// detection of the User button to active or disactive the door
{
 8000f6c:	b580      	push	{r7, lr}
 8000f6e:	b082      	sub	sp, #8
 8000f70:	af00      	add	r7, sp, #0
	uint16_t adc_val =0;
 8000f72:	2300      	movs	r3, #0
 8000f74:	80fb      	strh	r3, [r7, #6]
	if (HAL_ADC_PollForConversion(&hadc1, 10) == HAL_OK){
 8000f76:	210a      	movs	r1, #10
 8000f78:	481a      	ldr	r0, [pc, #104]	; (8000fe4 <door+0x78>)
 8000f7a:	f001 fad3 	bl	8002524 <HAL_ADC_PollForConversion>
 8000f7e:	4603      	mov	r3, r0
 8000f80:	2b00      	cmp	r3, #0
 8000f82:	d12b      	bne.n	8000fdc <door+0x70>
	 adc_val = HAL_ADC_GetValue(&hadc1);
 8000f84:	4817      	ldr	r0, [pc, #92]	; (8000fe4 <door+0x78>)
 8000f86:	f001 fb58 	bl	800263a <HAL_ADC_GetValue>
 8000f8a:	4603      	mov	r3, r0
 8000f8c:	80fb      	strh	r3, [r7, #6]

	 if(adc_val > 3900){
 8000f8e:	88fb      	ldrh	r3, [r7, #6]
 8000f90:	f640 723c 	movw	r2, #3900	; 0xf3c
 8000f94:	4293      	cmp	r3, r2
 8000f96:	d921      	bls.n	8000fdc <door+0x70>
		 HAL_GPIO_WritePin(Door_GPIO_Port, Door_Pin, GPIO_PIN_SET);
 8000f98:	2201      	movs	r2, #1
 8000f9a:	f44f 5180 	mov.w	r1, #4096	; 0x1000
 8000f9e:	4812      	ldr	r0, [pc, #72]	; (8000fe8 <door+0x7c>)
 8000fa0:	f002 fbb4 	bl	800370c <HAL_GPIO_WritePin>
		 HAL_GPIO_WritePin(Alert_GPIO_Port, Alert_Pin, GPIO_PIN_SET);
 8000fa4:	2201      	movs	r2, #1
 8000fa6:	f44f 4180 	mov.w	r1, #16384	; 0x4000
 8000faa:	480f      	ldr	r0, [pc, #60]	; (8000fe8 <door+0x7c>)
 8000fac:	f002 fbae 	bl	800370c <HAL_GPIO_WritePin>
		 printf("Door is open \r\n");
 8000fb0:	480e      	ldr	r0, [pc, #56]	; (8000fec <door+0x80>)
 8000fb2:	f005 fe11 	bl	8006bd8 <puts>
		 HAL_Delay(3000);
 8000fb6:	f640 30b8 	movw	r0, #3000	; 0xbb8
 8000fba:	f001 f979 	bl	80022b0 <HAL_Delay>
		 printf("Door is close \r\n");
 8000fbe:	480c      	ldr	r0, [pc, #48]	; (8000ff0 <door+0x84>)
 8000fc0:	f005 fe0a 	bl	8006bd8 <puts>
		 HAL_GPIO_WritePin(Door_GPIO_Port, Door_Pin, GPIO_PIN_RESET);
 8000fc4:	2200      	movs	r2, #0
 8000fc6:	f44f 5180 	mov.w	r1, #4096	; 0x1000
 8000fca:	4807      	ldr	r0, [pc, #28]	; (8000fe8 <door+0x7c>)
 8000fcc:	f002 fb9e 	bl	800370c <HAL_GPIO_WritePin>
		 HAL_GPIO_WritePin(Alert_GPIO_Port, Alert_Pin, GPIO_PIN_RESET);
 8000fd0:	2200      	movs	r2, #0
 8000fd2:	f44f 4180 	mov.w	r1, #16384	; 0x4000
 8000fd6:	4804      	ldr	r0, [pc, #16]	; (8000fe8 <door+0x7c>)
 8000fd8:	f002 fb98 	bl	800370c <HAL_GPIO_WritePin>

	 }

	}
}
 8000fdc:	bf00      	nop
 8000fde:	3708      	adds	r7, #8
 8000fe0:	46bd      	mov	sp, r7
 8000fe2:	bd80      	pop	{r7, pc}
 8000fe4:	200001f8 	.word	0x200001f8
 8000fe8:	40021800 	.word	0x40021800
 8000fec:	08008d58 	.word	0x08008d58
 8000ff0:	08008d68 	.word	0x08008d68

08000ff4 <heartbeat>:

void heartbeat(void) //   Heartbeat for the system
{
 8000ff4:	b580      	push	{r7, lr}
 8000ff6:	af00      	add	r7, sp, #0
	static uint32_t tick = 0;
	if(tick < HAL_GetTick()){
 8000ff8:	f001 f94e 	bl	8002298 <HAL_GetTick>
 8000ffc:	4602      	mov	r2, r0
 8000ffe:	4b0a      	ldr	r3, [pc, #40]	; (8001028 <heartbeat+0x34>)
 8001000:	681b      	ldr	r3, [r3, #0]
 8001002:	429a      	cmp	r2, r3
 8001004:	d90e      	bls.n	8001024 <heartbeat+0x30>
		tick = HAL_GetTick () + 1000;  // Get the period of 500 ms for the toggle LED.
 8001006:	f001 f947 	bl	8002298 <HAL_GetTick>
 800100a:	4603      	mov	r3, r0
 800100c:	f503 737a 	add.w	r3, r3, #1000	; 0x3e8
 8001010:	4a05      	ldr	r2, [pc, #20]	; (8001028 <heartbeat+0x34>)
 8001012:	6013      	str	r3, [r2, #0]
		HAL_ADC_Start(&hadc1);
 8001014:	4805      	ldr	r0, [pc, #20]	; (800102c <heartbeat+0x38>)
 8001016:	f001 f9b3 	bl	8002380 <HAL_ADC_Start>
		HAL_GPIO_TogglePin(Heartbeat_GPIO_Port, Heartbeat_Pin);
 800101a:	f44f 5100 	mov.w	r1, #8192	; 0x2000
 800101e:	4804      	ldr	r0, [pc, #16]	; (8001030 <heartbeat+0x3c>)
 8001020:	f002 fb8d 	bl	800373e <HAL_GPIO_TogglePin>
	}
}
 8001024:	bf00      	nop
 8001026:	bd80      	pop	{r7, pc}
 8001028:	20000384 	.word	0x20000384
 800102c:	200001f8 	.word	0x200001f8
 8001030:	40021800 	.word	0x40021800

08001034 <temp_meas>:

float temp_meas(uint32_t toggle_period_ms, uint8_t toogle_meas_enable )	       // read the sensor and take the temperature in degrees
{
 8001034:	b5b0      	push	{r4, r5, r7, lr}
 8001036:	b08e      	sub	sp, #56	; 0x38
 8001038:	af00      	add	r7, sp, #0
 800103a:	6078      	str	r0, [r7, #4]
 800103c:	460b      	mov	r3, r1
 800103e:	70fb      	strb	r3, [r7, #3]

	uint32_t meas_tick = 0;
 8001040:	2300      	movs	r3, #0
 8001042:	633b      	str	r3, [r7, #48]	; 0x30
	int32_t raw_temperature = 0;
 8001044:	2300      	movs	r3, #0
 8001046:	62fb      	str	r3, [r7, #44]	; 0x2c
	uint8_t spi_tx_data_meas_reg = 0x00;
 8001048:	2300      	movs	r3, #0
 800104a:	747b      	strb	r3, [r7, #17]
	uint8_t spi_rx_meas_data[6] = { 0x00 };
 800104c:	2300      	movs	r3, #0
 800104e:	60bb      	str	r3, [r7, #8]
 8001050:	2300      	movs	r3, #0
 8001052:	81bb      	strh	r3, [r7, #12]

	float temp_degr = 0;
 8001054:	f04f 0300 	mov.w	r3, #0
 8001058:	637b      	str	r3, [r7, #52]	; 0x34
	double var1 = 0;
 800105a:	f04f 0200 	mov.w	r2, #0
 800105e:	f04f 0300 	mov.w	r3, #0
 8001062:	e9c7 2308 	strd	r2, r3, [r7, #32]
	double var2 = 0;
 8001066:	f04f 0200 	mov.w	r2, #0
 800106a:	f04f 0300 	mov.w	r3, #0
 800106e:	e9c7 2306 	strd	r2, r3, [r7, #24]

	const uint16_t dig_T1 = 0b0110100110100011;
 8001072:	f646 13a3 	movw	r3, #27043	; 0x69a3
 8001076:	82fb      	strh	r3, [r7, #22]
	const int16_t dig_T2 = 0b0110101001000000;
 8001078:	f646 2340 	movw	r3, #27200	; 0x6a40
 800107c:	82bb      	strh	r3, [r7, #20]
	const int16_t dig_T3 = 0b1111110000011000;
 800107e:	f64f 4318 	movw	r3, #64536	; 0xfc18
 8001082:	827b      	strh	r3, [r7, #18]

	if (toogle_meas_enable) {
 8001084:	78fb      	ldrb	r3, [r7, #3]
 8001086:	2b00      	cmp	r3, #0
 8001088:	f000 80c5 	beq.w	8001216 <temp_meas+0x1e2>
				if ((HAL_GetTick() - meas_tick) > toggle_period_ms) {
 800108c:	f001 f904 	bl	8002298 <HAL_GetTick>
 8001090:	4602      	mov	r2, r0
 8001092:	6b3b      	ldr	r3, [r7, #48]	; 0x30
 8001094:	1ad3      	subs	r3, r2, r3
 8001096:	687a      	ldr	r2, [r7, #4]
 8001098:	429a      	cmp	r2, r3
 800109a:	f080 80bc 	bcs.w	8001216 <temp_meas+0x1e2>
					meas_tick = HAL_GetTick();				// Evaluate the period
 800109e:	f001 f8fb 	bl	8002298 <HAL_GetTick>
 80010a2:	6338      	str	r0, [r7, #48]	; 0x30

					///////////////// Take the temperature measurement /////////////////////////////////////////
					spi_tx_data_meas_reg = BMP280_REG_ADDR_TEMP_MSB;
 80010a4:	23fa      	movs	r3, #250	; 0xfa
 80010a6:	747b      	strb	r3, [r7, #17]
					HAL_GPIO_WritePin(bmp280_CS_GPIO_Port, bmp280_CS_Pin,GPIO_PIN_RESET);
 80010a8:	2200      	movs	r2, #0
 80010aa:	2110      	movs	r1, #16
 80010ac:	485e      	ldr	r0, [pc, #376]	; (8001228 <temp_meas+0x1f4>)
 80010ae:	f002 fb2d 	bl	800370c <HAL_GPIO_WritePin>
					if (HAL_SPI_Transmit(&hspi1, &spi_tx_data_meas_reg, 1, 10) == HAL_OK) {
 80010b2:	f107 0111 	add.w	r1, r7, #17
 80010b6:	230a      	movs	r3, #10
 80010b8:	2201      	movs	r2, #1
 80010ba:	485c      	ldr	r0, [pc, #368]	; (800122c <temp_meas+0x1f8>)
 80010bc:	f003 f87b 	bl	80041b6 <HAL_SPI_Transmit>
 80010c0:	4603      	mov	r3, r0
 80010c2:	2b00      	cmp	r3, #0
 80010c4:	f040 809e 	bne.w	8001204 <temp_meas+0x1d0>
						if (HAL_SPI_Receive(&hspi1, spi_rx_meas_data, 1, 10) == HAL_OK) {
 80010c8:	f107 0108 	add.w	r1, r7, #8
 80010cc:	230a      	movs	r3, #10
 80010ce:	2201      	movs	r2, #1
 80010d0:	4856      	ldr	r0, [pc, #344]	; (800122c <temp_meas+0x1f8>)
 80010d2:	f003 f9ac 	bl	800442e <HAL_SPI_Receive>
 80010d6:	4603      	mov	r3, r0
 80010d8:	2b00      	cmp	r3, #0
 80010da:	f040 8093 	bne.w	8001204 <temp_meas+0x1d0>
							HAL_Delay(10);
 80010de:	200a      	movs	r0, #10
 80010e0:	f001 f8e6 	bl	80022b0 <HAL_Delay>
							raw_temperature =(int32_t) (spi_rx_meas_data[2] & 0b00001111) | (spi_rx_meas_data[1] << 4) | (spi_rx_meas_data[0] << 12);
 80010e4:	7abb      	ldrb	r3, [r7, #10]
 80010e6:	f003 020f 	and.w	r2, r3, #15
 80010ea:	7a7b      	ldrb	r3, [r7, #9]
 80010ec:	011b      	lsls	r3, r3, #4
 80010ee:	431a      	orrs	r2, r3
 80010f0:	7a3b      	ldrb	r3, [r7, #8]
 80010f2:	031b      	lsls	r3, r3, #12
 80010f4:	4313      	orrs	r3, r2
 80010f6:	62fb      	str	r3, [r7, #44]	; 0x2c

							/////////////////////////////////////// Implementation of the transformation equation /////////////////////////////////
							var1 = (((double) raw_temperature) / 16384.0 - ((double) dig_T1) / 1024.0) * ((double) dig_T2);
 80010f8:	6af8      	ldr	r0, [r7, #44]	; 0x2c
 80010fa:	f7ff fa23 	bl	8000544 <__aeabi_i2d>
 80010fe:	f04f 0200 	mov.w	r2, #0
 8001102:	4b4b      	ldr	r3, [pc, #300]	; (8001230 <temp_meas+0x1fc>)
 8001104:	f7ff fbb2 	bl	800086c <__aeabi_ddiv>
 8001108:	4602      	mov	r2, r0
 800110a:	460b      	mov	r3, r1
 800110c:	4614      	mov	r4, r2
 800110e:	461d      	mov	r5, r3
 8001110:	8afb      	ldrh	r3, [r7, #22]
 8001112:	4618      	mov	r0, r3
 8001114:	f7ff fa06 	bl	8000524 <__aeabi_ui2d>
 8001118:	f04f 0200 	mov.w	r2, #0
 800111c:	4b45      	ldr	r3, [pc, #276]	; (8001234 <temp_meas+0x200>)
 800111e:	f7ff fba5 	bl	800086c <__aeabi_ddiv>
 8001122:	4602      	mov	r2, r0
 8001124:	460b      	mov	r3, r1
 8001126:	4620      	mov	r0, r4
 8001128:	4629      	mov	r1, r5
 800112a:	f7ff f8bd 	bl	80002a8 <__aeabi_dsub>
 800112e:	4602      	mov	r2, r0
 8001130:	460b      	mov	r3, r1
 8001132:	4614      	mov	r4, r2
 8001134:	461d      	mov	r5, r3
 8001136:	f9b7 3014 	ldrsh.w	r3, [r7, #20]
 800113a:	4618      	mov	r0, r3
 800113c:	f7ff fa02 	bl	8000544 <__aeabi_i2d>
 8001140:	4602      	mov	r2, r0
 8001142:	460b      	mov	r3, r1
 8001144:	4620      	mov	r0, r4
 8001146:	4629      	mov	r1, r5
 8001148:	f7ff fa66 	bl	8000618 <__aeabi_dmul>
 800114c:	4602      	mov	r2, r0
 800114e:	460b      	mov	r3, r1
 8001150:	e9c7 2308 	strd	r2, r3, [r7, #32]
							var2 = ((double) raw_temperature) / 131072.0 - ((double) dig_T1) / 8192.0;
 8001154:	6af8      	ldr	r0, [r7, #44]	; 0x2c
 8001156:	f7ff f9f5 	bl	8000544 <__aeabi_i2d>
 800115a:	f04f 0200 	mov.w	r2, #0
 800115e:	f04f 4382 	mov.w	r3, #1090519040	; 0x41000000
 8001162:	f7ff fb83 	bl	800086c <__aeabi_ddiv>
 8001166:	4602      	mov	r2, r0
 8001168:	460b      	mov	r3, r1
 800116a:	4614      	mov	r4, r2
 800116c:	461d      	mov	r5, r3
 800116e:	8afb      	ldrh	r3, [r7, #22]
 8001170:	4618      	mov	r0, r3
 8001172:	f7ff f9d7 	bl	8000524 <__aeabi_ui2d>
 8001176:	f04f 0200 	mov.w	r2, #0
 800117a:	4b2f      	ldr	r3, [pc, #188]	; (8001238 <temp_meas+0x204>)
 800117c:	f7ff fb76 	bl	800086c <__aeabi_ddiv>
 8001180:	4602      	mov	r2, r0
 8001182:	460b      	mov	r3, r1
 8001184:	4620      	mov	r0, r4
 8001186:	4629      	mov	r1, r5
 8001188:	f7ff f88e 	bl	80002a8 <__aeabi_dsub>
 800118c:	4602      	mov	r2, r0
 800118e:	460b      	mov	r3, r1
 8001190:	e9c7 2306 	strd	r2, r3, [r7, #24]
							var2 = (var2 * var2) * ((double) dig_T3);
 8001194:	e9d7 2306 	ldrd	r2, r3, [r7, #24]
 8001198:	e9d7 0106 	ldrd	r0, r1, [r7, #24]
 800119c:	f7ff fa3c 	bl	8000618 <__aeabi_dmul>
 80011a0:	4602      	mov	r2, r0
 80011a2:	460b      	mov	r3, r1
 80011a4:	4614      	mov	r4, r2
 80011a6:	461d      	mov	r5, r3
 80011a8:	f9b7 3012 	ldrsh.w	r3, [r7, #18]
 80011ac:	4618      	mov	r0, r3
 80011ae:	f7ff f9c9 	bl	8000544 <__aeabi_i2d>
 80011b2:	4602      	mov	r2, r0
 80011b4:	460b      	mov	r3, r1
 80011b6:	4620      	mov	r0, r4
 80011b8:	4629      	mov	r1, r5
 80011ba:	f7ff fa2d 	bl	8000618 <__aeabi_dmul>
 80011be:	4602      	mov	r2, r0
 80011c0:	460b      	mov	r3, r1
 80011c2:	e9c7 2306 	strd	r2, r3, [r7, #24]
							temp_degr = (float) (var1 + var2) / 5120.0;
 80011c6:	e9d7 2306 	ldrd	r2, r3, [r7, #24]
 80011ca:	e9d7 0108 	ldrd	r0, r1, [r7, #32]
 80011ce:	f7ff f86d 	bl	80002ac <__adddf3>
 80011d2:	4602      	mov	r2, r0
 80011d4:	460b      	mov	r3, r1
 80011d6:	4610      	mov	r0, r2
 80011d8:	4619      	mov	r1, r3
 80011da:	f7ff fcf5 	bl	8000bc8 <__aeabi_d2f>
 80011de:	ee06 0a90 	vmov	s13, r0
 80011e2:	ed9f 7a16 	vldr	s14, [pc, #88]	; 800123c <temp_meas+0x208>
 80011e6:	eec6 7a87 	vdiv.f32	s15, s13, s14
 80011ea:	edc7 7a0d 	vstr	s15, [r7, #52]	; 0x34

							/////////////////////////////////////////////// Send the value of the degrees on the UART /////////////////////////////////
							printf("Temp: %.2f",temp_degr);
 80011ee:	6b78      	ldr	r0, [r7, #52]	; 0x34
 80011f0:	f7ff f9ba 	bl	8000568 <__aeabi_f2d>
 80011f4:	4602      	mov	r2, r0
 80011f6:	460b      	mov	r3, r1
 80011f8:	4811      	ldr	r0, [pc, #68]	; (8001240 <temp_meas+0x20c>)
 80011fa:	f005 fc67 	bl	8006acc <iprintf>
							printf("°C\r\n");
 80011fe:	4811      	ldr	r0, [pc, #68]	; (8001244 <temp_meas+0x210>)
 8001200:	f005 fcea 	bl	8006bd8 <puts>
						  }
					  }
						HAL_GPIO_WritePin(bmp280_CS_GPIO_Port, bmp280_CS_Pin,GPIO_PIN_SET);
 8001204:	2201      	movs	r2, #1
 8001206:	2110      	movs	r1, #16
 8001208:	4807      	ldr	r0, [pc, #28]	; (8001228 <temp_meas+0x1f4>)
 800120a:	f002 fa7f 	bl	800370c <HAL_GPIO_WritePin>
						HAL_Delay(1000);
 800120e:	f44f 707a 	mov.w	r0, #1000	; 0x3e8
 8001212:	f001 f84d 	bl	80022b0 <HAL_Delay>
					 }
				  }
	return temp_degr;
 8001216:	6b7b      	ldr	r3, [r7, #52]	; 0x34
 8001218:	ee07 3a90 	vmov	s15, r3
}
 800121c:	eeb0 0a67 	vmov.f32	s0, s15
 8001220:	3738      	adds	r7, #56	; 0x38
 8001222:	46bd      	mov	sp, r7
 8001224:	bdb0      	pop	{r4, r5, r7, pc}
 8001226:	bf00      	nop
 8001228:	40020800 	.word	0x40020800
 800122c:	20000240 	.word	0x20000240
 8001230:	40d00000 	.word	0x40d00000
 8001234:	40900000 	.word	0x40900000
 8001238:	40c00000 	.word	0x40c00000
 800123c:	45a00000 	.word	0x45a00000
 8001240:	08008d78 	.word	0x08008d78
 8001244:	08008d84 	.word	0x08008d84

08001248 <PWM_DMA>:

void PWM_DMA(float lim_initial, float lim_final)							  // Produce the PWM signal
{
 8001248:	b5b0      	push	{r4, r5, r7, lr}
 800124a:	f5ad 6d01 	sub.w	sp, sp, #2064	; 0x810
 800124e:	af00      	add	r7, sp, #0
 8001250:	f507 6301 	add.w	r3, r7, #2064	; 0x810
 8001254:	f6a3 030c 	subw	r3, r3, #2060	; 0x80c
 8001258:	ed83 0a00 	vstr	s0, [r3]
 800125c:	f507 6301 	add.w	r3, r7, #2064	; 0x810
 8001260:	f5a3 6301 	sub.w	r3, r3, #2064	; 0x810
 8001264:	edc3 0a00 	vstr	s1, [r3]
	uint16_t pwm_dma[Buffer_PWM_size] = { 0 };								  // Buffer for PWM data
 8001268:	f507 6301 	add.w	r3, r7, #2064	; 0x810
 800126c:	f6a3 0308 	subw	r3, r3, #2056	; 0x808
 8001270:	4618      	mov	r0, r3
 8001272:	f44f 6300 	mov.w	r3, #2048	; 0x800
 8001276:	461a      	mov	r2, r3
 8001278:	2100      	movs	r1, #0
 800127a:	f004 ffb5 	bl	80061e8 <memset>
	const float step = (1023.0 * lim_final - 1023.0 * lim_initial )/ 1023.0;  // calculate the value of the step of each iteration
 800127e:	f507 6301 	add.w	r3, r7, #2064	; 0x810
 8001282:	f5a3 6301 	sub.w	r3, r3, #2064	; 0x810
 8001286:	6818      	ldr	r0, [r3, #0]
 8001288:	f7ff f96e 	bl	8000568 <__aeabi_f2d>
 800128c:	a33d      	add	r3, pc, #244	; (adr r3, 8001384 <PWM_DMA+0x13c>)
 800128e:	e9d3 2300 	ldrd	r2, r3, [r3]
 8001292:	f7ff f9c1 	bl	8000618 <__aeabi_dmul>
 8001296:	4602      	mov	r2, r0
 8001298:	460b      	mov	r3, r1
 800129a:	4614      	mov	r4, r2
 800129c:	461d      	mov	r5, r3
 800129e:	f507 6301 	add.w	r3, r7, #2064	; 0x810
 80012a2:	f6a3 030c 	subw	r3, r3, #2060	; 0x80c
 80012a6:	6818      	ldr	r0, [r3, #0]
 80012a8:	f7ff f95e 	bl	8000568 <__aeabi_f2d>
 80012ac:	a335      	add	r3, pc, #212	; (adr r3, 8001384 <PWM_DMA+0x13c>)
 80012ae:	e9d3 2300 	ldrd	r2, r3, [r3]
 80012b2:	f7ff f9b1 	bl	8000618 <__aeabi_dmul>
 80012b6:	4602      	mov	r2, r0
 80012b8:	460b      	mov	r3, r1
 80012ba:	4620      	mov	r0, r4
 80012bc:	4629      	mov	r1, r5
 80012be:	f7fe fff3 	bl	80002a8 <__aeabi_dsub>
 80012c2:	4602      	mov	r2, r0
 80012c4:	460b      	mov	r3, r1
 80012c6:	4610      	mov	r0, r2
 80012c8:	4619      	mov	r1, r3
 80012ca:	a32e      	add	r3, pc, #184	; (adr r3, 8001384 <PWM_DMA+0x13c>)
 80012cc:	e9d3 2300 	ldrd	r2, r3, [r3]
 80012d0:	f7ff facc 	bl	800086c <__aeabi_ddiv>
 80012d4:	4602      	mov	r2, r0
 80012d6:	460b      	mov	r3, r1
 80012d8:	4610      	mov	r0, r2
 80012da:	4619      	mov	r1, r3
 80012dc:	f7ff fc74 	bl	8000bc8 <__aeabi_d2f>
 80012e0:	4603      	mov	r3, r0
 80012e2:	f607 0208 	addw	r2, r7, #2056	; 0x808
 80012e6:	6013      	str	r3, [r2, #0]

	for (uint16_t i = 0; i < Buffer_PWM_size; i++) { 						  // PWM of DMA was initialized
 80012e8:	2300      	movs	r3, #0
 80012ea:	f8a7 380e 	strh.w	r3, [r7, #2062]	; 0x80e
 80012ee:	e033      	b.n	8001358 <PWM_DMA+0x110>
		pwm_dma[i] = (int)(1023.0 * lim_initial)+ (int) (step * i); 		  // save the value of the PWM in the actual step
 80012f0:	f507 6301 	add.w	r3, r7, #2064	; 0x810
 80012f4:	f6a3 030c 	subw	r3, r3, #2060	; 0x80c
 80012f8:	6818      	ldr	r0, [r3, #0]
 80012fa:	f7ff f935 	bl	8000568 <__aeabi_f2d>
 80012fe:	a321      	add	r3, pc, #132	; (adr r3, 8001384 <PWM_DMA+0x13c>)
 8001300:	e9d3 2300 	ldrd	r2, r3, [r3]
 8001304:	f7ff f988 	bl	8000618 <__aeabi_dmul>
 8001308:	4602      	mov	r2, r0
 800130a:	460b      	mov	r3, r1
 800130c:	4610      	mov	r0, r2
 800130e:	4619      	mov	r1, r3
 8001310:	f7ff fc32 	bl	8000b78 <__aeabi_d2iz>
 8001314:	4603      	mov	r3, r0
 8001316:	b299      	uxth	r1, r3
 8001318:	f8b7 380e 	ldrh.w	r3, [r7, #2062]	; 0x80e
 800131c:	ee07 3a90 	vmov	s15, r3
 8001320:	eeb8 7ae7 	vcvt.f32.s32	s14, s15
 8001324:	f607 0308 	addw	r3, r7, #2056	; 0x808
 8001328:	edd3 7a00 	vldr	s15, [r3]
 800132c:	ee67 7a27 	vmul.f32	s15, s14, s15
 8001330:	eefd 7ae7 	vcvt.s32.f32	s15, s15
 8001334:	ee17 3a90 	vmov	r3, s15
 8001338:	b29b      	uxth	r3, r3
 800133a:	f8b7 280e 	ldrh.w	r2, [r7, #2062]	; 0x80e
 800133e:	440b      	add	r3, r1
 8001340:	b299      	uxth	r1, r3
 8001342:	f507 6301 	add.w	r3, r7, #2064	; 0x810
 8001346:	f6a3 0308 	subw	r3, r3, #2056	; 0x808
 800134a:	f823 1012 	strh.w	r1, [r3, r2, lsl #1]
	for (uint16_t i = 0; i < Buffer_PWM_size; i++) { 						  // PWM of DMA was initialized
 800134e:	f8b7 380e 	ldrh.w	r3, [r7, #2062]	; 0x80e
 8001352:	3301      	adds	r3, #1
 8001354:	f8a7 380e 	strh.w	r3, [r7, #2062]	; 0x80e
 8001358:	f8b7 380e 	ldrh.w	r3, [r7, #2062]	; 0x80e
 800135c:	f5b3 6f80 	cmp.w	r3, #1024	; 0x400
 8001360:	d3c6      	bcc.n	80012f0 <PWM_DMA+0xa8>
	}

	HAL_TIM_PWM_Start_DMA(&htim1, TIM_CHANNEL_1, (uint32_t*) pwm_dma,Buffer_PWM_size);	// Put the buffer on the DMA to the timer PWM
 8001362:	f107 0208 	add.w	r2, r7, #8
 8001366:	f44f 6380 	mov.w	r3, #1024	; 0x400
 800136a:	2100      	movs	r1, #0
 800136c:	4804      	ldr	r0, [pc, #16]	; (8001380 <PWM_DMA+0x138>)
 800136e:	f003 fc91 	bl	8004c94 <HAL_TIM_PWM_Start_DMA>
}
 8001372:	bf00      	nop
 8001374:	f507 6701 	add.w	r7, r7, #2064	; 0x810
 8001378:	46bd      	mov	sp, r7
 800137a:	bdb0      	pop	{r4, r5, r7, pc}
 800137c:	f3af 8000 	nop.w
 8001380:	20000298 	.word	0x20000298
 8001384:	00000000 	.word	0x00000000
 8001388:	408ff800 	.word	0x408ff800

0800138c <_write>:

int _write(int file, char *ptr, int len) // Use the Wirte function to the UART1
{
 800138c:	b580      	push	{r7, lr}
 800138e:	b084      	sub	sp, #16
 8001390:	af00      	add	r7, sp, #0
 8001392:	60f8      	str	r0, [r7, #12]
 8001394:	60b9      	str	r1, [r7, #8]
 8001396:	607a      	str	r2, [r7, #4]
	HAL_UART_Transmit(&huart1,(uint8_t *)ptr, len, 10);
 8001398:	687b      	ldr	r3, [r7, #4]
 800139a:	b29a      	uxth	r2, r3
 800139c:	230a      	movs	r3, #10
 800139e:	68b9      	ldr	r1, [r7, #8]
 80013a0:	4803      	ldr	r0, [pc, #12]	; (80013b0 <_write+0x24>)
 80013a2:	f004 fb82 	bl	8005aaa <HAL_UART_Transmit>
	return len;
 80013a6:	687b      	ldr	r3, [r7, #4]
}
 80013a8:	4618      	mov	r0, r3
 80013aa:	3710      	adds	r7, #16
 80013ac:	46bd      	mov	sp, r7
 80013ae:	bd80      	pop	{r7, pc}
 80013b0:	20000340 	.word	0x20000340

080013b4 <main>:
 *
  * @brief  The application entry point.
  * @retval int
  */
int main(void)
{
 80013b4:	b580      	push	{r7, lr}
 80013b6:	b086      	sub	sp, #24
 80013b8:	af00      	add	r7, sp, #0
  /* USER CODE END 1 */

  /* MCU Configuration--------------------------------------------------------*/

  /* Reset of all peripherals, Initializes the Flash interface and the Systick. */
  HAL_Init();
 80013ba:	f000 ff07 	bl	80021cc <HAL_Init>
  /* USER CODE BEGIN Init */

  /* USER CODE END Init */

  /* Configure the system clock */
  SystemClock_Config();
 80013be:	f000 fa13 	bl	80017e8 <SystemClock_Config>
  /* USER CODE BEGIN SysInit */

  /* USER CODE END SysInit */

  /* Initialize all configured peripherals */
  MX_GPIO_Init();
 80013c2:	f000 fbd3 	bl	8001b6c <MX_GPIO_Init>
  MX_DMA_Init();
 80013c6:	f000 fbb1 	bl	8001b2c <MX_DMA_Init>
  MX_ADC1_Init();
 80013ca:	f000 fa79 	bl	80018c0 <MX_ADC1_Init>
  MX_TIM1_Init();
 80013ce:	f000 faff 	bl	80019d0 <MX_TIM1_Init>
  MX_SPI1_Init();
 80013d2:	f000 fac7 	bl	8001964 <MX_SPI1_Init>
  MX_USART1_UART_Init();
 80013d6:	f000 fb7f 	bl	8001ad8 <MX_USART1_UART_Init>
  /* USER CODE BEGIN 2 */

  ////////////////////// Variables ///////////////////////

  uint8_t spi_tx_data_reg = 0x00;			// Address of the registers for the bmp280 sensor
 80013da:	2300      	movs	r3, #0
 80013dc:	72bb      	strb	r3, [r7, #10]
  uint8_t spi_rx_data[6] = { 0x00 };		// Buffer of the sensor
 80013de:	2300      	movs	r3, #0
 80013e0:	607b      	str	r3, [r7, #4]
 80013e2:	2300      	movs	r3, #0
 80013e4:	813b      	strh	r3, [r7, #8]
  uint8_t toogle_meas_enable = 1;			// enable the sensor
 80013e6:	2301      	movs	r3, #1
 80013e8:	75bb      	strb	r3, [r7, #22]
  uint32_t toggle_period_ms = 1000;			// Period of the reading temperature
 80013ea:	f44f 737a 	mov.w	r3, #1000	; 0x3e8
 80013ee:	613b      	str	r3, [r7, #16]

  char state = 0;							// Initial state of the state machine
 80013f0:	2300      	movs	r3, #0
 80013f2:	75fb      	strb	r3, [r7, #23]
  float temp = 0.0;							// Temperature in degrees
 80013f4:	f04f 0300 	mov.w	r3, #0
 80013f8:	60fb      	str	r3, [r7, #12]



  ///////////////////////////////////////// Configuration of the BMP280 temperature sensor ///////////////////////////////
  // Search the sensor ID
  spi_tx_data_reg = BMP280_REG_ADDR_ID;
 80013fa:	23d0      	movs	r3, #208	; 0xd0
 80013fc:	72bb      	strb	r3, [r7, #10]
  HAL_GPIO_WritePin(bmp280_CS_GPIO_Port, bmp280_CS_Pin, GPIO_PIN_RESET);
 80013fe:	2200      	movs	r2, #0
 8001400:	2110      	movs	r1, #16
 8001402:	48ce      	ldr	r0, [pc, #824]	; (800173c <main+0x388>)
 8001404:	f002 f982 	bl	800370c <HAL_GPIO_WritePin>
  if (HAL_SPI_Transmit(&hspi1, &spi_tx_data_reg, 1, 10) == HAL_OK) {
 8001408:	f107 010a 	add.w	r1, r7, #10
 800140c:	230a      	movs	r3, #10
 800140e:	2201      	movs	r2, #1
 8001410:	48cb      	ldr	r0, [pc, #812]	; (8001740 <main+0x38c>)
 8001412:	f002 fed0 	bl	80041b6 <HAL_SPI_Transmit>
 8001416:	4603      	mov	r3, r0
 8001418:	2b00      	cmp	r3, #0
 800141a:	d10b      	bne.n	8001434 <main+0x80>
  	if (HAL_SPI_Receive(&hspi1, spi_rx_data, 1, 10) == HAL_OK) {
 800141c:	1d39      	adds	r1, r7, #4
 800141e:	230a      	movs	r3, #10
 8001420:	2201      	movs	r2, #1
 8001422:	48c7      	ldr	r0, [pc, #796]	; (8001740 <main+0x38c>)
 8001424:	f003 f803 	bl	800442e <HAL_SPI_Receive>
 8001428:	4603      	mov	r3, r0
 800142a:	2b00      	cmp	r3, #0
 800142c:	d102      	bne.n	8001434 <main+0x80>
  		HAL_Delay(10);
 800142e:	200a      	movs	r0, #10
 8001430:	f000 ff3e 	bl	80022b0 <HAL_Delay>
  	}
  }
  HAL_GPIO_WritePin(bmp280_CS_GPIO_Port, bmp280_CS_Pin, GPIO_PIN_SET);
 8001434:	2201      	movs	r2, #1
 8001436:	2110      	movs	r1, #16
 8001438:	48c0      	ldr	r0, [pc, #768]	; (800173c <main+0x388>)
 800143a:	f002 f967 	bl	800370c <HAL_GPIO_WritePin>

  // Change the Config sensor (temp over samp x2, skipped the press meas, normal power mode)
  uint8_t ctrl_meas_Bytes = 0x23;
 800143e:	2323      	movs	r3, #35	; 0x23
 8001440:	72fb      	strb	r3, [r7, #11]
  uint8_t spi_config[2] = { 0x74, ctrl_meas_Bytes };
 8001442:	2374      	movs	r3, #116	; 0x74
 8001444:	703b      	strb	r3, [r7, #0]
 8001446:	7afb      	ldrb	r3, [r7, #11]
 8001448:	707b      	strb	r3, [r7, #1]

  HAL_GPIO_WritePin(bmp280_CS_GPIO_Port, bmp280_CS_Pin, GPIO_PIN_RESET);
 800144a:	2200      	movs	r2, #0
 800144c:	2110      	movs	r1, #16
 800144e:	48bb      	ldr	r0, [pc, #748]	; (800173c <main+0x388>)
 8001450:	f002 f95c 	bl	800370c <HAL_GPIO_WritePin>
  if (HAL_SPI_Transmit(&hspi1, spi_config, 2, 10) == HAL_OK) {
 8001454:	4639      	mov	r1, r7
 8001456:	230a      	movs	r3, #10
 8001458:	2202      	movs	r2, #2
 800145a:	48b9      	ldr	r0, [pc, #740]	; (8001740 <main+0x38c>)
 800145c:	f002 feab 	bl	80041b6 <HAL_SPI_Transmit>
 8001460:	4603      	mov	r3, r0
 8001462:	2b00      	cmp	r3, #0
 8001464:	d102      	bne.n	800146c <main+0xb8>
  	HAL_Delay(10);
 8001466:	200a      	movs	r0, #10
 8001468:	f000 ff22 	bl	80022b0 <HAL_Delay>
  }
  HAL_GPIO_WritePin(bmp280_CS_GPIO_Port, bmp280_CS_Pin, GPIO_PIN_SET);
 800146c:	2201      	movs	r2, #1
 800146e:	2110      	movs	r1, #16
 8001470:	48b2      	ldr	r0, [pc, #712]	; (800173c <main+0x388>)
 8001472:	f002 f94b 	bl	800370c <HAL_GPIO_WritePin>

  // Verify the CTRL_MEAS register configuration
  spi_tx_data_reg = BMP280_REG_ADDR_CTRL_MEAS;
 8001476:	23f4      	movs	r3, #244	; 0xf4
 8001478:	72bb      	strb	r3, [r7, #10]
  HAL_GPIO_WritePin(bmp280_CS_GPIO_Port, bmp280_CS_Pin, GPIO_PIN_RESET);
 800147a:	2200      	movs	r2, #0
 800147c:	2110      	movs	r1, #16
 800147e:	48af      	ldr	r0, [pc, #700]	; (800173c <main+0x388>)
 8001480:	f002 f944 	bl	800370c <HAL_GPIO_WritePin>
  if (HAL_SPI_Transmit(&hspi1, &spi_tx_data_reg, 1, 10) == HAL_OK) {
 8001484:	f107 010a 	add.w	r1, r7, #10
 8001488:	230a      	movs	r3, #10
 800148a:	2201      	movs	r2, #1
 800148c:	48ac      	ldr	r0, [pc, #688]	; (8001740 <main+0x38c>)
 800148e:	f002 fe92 	bl	80041b6 <HAL_SPI_Transmit>
 8001492:	4603      	mov	r3, r0
 8001494:	2b00      	cmp	r3, #0
 8001496:	d10b      	bne.n	80014b0 <main+0xfc>
  	if (HAL_SPI_Receive(&hspi1, spi_rx_data, 1, 10) == HAL_OK) {
 8001498:	1d39      	adds	r1, r7, #4
 800149a:	230a      	movs	r3, #10
 800149c:	2201      	movs	r2, #1
 800149e:	48a8      	ldr	r0, [pc, #672]	; (8001740 <main+0x38c>)
 80014a0:	f002 ffc5 	bl	800442e <HAL_SPI_Receive>
 80014a4:	4603      	mov	r3, r0
 80014a6:	2b00      	cmp	r3, #0
 80014a8:	d102      	bne.n	80014b0 <main+0xfc>
  		HAL_Delay(10);
 80014aa:	200a      	movs	r0, #10
 80014ac:	f000 ff00 	bl	80022b0 <HAL_Delay>
  	}
  }
  HAL_GPIO_WritePin(bmp280_CS_GPIO_Port, bmp280_CS_Pin, GPIO_PIN_SET);
 80014b0:	2201      	movs	r2, #1
 80014b2:	2110      	movs	r1, #16
 80014b4:	48a1      	ldr	r0, [pc, #644]	; (800173c <main+0x388>)
 80014b6:	f002 f929 	bl	800370c <HAL_GPIO_WritePin>
  HAL_Delay(10);
 80014ba:	200a      	movs	r0, #10
 80014bc:	f000 fef8 	bl	80022b0 <HAL_Delay>

  printf("Temperature system control\r\n");
 80014c0:	48a0      	ldr	r0, [pc, #640]	; (8001744 <main+0x390>)
 80014c2:	f005 fb89 	bl	8006bd8 <puts>

  /* Infinite loop */
  /* USER CODE BEGIN WHILE */
  while (1)
  {
		heartbeat();													// System was initialized
 80014c6:	f7ff fd95 	bl	8000ff4 <heartbeat>
		door();															// function of open the door
 80014ca:	f7ff fd4f 	bl	8000f6c <door>
		temp = temp_meas(toggle_period_ms, toogle_meas_enable);		    // Take the measurement of the temperature sensor
 80014ce:	7dbb      	ldrb	r3, [r7, #22]
 80014d0:	4619      	mov	r1, r3
 80014d2:	6938      	ldr	r0, [r7, #16]
 80014d4:	f7ff fdae 	bl	8001034 <temp_meas>
 80014d8:	ed87 0a03 	vstr	s0, [r7, #12]

		switch(state){ 													// State Machine was initialized
 80014dc:	7dfb      	ldrb	r3, [r7, #23]
 80014de:	2b05      	cmp	r3, #5
 80014e0:	f200 8172 	bhi.w	80017c8 <main+0x414>
 80014e4:	a201      	add	r2, pc, #4	; (adr r2, 80014ec <main+0x138>)
 80014e6:	f852 f023 	ldr.w	pc, [r2, r3, lsl #2]
 80014ea:	bf00      	nop
 80014ec:	08001505 	.word	0x08001505
 80014f0:	0800156d 	.word	0x0800156d
 80014f4:	080015d1 	.word	0x080015d1
 80014f8:	0800163f 	.word	0x0800163f
 80014fc:	080016a3 	.word	0x080016a3
 8001500:	0800170b 	.word	0x0800170b
		case 0: // COLD
			if (temp > 20.0){
 8001504:	edd7 7a03 	vldr	s15, [r7, #12]
 8001508:	eeb3 7a04 	vmov.f32	s14, #52	; 0x41a00000  20.0
 800150c:	eef4 7ac7 	vcmpe.f32	s15, s14
 8001510:	eef1 fa10 	vmrs	APSR_nzcv, fpscr
 8001514:	dd02      	ble.n	800151c <main+0x168>
				state = 2;
 8001516:	2302      	movs	r3, #2
 8001518:	75fb      	strb	r3, [r7, #23]
				break;
 800151a:	e156      	b.n	80017ca <main+0x416>
			} else if (temp < 10.0){
 800151c:	edd7 7a03 	vldr	s15, [r7, #12]
 8001520:	eeb2 7a04 	vmov.f32	s14, #36	; 0x41200000  10.0
 8001524:	eef4 7ac7 	vcmpe.f32	s15, s14
 8001528:	eef1 fa10 	vmrs	APSR_nzcv, fpscr
 800152c:	d502      	bpl.n	8001534 <main+0x180>
				state = 1;
 800152e:	2301      	movs	r3, #1
 8001530:	75fb      	strb	r3, [r7, #23]
				break;
 8001532:	e14a      	b.n	80017ca <main+0x416>
			}
			printf("COLD\r\n");
 8001534:	4884      	ldr	r0, [pc, #528]	; (8001748 <main+0x394>)
 8001536:	f005 fb4f 	bl	8006bd8 <puts>
			printf("--> Heater OFF\r\n");
 800153a:	4884      	ldr	r0, [pc, #528]	; (800174c <main+0x398>)
 800153c:	f005 fb4c 	bl	8006bd8 <puts>
			printf("--> Fan OFF\r\n");
 8001540:	4883      	ldr	r0, [pc, #524]	; (8001750 <main+0x39c>)
 8001542:	f005 fb49 	bl	8006bd8 <puts>
			HAL_GPIO_WritePin(Heater_GPIO_Port, Heater_Pin, GPIO_PIN_RESET);	// Heater OF
 8001546:	2200      	movs	r2, #0
 8001548:	f44f 6100 	mov.w	r1, #2048	; 0x800
 800154c:	4881      	ldr	r0, [pc, #516]	; (8001754 <main+0x3a0>)
 800154e:	f002 f8dd 	bl	800370c <HAL_GPIO_WritePin>
			HAL_GPIO_WritePin(Alert_GPIO_Port, Alert_Pin, GPIO_PIN_RESET);		// Alert OFF
 8001552:	2200      	movs	r2, #0
 8001554:	f44f 4180 	mov.w	r1, #16384	; 0x4000
 8001558:	487e      	ldr	r0, [pc, #504]	; (8001754 <main+0x3a0>)
 800155a:	f002 f8d7 	bl	800370c <HAL_GPIO_WritePin>
			PWM_DMA(0.0, 0.0);													// Fan OFF
 800155e:	eddf 0a7e 	vldr	s1, [pc, #504]	; 8001758 <main+0x3a4>
 8001562:	ed9f 0a7d 	vldr	s0, [pc, #500]	; 8001758 <main+0x3a4>
 8001566:	f7ff fe6f 	bl	8001248 <PWM_DMA>

			break;
 800156a:	e12e      	b.n	80017ca <main+0x416>
		case 1: //VERY COLD
			if (temp > 12.0){
 800156c:	edd7 7a03 	vldr	s15, [r7, #12]
 8001570:	eeb2 7a08 	vmov.f32	s14, #40	; 0x41400000  12.0
 8001574:	eef4 7ac7 	vcmpe.f32	s15, s14
 8001578:	eef1 fa10 	vmrs	APSR_nzcv, fpscr
 800157c:	dd02      	ble.n	8001584 <main+0x1d0>
				state = 0;
 800157e:	2300      	movs	r3, #0
 8001580:	75fb      	strb	r3, [r7, #23]
				break;
 8001582:	e122      	b.n	80017ca <main+0x416>
			} else if (temp < 0.0){
 8001584:	edd7 7a03 	vldr	s15, [r7, #12]
 8001588:	eef5 7ac0 	vcmpe.f32	s15, #0.0
 800158c:	eef1 fa10 	vmrs	APSR_nzcv, fpscr
 8001590:	d502      	bpl.n	8001598 <main+0x1e4>
				state = 3;
 8001592:	2303      	movs	r3, #3
 8001594:	75fb      	strb	r3, [r7, #23]
				break;
 8001596:	e118      	b.n	80017ca <main+0x416>
			}

			printf("VERY COLD\r\n");
 8001598:	4870      	ldr	r0, [pc, #448]	; (800175c <main+0x3a8>)
 800159a:	f005 fb1d 	bl	8006bd8 <puts>
			HAL_GPIO_WritePin(Heater_GPIO_Port, Heater_Pin, GPIO_PIN_SET);		// Heater ON
 800159e:	2201      	movs	r2, #1
 80015a0:	f44f 6100 	mov.w	r1, #2048	; 0x800
 80015a4:	486b      	ldr	r0, [pc, #428]	; (8001754 <main+0x3a0>)
 80015a6:	f002 f8b1 	bl	800370c <HAL_GPIO_WritePin>
			HAL_GPIO_WritePin(Alert_GPIO_Port, Alert_Pin, GPIO_PIN_RESET);		// Alert OFF
 80015aa:	2200      	movs	r2, #0
 80015ac:	f44f 4180 	mov.w	r1, #16384	; 0x4000
 80015b0:	4868      	ldr	r0, [pc, #416]	; (8001754 <main+0x3a0>)
 80015b2:	f002 f8ab 	bl	800370c <HAL_GPIO_WritePin>
			PWM_DMA(0.0, 0.0);													// Fan OFF
 80015b6:	eddf 0a68 	vldr	s1, [pc, #416]	; 8001758 <main+0x3a4>
 80015ba:	ed9f 0a67 	vldr	s0, [pc, #412]	; 8001758 <main+0x3a4>
 80015be:	f7ff fe43 	bl	8001248 <PWM_DMA>
			printf("--> Heater ON\r\n");
 80015c2:	4867      	ldr	r0, [pc, #412]	; (8001760 <main+0x3ac>)
 80015c4:	f005 fb08 	bl	8006bd8 <puts>
			printf("--> Fan OFF\r\n");
 80015c8:	4861      	ldr	r0, [pc, #388]	; (8001750 <main+0x39c>)
 80015ca:	f005 fb05 	bl	8006bd8 <puts>

			break;
 80015ce:	e0fc      	b.n	80017ca <main+0x416>
		case 2: //MILD
			if (temp > 30.0){
 80015d0:	edd7 7a03 	vldr	s15, [r7, #12]
 80015d4:	eeb3 7a0e 	vmov.f32	s14, #62	; 0x41f00000  30.0
 80015d8:	eef4 7ac7 	vcmpe.f32	s15, s14
 80015dc:	eef1 fa10 	vmrs	APSR_nzcv, fpscr
 80015e0:	dd02      	ble.n	80015e8 <main+0x234>
					state = 4;
 80015e2:	2304      	movs	r3, #4
 80015e4:	75fb      	strb	r3, [r7, #23]
					break;
 80015e6:	e0f0      	b.n	80017ca <main+0x416>
				} else if (temp < 18.0){
 80015e8:	edd7 7a03 	vldr	s15, [r7, #12]
 80015ec:	eeb3 7a02 	vmov.f32	s14, #50	; 0x41900000  18.0
 80015f0:	eef4 7ac7 	vcmpe.f32	s15, s14
 80015f4:	eef1 fa10 	vmrs	APSR_nzcv, fpscr
 80015f8:	d502      	bpl.n	8001600 <main+0x24c>
					state = 0;
 80015fa:	2300      	movs	r3, #0
 80015fc:	75fb      	strb	r3, [r7, #23]
					break;
 80015fe:	e0e4      	b.n	80017ca <main+0x416>
				}
			printf("MILD\r\n");
 8001600:	4858      	ldr	r0, [pc, #352]	; (8001764 <main+0x3b0>)
 8001602:	f005 fae9 	bl	8006bd8 <puts>
			HAL_GPIO_WritePin(Heater_GPIO_Port, Heater_Pin, GPIO_PIN_RESET);	// Heater OF
 8001606:	2200      	movs	r2, #0
 8001608:	f44f 6100 	mov.w	r1, #2048	; 0x800
 800160c:	4851      	ldr	r0, [pc, #324]	; (8001754 <main+0x3a0>)
 800160e:	f002 f87d 	bl	800370c <HAL_GPIO_WritePin>
			HAL_GPIO_WritePin(Alert_GPIO_Port, Alert_Pin, GPIO_PIN_RESET);		// Alert OFF
 8001612:	2200      	movs	r2, #0
 8001614:	f44f 4180 	mov.w	r1, #16384	; 0x4000
 8001618:	484e      	ldr	r0, [pc, #312]	; (8001754 <main+0x3a0>)
 800161a:	f002 f877 	bl	800370c <HAL_GPIO_WritePin>
			PWM_DMA(0.0, 0.2);													// Fan at 20% ON
 800161e:	eddf 0a52 	vldr	s1, [pc, #328]	; 8001768 <main+0x3b4>
 8001622:	ed9f 0a4d 	vldr	s0, [pc, #308]	; 8001758 <main+0x3a4>
 8001626:	f7ff fe0f 	bl	8001248 <PWM_DMA>
			printf("--> Heater OFF\r\n");
 800162a:	4848      	ldr	r0, [pc, #288]	; (800174c <main+0x398>)
 800162c:	f005 fad4 	bl	8006bd8 <puts>
			printf("--> Fan on 20 prct \r\n");
 8001630:	484e      	ldr	r0, [pc, #312]	; (800176c <main+0x3b8>)
 8001632:	f005 fad1 	bl	8006bd8 <puts>
			HAL_Delay(100);
 8001636:	2064      	movs	r0, #100	; 0x64
 8001638:	f000 fe3a 	bl	80022b0 <HAL_Delay>
			break;
 800163c:	e0c5      	b.n	80017ca <main+0x416>
		case 3: // ALERT

			printf("ALERT !!\r\n");
 800163e:	484c      	ldr	r0, [pc, #304]	; (8001770 <main+0x3bc>)
 8001640:	f005 faca 	bl	8006bd8 <puts>
			HAL_GPIO_WritePin(Heater_GPIO_Port, Heater_Pin, GPIO_PIN_RESET);	// Heater OF
 8001644:	2200      	movs	r2, #0
 8001646:	f44f 6100 	mov.w	r1, #2048	; 0x800
 800164a:	4842      	ldr	r0, [pc, #264]	; (8001754 <main+0x3a0>)
 800164c:	f002 f85e 	bl	800370c <HAL_GPIO_WritePin>
			HAL_GPIO_WritePin(Alert_GPIO_Port, Alert_Pin, GPIO_PIN_SET);		// Alert ON
 8001650:	2201      	movs	r2, #1
 8001652:	f44f 4180 	mov.w	r1, #16384	; 0x4000
 8001656:	483f      	ldr	r0, [pc, #252]	; (8001754 <main+0x3a0>)
 8001658:	f002 f858 	bl	800370c <HAL_GPIO_WritePin>
			PWM_DMA(0.0, 0.0);													// Fan OFF
 800165c:	eddf 0a3e 	vldr	s1, [pc, #248]	; 8001758 <main+0x3a4>
 8001660:	ed9f 0a3d 	vldr	s0, [pc, #244]	; 8001758 <main+0x3a4>
 8001664:	f7ff fdf0 	bl	8001248 <PWM_DMA>
			printf("--> Heater OFF\r\n");
 8001668:	4838      	ldr	r0, [pc, #224]	; (800174c <main+0x398>)
 800166a:	f005 fab5 	bl	8006bd8 <puts>
			printf("--> Fan OFF \r\n");
 800166e:	4841      	ldr	r0, [pc, #260]	; (8001774 <main+0x3c0>)
 8001670:	f005 fab2 	bl	8006bd8 <puts>

			if (temp > 0.0){
 8001674:	edd7 7a03 	vldr	s15, [r7, #12]
 8001678:	eef5 7ac0 	vcmpe.f32	s15, #0.0
 800167c:	eef1 fa10 	vmrs	APSR_nzcv, fpscr
 8001680:	dd02      	ble.n	8001688 <main+0x2d4>
				state = 1;
 8001682:	2301      	movs	r3, #1
 8001684:	75fb      	strb	r3, [r7, #23]
				break;
 8001686:	e0a0      	b.n	80017ca <main+0x416>
			} if (temp < 45.0){
 8001688:	edd7 7a03 	vldr	s15, [r7, #12]
 800168c:	ed9f 7a3a 	vldr	s14, [pc, #232]	; 8001778 <main+0x3c4>
 8001690:	eef4 7ac7 	vcmpe.f32	s15, s14
 8001694:	eef1 fa10 	vmrs	APSR_nzcv, fpscr
 8001698:	d400      	bmi.n	800169c <main+0x2e8>
				state = 5;
				break;
			}

			break;
 800169a:	e096      	b.n	80017ca <main+0x416>
				state = 5;
 800169c:	2305      	movs	r3, #5
 800169e:	75fb      	strb	r3, [r7, #23]
				break;
 80016a0:	e093      	b.n	80017ca <main+0x416>

		case 4: //HOT
			if (temp > 40.0){
 80016a2:	edd7 7a03 	vldr	s15, [r7, #12]
 80016a6:	ed9f 7a35 	vldr	s14, [pc, #212]	; 800177c <main+0x3c8>
 80016aa:	eef4 7ac7 	vcmpe.f32	s15, s14
 80016ae:	eef1 fa10 	vmrs	APSR_nzcv, fpscr
 80016b2:	dd02      	ble.n	80016ba <main+0x306>
				state = 5;
 80016b4:	2305      	movs	r3, #5
 80016b6:	75fb      	strb	r3, [r7, #23]
				break;
 80016b8:	e087      	b.n	80017ca <main+0x416>
			} else if (temp < 28.0){
 80016ba:	edd7 7a03 	vldr	s15, [r7, #12]
 80016be:	eeb3 7a0c 	vmov.f32	s14, #60	; 0x41e00000  28.0
 80016c2:	eef4 7ac7 	vcmpe.f32	s15, s14
 80016c6:	eef1 fa10 	vmrs	APSR_nzcv, fpscr
 80016ca:	d502      	bpl.n	80016d2 <main+0x31e>
				state = 2;
 80016cc:	2302      	movs	r3, #2
 80016ce:	75fb      	strb	r3, [r7, #23]
				break;
 80016d0:	e07b      	b.n	80017ca <main+0x416>
			}
			printf("HOT\r\n");
 80016d2:	482b      	ldr	r0, [pc, #172]	; (8001780 <main+0x3cc>)
 80016d4:	f005 fa80 	bl	8006bd8 <puts>
			HAL_GPIO_WritePin(Heater_GPIO_Port, Heater_Pin, GPIO_PIN_RESET);	// Heater OF
 80016d8:	2200      	movs	r2, #0
 80016da:	f44f 6100 	mov.w	r1, #2048	; 0x800
 80016de:	481d      	ldr	r0, [pc, #116]	; (8001754 <main+0x3a0>)
 80016e0:	f002 f814 	bl	800370c <HAL_GPIO_WritePin>
			HAL_GPIO_WritePin(Alert_GPIO_Port, Alert_Pin, GPIO_PIN_RESET);		// Alert OFF
 80016e4:	2200      	movs	r2, #0
 80016e6:	f44f 4180 	mov.w	r1, #16384	; 0x4000
 80016ea:	481a      	ldr	r0, [pc, #104]	; (8001754 <main+0x3a0>)
 80016ec:	f002 f80e 	bl	800370c <HAL_GPIO_WritePin>
			PWM_DMA(0.2, 0.6);													// Fan at 60% ON
 80016f0:	eddf 0a24 	vldr	s1, [pc, #144]	; 8001784 <main+0x3d0>
 80016f4:	ed9f 0a1c 	vldr	s0, [pc, #112]	; 8001768 <main+0x3b4>
 80016f8:	f7ff fda6 	bl	8001248 <PWM_DMA>
			printf("--> Heater OFF\r\n");
 80016fc:	4813      	ldr	r0, [pc, #76]	; (800174c <main+0x398>)
 80016fe:	f005 fa6b 	bl	8006bd8 <puts>
			printf("--> Fan on 60 prct \r\n");
 8001702:	4821      	ldr	r0, [pc, #132]	; (8001788 <main+0x3d4>)
 8001704:	f005 fa68 	bl	8006bd8 <puts>

			break;
 8001708:	e05f      	b.n	80017ca <main+0x416>
		case 5:	// VERY HOT
			if (temp >= 45.0){
 800170a:	edd7 7a03 	vldr	s15, [r7, #12]
 800170e:	ed9f 7a1a 	vldr	s14, [pc, #104]	; 8001778 <main+0x3c4>
 8001712:	eef4 7ac7 	vcmpe.f32	s15, s14
 8001716:	eef1 fa10 	vmrs	APSR_nzcv, fpscr
 800171a:	db02      	blt.n	8001722 <main+0x36e>
				state = 3;
 800171c:	2303      	movs	r3, #3
 800171e:	75fb      	strb	r3, [r7, #23]
				break;
 8001720:	e053      	b.n	80017ca <main+0x416>
			} else if (temp < 38.0){
 8001722:	edd7 7a03 	vldr	s15, [r7, #12]
 8001726:	ed9f 7a19 	vldr	s14, [pc, #100]	; 800178c <main+0x3d8>
 800172a:	eef4 7ac7 	vcmpe.f32	s15, s14
 800172e:	eef1 fa10 	vmrs	APSR_nzcv, fpscr
 8001732:	d52d      	bpl.n	8001790 <main+0x3dc>
				state = 4;
 8001734:	2304      	movs	r3, #4
 8001736:	75fb      	strb	r3, [r7, #23]
				break;
 8001738:	e047      	b.n	80017ca <main+0x416>
 800173a:	bf00      	nop
 800173c:	40020800 	.word	0x40020800
 8001740:	20000240 	.word	0x20000240
 8001744:	08008d8c 	.word	0x08008d8c
 8001748:	08008da8 	.word	0x08008da8
 800174c:	08008db0 	.word	0x08008db0
 8001750:	08008dc0 	.word	0x08008dc0
 8001754:	40021800 	.word	0x40021800
 8001758:	00000000 	.word	0x00000000
 800175c:	08008dd0 	.word	0x08008dd0
 8001760:	08008ddc 	.word	0x08008ddc
 8001764:	08008dec 	.word	0x08008dec
 8001768:	3e4ccccd 	.word	0x3e4ccccd
 800176c:	08008df4 	.word	0x08008df4
 8001770:	08008e0c 	.word	0x08008e0c
 8001774:	08008e18 	.word	0x08008e18
 8001778:	42340000 	.word	0x42340000
 800177c:	42200000 	.word	0x42200000
 8001780:	08008e28 	.word	0x08008e28
 8001784:	3f19999a 	.word	0x3f19999a
 8001788:	08008e30 	.word	0x08008e30
 800178c:	42180000 	.word	0x42180000
			}
			printf("VERY HOT\r\n");
 8001790:	4810      	ldr	r0, [pc, #64]	; (80017d4 <main+0x420>)
 8001792:	f005 fa21 	bl	8006bd8 <puts>
			HAL_GPIO_WritePin(Heater_GPIO_Port, Heater_Pin, GPIO_PIN_RESET);	// Heater OF
 8001796:	2200      	movs	r2, #0
 8001798:	f44f 6100 	mov.w	r1, #2048	; 0x800
 800179c:	480e      	ldr	r0, [pc, #56]	; (80017d8 <main+0x424>)
 800179e:	f001 ffb5 	bl	800370c <HAL_GPIO_WritePin>
			HAL_GPIO_WritePin(Alert_GPIO_Port, Alert_Pin, GPIO_PIN_RESET);		// Alert OFF
 80017a2:	2200      	movs	r2, #0
 80017a4:	f44f 4180 	mov.w	r1, #16384	; 0x4000
 80017a8:	480b      	ldr	r0, [pc, #44]	; (80017d8 <main+0x424>)
 80017aa:	f001 ffaf 	bl	800370c <HAL_GPIO_WritePin>
			PWM_DMA(0.6, 1);													// Fan at 100% ON
 80017ae:	eef7 0a00 	vmov.f32	s1, #112	; 0x3f800000  1.0
 80017b2:	ed9f 0a0a 	vldr	s0, [pc, #40]	; 80017dc <main+0x428>
 80017b6:	f7ff fd47 	bl	8001248 <PWM_DMA>
			printf("--> Heater OFF\r\n");
 80017ba:	4809      	ldr	r0, [pc, #36]	; (80017e0 <main+0x42c>)
 80017bc:	f005 fa0c 	bl	8006bd8 <puts>
			printf("--> Fan on 100 prct \r\n");
 80017c0:	4808      	ldr	r0, [pc, #32]	; (80017e4 <main+0x430>)
 80017c2:	f005 fa09 	bl	8006bd8 <puts>

			break;
 80017c6:	e000      	b.n	80017ca <main+0x416>
		default:
			// do nothing
		break;
 80017c8:	bf00      	nop

		printf("\r\n");
		}
		HAL_Delay(100);
 80017ca:	2064      	movs	r0, #100	; 0x64
 80017cc:	f000 fd70 	bl	80022b0 <HAL_Delay>
		heartbeat();													// System was initialized
 80017d0:	e679      	b.n	80014c6 <main+0x112>
 80017d2:	bf00      	nop
 80017d4:	08008e48 	.word	0x08008e48
 80017d8:	40021800 	.word	0x40021800
 80017dc:	3f19999a 	.word	0x3f19999a
 80017e0:	08008db0 	.word	0x08008db0
 80017e4:	08008e54 	.word	0x08008e54

080017e8 <SystemClock_Config>:
/**
  * @brief System Clock Configuration
  * @retval None
  */
void SystemClock_Config(void)
{
 80017e8:	b580      	push	{r7, lr}
 80017ea:	b094      	sub	sp, #80	; 0x50
 80017ec:	af00      	add	r7, sp, #0
  RCC_OscInitTypeDef RCC_OscInitStruct = {0};
 80017ee:	f107 0320 	add.w	r3, r7, #32
 80017f2:	2230      	movs	r2, #48	; 0x30
 80017f4:	2100      	movs	r1, #0
 80017f6:	4618      	mov	r0, r3
 80017f8:	f004 fcf6 	bl	80061e8 <memset>
  RCC_ClkInitTypeDef RCC_ClkInitStruct = {0};
 80017fc:	f107 030c 	add.w	r3, r7, #12
 8001800:	2200      	movs	r2, #0
 8001802:	601a      	str	r2, [r3, #0]
 8001804:	605a      	str	r2, [r3, #4]
 8001806:	609a      	str	r2, [r3, #8]
 8001808:	60da      	str	r2, [r3, #12]
 800180a:	611a      	str	r2, [r3, #16]

  /** Configure the main internal regulator output voltage
  */
  __HAL_RCC_PWR_CLK_ENABLE();
 800180c:	2300      	movs	r3, #0
 800180e:	60bb      	str	r3, [r7, #8]
 8001810:	4b29      	ldr	r3, [pc, #164]	; (80018b8 <SystemClock_Config+0xd0>)
 8001812:	6c1b      	ldr	r3, [r3, #64]	; 0x40
 8001814:	4a28      	ldr	r2, [pc, #160]	; (80018b8 <SystemClock_Config+0xd0>)
 8001816:	f043 5380 	orr.w	r3, r3, #268435456	; 0x10000000
 800181a:	6413      	str	r3, [r2, #64]	; 0x40
 800181c:	4b26      	ldr	r3, [pc, #152]	; (80018b8 <SystemClock_Config+0xd0>)
 800181e:	6c1b      	ldr	r3, [r3, #64]	; 0x40
 8001820:	f003 5380 	and.w	r3, r3, #268435456	; 0x10000000
 8001824:	60bb      	str	r3, [r7, #8]
 8001826:	68bb      	ldr	r3, [r7, #8]
  __HAL_PWR_VOLTAGESCALING_CONFIG(PWR_REGULATOR_VOLTAGE_SCALE3);
 8001828:	2300      	movs	r3, #0
 800182a:	607b      	str	r3, [r7, #4]
 800182c:	4b23      	ldr	r3, [pc, #140]	; (80018bc <SystemClock_Config+0xd4>)
 800182e:	681b      	ldr	r3, [r3, #0]
 8001830:	f423 4340 	bic.w	r3, r3, #49152	; 0xc000
 8001834:	4a21      	ldr	r2, [pc, #132]	; (80018bc <SystemClock_Config+0xd4>)
 8001836:	f443 4380 	orr.w	r3, r3, #16384	; 0x4000
 800183a:	6013      	str	r3, [r2, #0]
 800183c:	4b1f      	ldr	r3, [pc, #124]	; (80018bc <SystemClock_Config+0xd4>)
 800183e:	681b      	ldr	r3, [r3, #0]
 8001840:	f403 4340 	and.w	r3, r3, #49152	; 0xc000
 8001844:	607b      	str	r3, [r7, #4]
 8001846:	687b      	ldr	r3, [r7, #4]

  /** Initializes the RCC Oscillators according to the specified parameters
  * in the RCC_OscInitTypeDef structure.
  */
  RCC_OscInitStruct.OscillatorType = RCC_OSCILLATORTYPE_HSI;
 8001848:	2302      	movs	r3, #2
 800184a:	623b      	str	r3, [r7, #32]
  RCC_OscInitStruct.HSIState = RCC_HSI_ON;
 800184c:	2301      	movs	r3, #1
 800184e:	62fb      	str	r3, [r7, #44]	; 0x2c
  RCC_OscInitStruct.HSICalibrationValue = RCC_HSICALIBRATION_DEFAULT;
 8001850:	2310      	movs	r3, #16
 8001852:	633b      	str	r3, [r7, #48]	; 0x30
  RCC_OscInitStruct.PLL.PLLState = RCC_PLL_ON;
 8001854:	2302      	movs	r3, #2
 8001856:	63bb      	str	r3, [r7, #56]	; 0x38
  RCC_OscInitStruct.PLL.PLLSource = RCC_PLLSOURCE_HSI;
 8001858:	2300      	movs	r3, #0
 800185a:	63fb      	str	r3, [r7, #60]	; 0x3c
  RCC_OscInitStruct.PLL.PLLM = 8;
 800185c:	2308      	movs	r3, #8
 800185e:	643b      	str	r3, [r7, #64]	; 0x40
  RCC_OscInitStruct.PLL.PLLN = 50;
 8001860:	2332      	movs	r3, #50	; 0x32
 8001862:	647b      	str	r3, [r7, #68]	; 0x44
  RCC_OscInitStruct.PLL.PLLP = RCC_PLLP_DIV2;
 8001864:	2302      	movs	r3, #2
 8001866:	64bb      	str	r3, [r7, #72]	; 0x48
  RCC_OscInitStruct.PLL.PLLQ = 7;
 8001868:	2307      	movs	r3, #7
 800186a:	64fb      	str	r3, [r7, #76]	; 0x4c
  if (HAL_RCC_OscConfig(&RCC_OscInitStruct) != HAL_OK)
 800186c:	f107 0320 	add.w	r3, r7, #32
 8001870:	4618      	mov	r0, r3
 8001872:	f001 ff7f 	bl	8003774 <HAL_RCC_OscConfig>
 8001876:	4603      	mov	r3, r0
 8001878:	2b00      	cmp	r3, #0
 800187a:	d001      	beq.n	8001880 <SystemClock_Config+0x98>
  {
    Error_Handler();
 800187c:	f000 f9fa 	bl	8001c74 <Error_Handler>
  }

  /** Initializes the CPU, AHB and APB buses clocks
  */
  RCC_ClkInitStruct.ClockType = RCC_CLOCKTYPE_HCLK|RCC_CLOCKTYPE_SYSCLK
 8001880:	230f      	movs	r3, #15
 8001882:	60fb      	str	r3, [r7, #12]
                              |RCC_CLOCKTYPE_PCLK1|RCC_CLOCKTYPE_PCLK2;
  RCC_ClkInitStruct.SYSCLKSource = RCC_SYSCLKSOURCE_PLLCLK;
 8001884:	2302      	movs	r3, #2
 8001886:	613b      	str	r3, [r7, #16]
  RCC_ClkInitStruct.AHBCLKDivider = RCC_SYSCLK_DIV2;
 8001888:	2380      	movs	r3, #128	; 0x80
 800188a:	617b      	str	r3, [r7, #20]
  RCC_ClkInitStruct.APB1CLKDivider = RCC_HCLK_DIV4;
 800188c:	f44f 53a0 	mov.w	r3, #5120	; 0x1400
 8001890:	61bb      	str	r3, [r7, #24]
  RCC_ClkInitStruct.APB2CLKDivider = RCC_HCLK_DIV2;
 8001892:	f44f 5380 	mov.w	r3, #4096	; 0x1000
 8001896:	61fb      	str	r3, [r7, #28]

  if (HAL_RCC_ClockConfig(&RCC_ClkInitStruct, FLASH_LATENCY_0) != HAL_OK)
 8001898:	f107 030c 	add.w	r3, r7, #12
 800189c:	2100      	movs	r1, #0
 800189e:	4618      	mov	r0, r3
 80018a0:	f002 f9e0 	bl	8003c64 <HAL_RCC_ClockConfig>
 80018a4:	4603      	mov	r3, r0
 80018a6:	2b00      	cmp	r3, #0
 80018a8:	d001      	beq.n	80018ae <SystemClock_Config+0xc6>
  {
    Error_Handler();
 80018aa:	f000 f9e3 	bl	8001c74 <Error_Handler>
  }
}
 80018ae:	bf00      	nop
 80018b0:	3750      	adds	r7, #80	; 0x50
 80018b2:	46bd      	mov	sp, r7
 80018b4:	bd80      	pop	{r7, pc}
 80018b6:	bf00      	nop
 80018b8:	40023800 	.word	0x40023800
 80018bc:	40007000 	.word	0x40007000

080018c0 <MX_ADC1_Init>:
  * @brief ADC1 Initialization Function
  * @param None
  * @retval None
  */
static void MX_ADC1_Init(void)
{
 80018c0:	b580      	push	{r7, lr}
 80018c2:	b084      	sub	sp, #16
 80018c4:	af00      	add	r7, sp, #0

  /* USER CODE BEGIN ADC1_Init 0 */

  /* USER CODE END ADC1_Init 0 */

  ADC_ChannelConfTypeDef sConfig = {0};
 80018c6:	463b      	mov	r3, r7
 80018c8:	2200      	movs	r2, #0
 80018ca:	601a      	str	r2, [r3, #0]
 80018cc:	605a      	str	r2, [r3, #4]
 80018ce:	609a      	str	r2, [r3, #8]
 80018d0:	60da      	str	r2, [r3, #12]

  /* USER CODE END ADC1_Init 1 */

  /** Configure the global features of the ADC (Clock, Resolution, Data Alignment and number of conversion)
  */
  hadc1.Instance = ADC1;
 80018d2:	4b21      	ldr	r3, [pc, #132]	; (8001958 <MX_ADC1_Init+0x98>)
 80018d4:	4a21      	ldr	r2, [pc, #132]	; (800195c <MX_ADC1_Init+0x9c>)
 80018d6:	601a      	str	r2, [r3, #0]
  hadc1.Init.ClockPrescaler = ADC_CLOCK_SYNC_PCLK_DIV2;
 80018d8:	4b1f      	ldr	r3, [pc, #124]	; (8001958 <MX_ADC1_Init+0x98>)
 80018da:	2200      	movs	r2, #0
 80018dc:	605a      	str	r2, [r3, #4]
  hadc1.Init.Resolution = ADC_RESOLUTION_12B;
 80018de:	4b1e      	ldr	r3, [pc, #120]	; (8001958 <MX_ADC1_Init+0x98>)
 80018e0:	2200      	movs	r2, #0
 80018e2:	609a      	str	r2, [r3, #8]
  hadc1.Init.ScanConvMode = DISABLE;
 80018e4:	4b1c      	ldr	r3, [pc, #112]	; (8001958 <MX_ADC1_Init+0x98>)
 80018e6:	2200      	movs	r2, #0
 80018e8:	611a      	str	r2, [r3, #16]
  hadc1.Init.ContinuousConvMode = DISABLE;
 80018ea:	4b1b      	ldr	r3, [pc, #108]	; (8001958 <MX_ADC1_Init+0x98>)
 80018ec:	2200      	movs	r2, #0
 80018ee:	761a      	strb	r2, [r3, #24]
  hadc1.Init.DiscontinuousConvMode = DISABLE;
 80018f0:	4b19      	ldr	r3, [pc, #100]	; (8001958 <MX_ADC1_Init+0x98>)
 80018f2:	2200      	movs	r2, #0
 80018f4:	f883 2020 	strb.w	r2, [r3, #32]
  hadc1.Init.ExternalTrigConvEdge = ADC_EXTERNALTRIGCONVEDGE_NONE;
 80018f8:	4b17      	ldr	r3, [pc, #92]	; (8001958 <MX_ADC1_Init+0x98>)
 80018fa:	2200      	movs	r2, #0
 80018fc:	62da      	str	r2, [r3, #44]	; 0x2c
  hadc1.Init.ExternalTrigConv = ADC_SOFTWARE_START;
 80018fe:	4b16      	ldr	r3, [pc, #88]	; (8001958 <MX_ADC1_Init+0x98>)
 8001900:	4a17      	ldr	r2, [pc, #92]	; (8001960 <MX_ADC1_Init+0xa0>)
 8001902:	629a      	str	r2, [r3, #40]	; 0x28
  hadc1.Init.DataAlign = ADC_DATAALIGN_RIGHT;
 8001904:	4b14      	ldr	r3, [pc, #80]	; (8001958 <MX_ADC1_Init+0x98>)
 8001906:	2200      	movs	r2, #0
 8001908:	60da      	str	r2, [r3, #12]
  hadc1.Init.NbrOfConversion = 1;
 800190a:	4b13      	ldr	r3, [pc, #76]	; (8001958 <MX_ADC1_Init+0x98>)
 800190c:	2201      	movs	r2, #1
 800190e:	61da      	str	r2, [r3, #28]
  hadc1.Init.DMAContinuousRequests = DISABLE;
 8001910:	4b11      	ldr	r3, [pc, #68]	; (8001958 <MX_ADC1_Init+0x98>)
 8001912:	2200      	movs	r2, #0
 8001914:	f883 2030 	strb.w	r2, [r3, #48]	; 0x30
  hadc1.Init.EOCSelection = ADC_EOC_SINGLE_CONV;
 8001918:	4b0f      	ldr	r3, [pc, #60]	; (8001958 <MX_ADC1_Init+0x98>)
 800191a:	2201      	movs	r2, #1
 800191c:	615a      	str	r2, [r3, #20]
  if (HAL_ADC_Init(&hadc1) != HAL_OK)
 800191e:	480e      	ldr	r0, [pc, #56]	; (8001958 <MX_ADC1_Init+0x98>)
 8001920:	f000 fcea 	bl	80022f8 <HAL_ADC_Init>
 8001924:	4603      	mov	r3, r0
 8001926:	2b00      	cmp	r3, #0
 8001928:	d001      	beq.n	800192e <MX_ADC1_Init+0x6e>
  {
    Error_Handler();
 800192a:	f000 f9a3 	bl	8001c74 <Error_Handler>
  }

  /** Configure for the selected ADC regular channel its corresponding rank in the sequencer and its sample time.
  */
  sConfig.Channel = ADC_CHANNEL_0;
 800192e:	2300      	movs	r3, #0
 8001930:	603b      	str	r3, [r7, #0]
  sConfig.Rank = 1;
 8001932:	2301      	movs	r3, #1
 8001934:	607b      	str	r3, [r7, #4]
  sConfig.SamplingTime = ADC_SAMPLETIME_3CYCLES;
 8001936:	2300      	movs	r3, #0
 8001938:	60bb      	str	r3, [r7, #8]
  if (HAL_ADC_ConfigChannel(&hadc1, &sConfig) != HAL_OK)
 800193a:	463b      	mov	r3, r7
 800193c:	4619      	mov	r1, r3
 800193e:	4806      	ldr	r0, [pc, #24]	; (8001958 <MX_ADC1_Init+0x98>)
 8001940:	f000 fe88 	bl	8002654 <HAL_ADC_ConfigChannel>
 8001944:	4603      	mov	r3, r0
 8001946:	2b00      	cmp	r3, #0
 8001948:	d001      	beq.n	800194e <MX_ADC1_Init+0x8e>
  {
    Error_Handler();
 800194a:	f000 f993 	bl	8001c74 <Error_Handler>
  }
  /* USER CODE BEGIN ADC1_Init 2 */

  /* USER CODE END ADC1_Init 2 */

}
 800194e:	bf00      	nop
 8001950:	3710      	adds	r7, #16
 8001952:	46bd      	mov	sp, r7
 8001954:	bd80      	pop	{r7, pc}
 8001956:	bf00      	nop
 8001958:	200001f8 	.word	0x200001f8
 800195c:	40012000 	.word	0x40012000
 8001960:	0f000001 	.word	0x0f000001

08001964 <MX_SPI1_Init>:
  * @brief SPI1 Initialization Function
  * @param None
  * @retval None
  */
static void MX_SPI1_Init(void)
{
 8001964:	b580      	push	{r7, lr}
 8001966:	af00      	add	r7, sp, #0

  /* USER CODE BEGIN SPI1_Init 1 */

  /* USER CODE END SPI1_Init 1 */
  /* SPI1 parameter configuration*/
  hspi1.Instance = SPI1;
 8001968:	4b17      	ldr	r3, [pc, #92]	; (80019c8 <MX_SPI1_Init+0x64>)
 800196a:	4a18      	ldr	r2, [pc, #96]	; (80019cc <MX_SPI1_Init+0x68>)
 800196c:	601a      	str	r2, [r3, #0]
  hspi1.Init.Mode = SPI_MODE_MASTER;
 800196e:	4b16      	ldr	r3, [pc, #88]	; (80019c8 <MX_SPI1_Init+0x64>)
 8001970:	f44f 7282 	mov.w	r2, #260	; 0x104
 8001974:	605a      	str	r2, [r3, #4]
  hspi1.Init.Direction = SPI_DIRECTION_2LINES;
 8001976:	4b14      	ldr	r3, [pc, #80]	; (80019c8 <MX_SPI1_Init+0x64>)
 8001978:	2200      	movs	r2, #0
 800197a:	609a      	str	r2, [r3, #8]
  hspi1.Init.DataSize = SPI_DATASIZE_8BIT;
 800197c:	4b12      	ldr	r3, [pc, #72]	; (80019c8 <MX_SPI1_Init+0x64>)
 800197e:	2200      	movs	r2, #0
 8001980:	60da      	str	r2, [r3, #12]
  hspi1.Init.CLKPolarity = SPI_POLARITY_LOW;
 8001982:	4b11      	ldr	r3, [pc, #68]	; (80019c8 <MX_SPI1_Init+0x64>)
 8001984:	2200      	movs	r2, #0
 8001986:	611a      	str	r2, [r3, #16]
  hspi1.Init.CLKPhase = SPI_PHASE_1EDGE;
 8001988:	4b0f      	ldr	r3, [pc, #60]	; (80019c8 <MX_SPI1_Init+0x64>)
 800198a:	2200      	movs	r2, #0
 800198c:	615a      	str	r2, [r3, #20]
  hspi1.Init.NSS = SPI_NSS_SOFT;
 800198e:	4b0e      	ldr	r3, [pc, #56]	; (80019c8 <MX_SPI1_Init+0x64>)
 8001990:	f44f 7200 	mov.w	r2, #512	; 0x200
 8001994:	619a      	str	r2, [r3, #24]
  hspi1.Init.BaudRatePrescaler = SPI_BAUDRATEPRESCALER_2;
 8001996:	4b0c      	ldr	r3, [pc, #48]	; (80019c8 <MX_SPI1_Init+0x64>)
 8001998:	2200      	movs	r2, #0
 800199a:	61da      	str	r2, [r3, #28]
  hspi1.Init.FirstBit = SPI_FIRSTBIT_MSB;
 800199c:	4b0a      	ldr	r3, [pc, #40]	; (80019c8 <MX_SPI1_Init+0x64>)
 800199e:	2200      	movs	r2, #0
 80019a0:	621a      	str	r2, [r3, #32]
  hspi1.Init.TIMode = SPI_TIMODE_DISABLE;
 80019a2:	4b09      	ldr	r3, [pc, #36]	; (80019c8 <MX_SPI1_Init+0x64>)
 80019a4:	2200      	movs	r2, #0
 80019a6:	625a      	str	r2, [r3, #36]	; 0x24
  hspi1.Init.CRCCalculation = SPI_CRCCALCULATION_DISABLE;
 80019a8:	4b07      	ldr	r3, [pc, #28]	; (80019c8 <MX_SPI1_Init+0x64>)
 80019aa:	2200      	movs	r2, #0
 80019ac:	629a      	str	r2, [r3, #40]	; 0x28
  hspi1.Init.CRCPolynomial = 10;
 80019ae:	4b06      	ldr	r3, [pc, #24]	; (80019c8 <MX_SPI1_Init+0x64>)
 80019b0:	220a      	movs	r2, #10
 80019b2:	62da      	str	r2, [r3, #44]	; 0x2c
  if (HAL_SPI_Init(&hspi1) != HAL_OK)
 80019b4:	4804      	ldr	r0, [pc, #16]	; (80019c8 <MX_SPI1_Init+0x64>)
 80019b6:	f002 fb75 	bl	80040a4 <HAL_SPI_Init>
 80019ba:	4603      	mov	r3, r0
 80019bc:	2b00      	cmp	r3, #0
 80019be:	d001      	beq.n	80019c4 <MX_SPI1_Init+0x60>
  {
    Error_Handler();
 80019c0:	f000 f958 	bl	8001c74 <Error_Handler>
  }
  /* USER CODE BEGIN SPI1_Init 2 */

  /* USER CODE END SPI1_Init 2 */

}
 80019c4:	bf00      	nop
 80019c6:	bd80      	pop	{r7, pc}
 80019c8:	20000240 	.word	0x20000240
 80019cc:	40013000 	.word	0x40013000

080019d0 <MX_TIM1_Init>:
  * @brief TIM1 Initialization Function
  * @param None
  * @retval None
  */
static void MX_TIM1_Init(void)
{
 80019d0:	b580      	push	{r7, lr}
 80019d2:	b092      	sub	sp, #72	; 0x48
 80019d4:	af00      	add	r7, sp, #0

  /* USER CODE BEGIN TIM1_Init 0 */

  /* USER CODE END TIM1_Init 0 */

  TIM_MasterConfigTypeDef sMasterConfig = {0};
 80019d6:	f107 0340 	add.w	r3, r7, #64	; 0x40
 80019da:	2200      	movs	r2, #0
 80019dc:	601a      	str	r2, [r3, #0]
 80019de:	605a      	str	r2, [r3, #4]
  TIM_OC_InitTypeDef sConfigOC = {0};
 80019e0:	f107 0324 	add.w	r3, r7, #36	; 0x24
 80019e4:	2200      	movs	r2, #0
 80019e6:	601a      	str	r2, [r3, #0]
 80019e8:	605a      	str	r2, [r3, #4]
 80019ea:	609a      	str	r2, [r3, #8]
 80019ec:	60da      	str	r2, [r3, #12]
 80019ee:	611a      	str	r2, [r3, #16]
 80019f0:	615a      	str	r2, [r3, #20]
 80019f2:	619a      	str	r2, [r3, #24]
  TIM_BreakDeadTimeConfigTypeDef sBreakDeadTimeConfig = {0};
 80019f4:	1d3b      	adds	r3, r7, #4
 80019f6:	2220      	movs	r2, #32
 80019f8:	2100      	movs	r1, #0
 80019fa:	4618      	mov	r0, r3
 80019fc:	f004 fbf4 	bl	80061e8 <memset>

  /* USER CODE BEGIN TIM1_Init 1 */

  /* USER CODE END TIM1_Init 1 */
  htim1.Instance = TIM1;
 8001a00:	4b33      	ldr	r3, [pc, #204]	; (8001ad0 <MX_TIM1_Init+0x100>)
 8001a02:	4a34      	ldr	r2, [pc, #208]	; (8001ad4 <MX_TIM1_Init+0x104>)
 8001a04:	601a      	str	r2, [r3, #0]
  htim1.Init.Prescaler = 1.5;
 8001a06:	4b32      	ldr	r3, [pc, #200]	; (8001ad0 <MX_TIM1_Init+0x100>)
 8001a08:	2201      	movs	r2, #1
 8001a0a:	605a      	str	r2, [r3, #4]
  htim1.Init.CounterMode = TIM_COUNTERMODE_UP;
 8001a0c:	4b30      	ldr	r3, [pc, #192]	; (8001ad0 <MX_TIM1_Init+0x100>)
 8001a0e:	2200      	movs	r2, #0
 8001a10:	609a      	str	r2, [r3, #8]
  htim1.Init.Period = 1000;
 8001a12:	4b2f      	ldr	r3, [pc, #188]	; (8001ad0 <MX_TIM1_Init+0x100>)
 8001a14:	f44f 727a 	mov.w	r2, #1000	; 0x3e8
 8001a18:	60da      	str	r2, [r3, #12]
  htim1.Init.ClockDivision = TIM_CLOCKDIVISION_DIV1;
 8001a1a:	4b2d      	ldr	r3, [pc, #180]	; (8001ad0 <MX_TIM1_Init+0x100>)
 8001a1c:	2200      	movs	r2, #0
 8001a1e:	611a      	str	r2, [r3, #16]
  htim1.Init.RepetitionCounter = 0;
 8001a20:	4b2b      	ldr	r3, [pc, #172]	; (8001ad0 <MX_TIM1_Init+0x100>)
 8001a22:	2200      	movs	r2, #0
 8001a24:	615a      	str	r2, [r3, #20]
  htim1.Init.AutoReloadPreload = TIM_AUTORELOAD_PRELOAD_DISABLE;
 8001a26:	4b2a      	ldr	r3, [pc, #168]	; (8001ad0 <MX_TIM1_Init+0x100>)
 8001a28:	2200      	movs	r2, #0
 8001a2a:	619a      	str	r2, [r3, #24]
  if (HAL_TIM_PWM_Init(&htim1) != HAL_OK)
 8001a2c:	4828      	ldr	r0, [pc, #160]	; (8001ad0 <MX_TIM1_Init+0x100>)
 8001a2e:	f003 f8e1 	bl	8004bf4 <HAL_TIM_PWM_Init>
 8001a32:	4603      	mov	r3, r0
 8001a34:	2b00      	cmp	r3, #0
 8001a36:	d001      	beq.n	8001a3c <MX_TIM1_Init+0x6c>
  {
    Error_Handler();
 8001a38:	f000 f91c 	bl	8001c74 <Error_Handler>
  }
  sMasterConfig.MasterOutputTrigger = TIM_TRGO_RESET;
 8001a3c:	2300      	movs	r3, #0
 8001a3e:	643b      	str	r3, [r7, #64]	; 0x40
  sMasterConfig.MasterSlaveMode = TIM_MASTERSLAVEMODE_DISABLE;
 8001a40:	2300      	movs	r3, #0
 8001a42:	647b      	str	r3, [r7, #68]	; 0x44
  if (HAL_TIMEx_MasterConfigSynchronization(&htim1, &sMasterConfig) != HAL_OK)
 8001a44:	f107 0340 	add.w	r3, r7, #64	; 0x40
 8001a48:	4619      	mov	r1, r3
 8001a4a:	4821      	ldr	r0, [pc, #132]	; (8001ad0 <MX_TIM1_Init+0x100>)
 8001a4c:	f003 ff12 	bl	8005874 <HAL_TIMEx_MasterConfigSynchronization>
 8001a50:	4603      	mov	r3, r0
 8001a52:	2b00      	cmp	r3, #0
 8001a54:	d001      	beq.n	8001a5a <MX_TIM1_Init+0x8a>
  {
    Error_Handler();
 8001a56:	f000 f90d 	bl	8001c74 <Error_Handler>
  }
  sConfigOC.OCMode = TIM_OCMODE_PWM1;
 8001a5a:	2360      	movs	r3, #96	; 0x60
 8001a5c:	627b      	str	r3, [r7, #36]	; 0x24
  sConfigOC.Pulse = 0;
 8001a5e:	2300      	movs	r3, #0
 8001a60:	62bb      	str	r3, [r7, #40]	; 0x28
  sConfigOC.OCPolarity = TIM_OCPOLARITY_HIGH;
 8001a62:	2300      	movs	r3, #0
 8001a64:	62fb      	str	r3, [r7, #44]	; 0x2c
  sConfigOC.OCNPolarity = TIM_OCNPOLARITY_HIGH;
 8001a66:	2300      	movs	r3, #0
 8001a68:	633b      	str	r3, [r7, #48]	; 0x30
  sConfigOC.OCFastMode = TIM_OCFAST_DISABLE;
 8001a6a:	2300      	movs	r3, #0
 8001a6c:	637b      	str	r3, [r7, #52]	; 0x34
  sConfigOC.OCIdleState = TIM_OCIDLESTATE_RESET;
 8001a6e:	2300      	movs	r3, #0
 8001a70:	63bb      	str	r3, [r7, #56]	; 0x38
  sConfigOC.OCNIdleState = TIM_OCNIDLESTATE_RESET;
 8001a72:	2300      	movs	r3, #0
 8001a74:	63fb      	str	r3, [r7, #60]	; 0x3c
  if (HAL_TIM_PWM_ConfigChannel(&htim1, &sConfigOC, TIM_CHANNEL_1) != HAL_OK)
 8001a76:	f107 0324 	add.w	r3, r7, #36	; 0x24
 8001a7a:	2200      	movs	r2, #0
 8001a7c:	4619      	mov	r1, r3
 8001a7e:	4814      	ldr	r0, [pc, #80]	; (8001ad0 <MX_TIM1_Init+0x100>)
 8001a80:	f003 fad0 	bl	8005024 <HAL_TIM_PWM_ConfigChannel>
 8001a84:	4603      	mov	r3, r0
 8001a86:	2b00      	cmp	r3, #0
 8001a88:	d001      	beq.n	8001a8e <MX_TIM1_Init+0xbe>
  {
    Error_Handler();
 8001a8a:	f000 f8f3 	bl	8001c74 <Error_Handler>
  }
  sBreakDeadTimeConfig.OffStateRunMode = TIM_OSSR_DISABLE;
 8001a8e:	2300      	movs	r3, #0
 8001a90:	607b      	str	r3, [r7, #4]
  sBreakDeadTimeConfig.OffStateIDLEMode = TIM_OSSI_DISABLE;
 8001a92:	2300      	movs	r3, #0
 8001a94:	60bb      	str	r3, [r7, #8]
  sBreakDeadTimeConfig.LockLevel = TIM_LOCKLEVEL_OFF;
 8001a96:	2300      	movs	r3, #0
 8001a98:	60fb      	str	r3, [r7, #12]
  sBreakDeadTimeConfig.DeadTime = 0;
 8001a9a:	2300      	movs	r3, #0
 8001a9c:	613b      	str	r3, [r7, #16]
  sBreakDeadTimeConfig.BreakState = TIM_BREAK_DISABLE;
 8001a9e:	2300      	movs	r3, #0
 8001aa0:	617b      	str	r3, [r7, #20]
  sBreakDeadTimeConfig.BreakPolarity = TIM_BREAKPOLARITY_HIGH;
 8001aa2:	f44f 5300 	mov.w	r3, #8192	; 0x2000
 8001aa6:	61bb      	str	r3, [r7, #24]
  sBreakDeadTimeConfig.AutomaticOutput = TIM_AUTOMATICOUTPUT_DISABLE;
 8001aa8:	2300      	movs	r3, #0
 8001aaa:	623b      	str	r3, [r7, #32]
  if (HAL_TIMEx_ConfigBreakDeadTime(&htim1, &sBreakDeadTimeConfig) != HAL_OK)
 8001aac:	1d3b      	adds	r3, r7, #4
 8001aae:	4619      	mov	r1, r3
 8001ab0:	4807      	ldr	r0, [pc, #28]	; (8001ad0 <MX_TIM1_Init+0x100>)
 8001ab2:	f003 ff5b 	bl	800596c <HAL_TIMEx_ConfigBreakDeadTime>
 8001ab6:	4603      	mov	r3, r0
 8001ab8:	2b00      	cmp	r3, #0
 8001aba:	d001      	beq.n	8001ac0 <MX_TIM1_Init+0xf0>
  {
    Error_Handler();
 8001abc:	f000 f8da 	bl	8001c74 <Error_Handler>
  }
  /* USER CODE BEGIN TIM1_Init 2 */

  /* USER CODE END TIM1_Init 2 */
  HAL_TIM_MspPostInit(&htim1);
 8001ac0:	4803      	ldr	r0, [pc, #12]	; (8001ad0 <MX_TIM1_Init+0x100>)
 8001ac2:	f000 f9e7 	bl	8001e94 <HAL_TIM_MspPostInit>

}
 8001ac6:	bf00      	nop
 8001ac8:	3748      	adds	r7, #72	; 0x48
 8001aca:	46bd      	mov	sp, r7
 8001acc:	bd80      	pop	{r7, pc}
 8001ace:	bf00      	nop
 8001ad0:	20000298 	.word	0x20000298
 8001ad4:	40010000 	.word	0x40010000

08001ad8 <MX_USART1_UART_Init>:
  * @brief USART1 Initialization Function
  * @param None
  * @retval None
  */
static void MX_USART1_UART_Init(void)
{
 8001ad8:	b580      	push	{r7, lr}
 8001ada:	af00      	add	r7, sp, #0
  /* USER CODE END USART1_Init 0 */

  /* USER CODE BEGIN USART1_Init 1 */

  /* USER CODE END USART1_Init 1 */
  huart1.Instance = USART1;
 8001adc:	4b11      	ldr	r3, [pc, #68]	; (8001b24 <MX_USART1_UART_Init+0x4c>)
 8001ade:	4a12      	ldr	r2, [pc, #72]	; (8001b28 <MX_USART1_UART_Init+0x50>)
 8001ae0:	601a      	str	r2, [r3, #0]
  huart1.Init.BaudRate = 115200;
 8001ae2:	4b10      	ldr	r3, [pc, #64]	; (8001b24 <MX_USART1_UART_Init+0x4c>)
 8001ae4:	f44f 32e1 	mov.w	r2, #115200	; 0x1c200
 8001ae8:	605a      	str	r2, [r3, #4]
  huart1.Init.WordLength = UART_WORDLENGTH_8B;
 8001aea:	4b0e      	ldr	r3, [pc, #56]	; (8001b24 <MX_USART1_UART_Init+0x4c>)
 8001aec:	2200      	movs	r2, #0
 8001aee:	609a      	str	r2, [r3, #8]
  huart1.Init.StopBits = UART_STOPBITS_1;
 8001af0:	4b0c      	ldr	r3, [pc, #48]	; (8001b24 <MX_USART1_UART_Init+0x4c>)
 8001af2:	2200      	movs	r2, #0
 8001af4:	60da      	str	r2, [r3, #12]
  huart1.Init.Parity = UART_PARITY_NONE;
 8001af6:	4b0b      	ldr	r3, [pc, #44]	; (8001b24 <MX_USART1_UART_Init+0x4c>)
 8001af8:	2200      	movs	r2, #0
 8001afa:	611a      	str	r2, [r3, #16]
  huart1.Init.Mode = UART_MODE_TX_RX;
 8001afc:	4b09      	ldr	r3, [pc, #36]	; (8001b24 <MX_USART1_UART_Init+0x4c>)
 8001afe:	220c      	movs	r2, #12
 8001b00:	615a      	str	r2, [r3, #20]
  huart1.Init.HwFlowCtl = UART_HWCONTROL_NONE;
 8001b02:	4b08      	ldr	r3, [pc, #32]	; (8001b24 <MX_USART1_UART_Init+0x4c>)
 8001b04:	2200      	movs	r2, #0
 8001b06:	619a      	str	r2, [r3, #24]
  huart1.Init.OverSampling = UART_OVERSAMPLING_16;
 8001b08:	4b06      	ldr	r3, [pc, #24]	; (8001b24 <MX_USART1_UART_Init+0x4c>)
 8001b0a:	2200      	movs	r2, #0
 8001b0c:	61da      	str	r2, [r3, #28]
  if (HAL_UART_Init(&huart1) != HAL_OK)
 8001b0e:	4805      	ldr	r0, [pc, #20]	; (8001b24 <MX_USART1_UART_Init+0x4c>)
 8001b10:	f003 ff7e 	bl	8005a10 <HAL_UART_Init>
 8001b14:	4603      	mov	r3, r0
 8001b16:	2b00      	cmp	r3, #0
 8001b18:	d001      	beq.n	8001b1e <MX_USART1_UART_Init+0x46>
  {
    Error_Handler();
 8001b1a:	f000 f8ab 	bl	8001c74 <Error_Handler>
  }
  /* USER CODE BEGIN USART1_Init 2 */

  /* USER CODE END USART1_Init 2 */

}
 8001b1e:	bf00      	nop
 8001b20:	bd80      	pop	{r7, pc}
 8001b22:	bf00      	nop
 8001b24:	20000340 	.word	0x20000340
 8001b28:	40011000 	.word	0x40011000

08001b2c <MX_DMA_Init>:

/**
  * Enable DMA controller clock
  */
static void MX_DMA_Init(void)
{
 8001b2c:	b580      	push	{r7, lr}
 8001b2e:	b082      	sub	sp, #8
 8001b30:	af00      	add	r7, sp, #0

  /* DMA controller clock enable */
  __HAL_RCC_DMA2_CLK_ENABLE();
 8001b32:	2300      	movs	r3, #0
 8001b34:	607b      	str	r3, [r7, #4]
 8001b36:	4b0c      	ldr	r3, [pc, #48]	; (8001b68 <MX_DMA_Init+0x3c>)
 8001b38:	6b1b      	ldr	r3, [r3, #48]	; 0x30
 8001b3a:	4a0b      	ldr	r2, [pc, #44]	; (8001b68 <MX_DMA_Init+0x3c>)
 8001b3c:	f443 0380 	orr.w	r3, r3, #4194304	; 0x400000
 8001b40:	6313      	str	r3, [r2, #48]	; 0x30
 8001b42:	4b09      	ldr	r3, [pc, #36]	; (8001b68 <MX_DMA_Init+0x3c>)
 8001b44:	6b1b      	ldr	r3, [r3, #48]	; 0x30
 8001b46:	f403 0380 	and.w	r3, r3, #4194304	; 0x400000
 8001b4a:	607b      	str	r3, [r7, #4]
 8001b4c:	687b      	ldr	r3, [r7, #4]

  /* DMA interrupt init */
  /* DMA2_Stream1_IRQn interrupt configuration */
  HAL_NVIC_SetPriority(DMA2_Stream1_IRQn, 0, 0);
 8001b4e:	2200      	movs	r2, #0
 8001b50:	2100      	movs	r1, #0
 8001b52:	2039      	movs	r0, #57	; 0x39
 8001b54:	f001 f887 	bl	8002c66 <HAL_NVIC_SetPriority>
  HAL_NVIC_EnableIRQ(DMA2_Stream1_IRQn);
 8001b58:	2039      	movs	r0, #57	; 0x39
 8001b5a:	f001 f8a0 	bl	8002c9e <HAL_NVIC_EnableIRQ>

}
 8001b5e:	bf00      	nop
 8001b60:	3708      	adds	r7, #8
 8001b62:	46bd      	mov	sp, r7
 8001b64:	bd80      	pop	{r7, pc}
 8001b66:	bf00      	nop
 8001b68:	40023800 	.word	0x40023800

08001b6c <MX_GPIO_Init>:
  * @brief GPIO Initialization Function
  * @param None
  * @retval None
  */
static void MX_GPIO_Init(void)
{
 8001b6c:	b580      	push	{r7, lr}
 8001b6e:	b08a      	sub	sp, #40	; 0x28
 8001b70:	af00      	add	r7, sp, #0
  GPIO_InitTypeDef GPIO_InitStruct = {0};
 8001b72:	f107 0314 	add.w	r3, r7, #20
 8001b76:	2200      	movs	r2, #0
 8001b78:	601a      	str	r2, [r3, #0]
 8001b7a:	605a      	str	r2, [r3, #4]
 8001b7c:	609a      	str	r2, [r3, #8]
 8001b7e:	60da      	str	r2, [r3, #12]
 8001b80:	611a      	str	r2, [r3, #16]

  /* GPIO Ports Clock Enable */
  __HAL_RCC_GPIOH_CLK_ENABLE();
 8001b82:	2300      	movs	r3, #0
 8001b84:	613b      	str	r3, [r7, #16]
 8001b86:	4b38      	ldr	r3, [pc, #224]	; (8001c68 <MX_GPIO_Init+0xfc>)
 8001b88:	6b1b      	ldr	r3, [r3, #48]	; 0x30
 8001b8a:	4a37      	ldr	r2, [pc, #220]	; (8001c68 <MX_GPIO_Init+0xfc>)
 8001b8c:	f043 0380 	orr.w	r3, r3, #128	; 0x80
 8001b90:	6313      	str	r3, [r2, #48]	; 0x30
 8001b92:	4b35      	ldr	r3, [pc, #212]	; (8001c68 <MX_GPIO_Init+0xfc>)
 8001b94:	6b1b      	ldr	r3, [r3, #48]	; 0x30
 8001b96:	f003 0380 	and.w	r3, r3, #128	; 0x80
 8001b9a:	613b      	str	r3, [r7, #16]
 8001b9c:	693b      	ldr	r3, [r7, #16]
  __HAL_RCC_GPIOA_CLK_ENABLE();
 8001b9e:	2300      	movs	r3, #0
 8001ba0:	60fb      	str	r3, [r7, #12]
 8001ba2:	4b31      	ldr	r3, [pc, #196]	; (8001c68 <MX_GPIO_Init+0xfc>)
 8001ba4:	6b1b      	ldr	r3, [r3, #48]	; 0x30
 8001ba6:	4a30      	ldr	r2, [pc, #192]	; (8001c68 <MX_GPIO_Init+0xfc>)
 8001ba8:	f043 0301 	orr.w	r3, r3, #1
 8001bac:	6313      	str	r3, [r2, #48]	; 0x30
 8001bae:	4b2e      	ldr	r3, [pc, #184]	; (8001c68 <MX_GPIO_Init+0xfc>)
 8001bb0:	6b1b      	ldr	r3, [r3, #48]	; 0x30
 8001bb2:	f003 0301 	and.w	r3, r3, #1
 8001bb6:	60fb      	str	r3, [r7, #12]
 8001bb8:	68fb      	ldr	r3, [r7, #12]
  __HAL_RCC_GPIOC_CLK_ENABLE();
 8001bba:	2300      	movs	r3, #0
 8001bbc:	60bb      	str	r3, [r7, #8]
 8001bbe:	4b2a      	ldr	r3, [pc, #168]	; (8001c68 <MX_GPIO_Init+0xfc>)
 8001bc0:	6b1b      	ldr	r3, [r3, #48]	; 0x30
 8001bc2:	4a29      	ldr	r2, [pc, #164]	; (8001c68 <MX_GPIO_Init+0xfc>)
 8001bc4:	f043 0304 	orr.w	r3, r3, #4
 8001bc8:	6313      	str	r3, [r2, #48]	; 0x30
 8001bca:	4b27      	ldr	r3, [pc, #156]	; (8001c68 <MX_GPIO_Init+0xfc>)
 8001bcc:	6b1b      	ldr	r3, [r3, #48]	; 0x30
 8001bce:	f003 0304 	and.w	r3, r3, #4
 8001bd2:	60bb      	str	r3, [r7, #8]
 8001bd4:	68bb      	ldr	r3, [r7, #8]
  __HAL_RCC_GPIOE_CLK_ENABLE();
 8001bd6:	2300      	movs	r3, #0
 8001bd8:	607b      	str	r3, [r7, #4]
 8001bda:	4b23      	ldr	r3, [pc, #140]	; (8001c68 <MX_GPIO_Init+0xfc>)
 8001bdc:	6b1b      	ldr	r3, [r3, #48]	; 0x30
 8001bde:	4a22      	ldr	r2, [pc, #136]	; (8001c68 <MX_GPIO_Init+0xfc>)
 8001be0:	f043 0310 	orr.w	r3, r3, #16
 8001be4:	6313      	str	r3, [r2, #48]	; 0x30
 8001be6:	4b20      	ldr	r3, [pc, #128]	; (8001c68 <MX_GPIO_Init+0xfc>)
 8001be8:	6b1b      	ldr	r3, [r3, #48]	; 0x30
 8001bea:	f003 0310 	and.w	r3, r3, #16
 8001bee:	607b      	str	r3, [r7, #4]
 8001bf0:	687b      	ldr	r3, [r7, #4]
  __HAL_RCC_GPIOG_CLK_ENABLE();
 8001bf2:	2300      	movs	r3, #0
 8001bf4:	603b      	str	r3, [r7, #0]
 8001bf6:	4b1c      	ldr	r3, [pc, #112]	; (8001c68 <MX_GPIO_Init+0xfc>)
 8001bf8:	6b1b      	ldr	r3, [r3, #48]	; 0x30
 8001bfa:	4a1b      	ldr	r2, [pc, #108]	; (8001c68 <MX_GPIO_Init+0xfc>)
 8001bfc:	f043 0340 	orr.w	r3, r3, #64	; 0x40
 8001c00:	6313      	str	r3, [r2, #48]	; 0x30
 8001c02:	4b19      	ldr	r3, [pc, #100]	; (8001c68 <MX_GPIO_Init+0xfc>)
 8001c04:	6b1b      	ldr	r3, [r3, #48]	; 0x30
 8001c06:	f003 0340 	and.w	r3, r3, #64	; 0x40
 8001c0a:	603b      	str	r3, [r7, #0]
 8001c0c:	683b      	ldr	r3, [r7, #0]

  /*Configure GPIO pin Output Level */
  HAL_GPIO_WritePin(bmp280_CS_GPIO_Port, bmp280_CS_Pin, GPIO_PIN_RESET);
 8001c0e:	2200      	movs	r2, #0
 8001c10:	2110      	movs	r1, #16
 8001c12:	4816      	ldr	r0, [pc, #88]	; (8001c6c <MX_GPIO_Init+0x100>)
 8001c14:	f001 fd7a 	bl	800370c <HAL_GPIO_WritePin>

  /*Configure GPIO pin Output Level */
  HAL_GPIO_WritePin(GPIOG, Heater_Pin|Door_Pin|Heartbeat_Pin|Alert_Pin, GPIO_PIN_RESET);
 8001c18:	2200      	movs	r2, #0
 8001c1a:	f44f 41f0 	mov.w	r1, #30720	; 0x7800
 8001c1e:	4814      	ldr	r0, [pc, #80]	; (8001c70 <MX_GPIO_Init+0x104>)
 8001c20:	f001 fd74 	bl	800370c <HAL_GPIO_WritePin>

  /*Configure GPIO pin : bmp280_CS_Pin */
  GPIO_InitStruct.Pin = bmp280_CS_Pin;
 8001c24:	2310      	movs	r3, #16
 8001c26:	617b      	str	r3, [r7, #20]
  GPIO_InitStruct.Mode = GPIO_MODE_OUTPUT_PP;
 8001c28:	2301      	movs	r3, #1
 8001c2a:	61bb      	str	r3, [r7, #24]
  GPIO_InitStruct.Pull = GPIO_NOPULL;
 8001c2c:	2300      	movs	r3, #0
 8001c2e:	61fb      	str	r3, [r7, #28]
  GPIO_InitStruct.Speed = GPIO_SPEED_FREQ_LOW;
 8001c30:	2300      	movs	r3, #0
 8001c32:	623b      	str	r3, [r7, #32]
  HAL_GPIO_Init(bmp280_CS_GPIO_Port, &GPIO_InitStruct);
 8001c34:	f107 0314 	add.w	r3, r7, #20
 8001c38:	4619      	mov	r1, r3
 8001c3a:	480c      	ldr	r0, [pc, #48]	; (8001c6c <MX_GPIO_Init+0x100>)
 8001c3c:	f001 fbba 	bl	80033b4 <HAL_GPIO_Init>

  /*Configure GPIO pins : Heater_Pin Door_Pin Heartbeat_Pin Alert_Pin */
  GPIO_InitStruct.Pin = Heater_Pin|Door_Pin|Heartbeat_Pin|Alert_Pin;
 8001c40:	f44f 43f0 	mov.w	r3, #30720	; 0x7800
 8001c44:	617b      	str	r3, [r7, #20]
  GPIO_InitStruct.Mode = GPIO_MODE_OUTPUT_PP;
 8001c46:	2301      	movs	r3, #1
 8001c48:	61bb      	str	r3, [r7, #24]
  GPIO_InitStruct.Pull = GPIO_NOPULL;
 8001c4a:	2300      	movs	r3, #0
 8001c4c:	61fb      	str	r3, [r7, #28]
  GPIO_InitStruct.Speed = GPIO_SPEED_FREQ_LOW;
 8001c4e:	2300      	movs	r3, #0
 8001c50:	623b      	str	r3, [r7, #32]
  HAL_GPIO_Init(GPIOG, &GPIO_InitStruct);
 8001c52:	f107 0314 	add.w	r3, r7, #20
 8001c56:	4619      	mov	r1, r3
 8001c58:	4805      	ldr	r0, [pc, #20]	; (8001c70 <MX_GPIO_Init+0x104>)
 8001c5a:	f001 fbab 	bl	80033b4 <HAL_GPIO_Init>

}
 8001c5e:	bf00      	nop
 8001c60:	3728      	adds	r7, #40	; 0x28
 8001c62:	46bd      	mov	sp, r7
 8001c64:	bd80      	pop	{r7, pc}
 8001c66:	bf00      	nop
 8001c68:	40023800 	.word	0x40023800
 8001c6c:	40020800 	.word	0x40020800
 8001c70:	40021800 	.word	0x40021800

08001c74 <Error_Handler>:
/**
  * @brief  This function is executed in case of error occurrence.
  * @retval None
  */
void Error_Handler(void)
{
 8001c74:	b480      	push	{r7}
 8001c76:	af00      	add	r7, sp, #0
  \details Disables IRQ interrupts by setting the I-bit in the CPSR.
           Can only be executed in Privileged modes.
 */
__STATIC_FORCEINLINE void __disable_irq(void)
{
  __ASM volatile ("cpsid i" : : : "memory");
 8001c78:	b672      	cpsid	i
}
 8001c7a:	bf00      	nop
  /* USER CODE BEGIN Error_Handler_Debug */
  /* User can add his own implementation to report the HAL error return state */
  __disable_irq();
  while (1)
 8001c7c:	e7fe      	b.n	8001c7c <Error_Handler+0x8>
	...

08001c80 <HAL_MspInit>:
void HAL_TIM_MspPostInit(TIM_HandleTypeDef *htim);
                    /**
  * Initializes the Global MSP.
  */
void HAL_MspInit(void)
{
 8001c80:	b580      	push	{r7, lr}
 8001c82:	b082      	sub	sp, #8
 8001c84:	af00      	add	r7, sp, #0
  /* USER CODE BEGIN MspInit 0 */

  /* USER CODE END MspInit 0 */

  __HAL_RCC_SYSCFG_CLK_ENABLE();
 8001c86:	2300      	movs	r3, #0
 8001c88:	607b      	str	r3, [r7, #4]
 8001c8a:	4b10      	ldr	r3, [pc, #64]	; (8001ccc <HAL_MspInit+0x4c>)
 8001c8c:	6c5b      	ldr	r3, [r3, #68]	; 0x44
 8001c8e:	4a0f      	ldr	r2, [pc, #60]	; (8001ccc <HAL_MspInit+0x4c>)
 8001c90:	f443 4380 	orr.w	r3, r3, #16384	; 0x4000
 8001c94:	6453      	str	r3, [r2, #68]	; 0x44
 8001c96:	4b0d      	ldr	r3, [pc, #52]	; (8001ccc <HAL_MspInit+0x4c>)
 8001c98:	6c5b      	ldr	r3, [r3, #68]	; 0x44
 8001c9a:	f403 4380 	and.w	r3, r3, #16384	; 0x4000
 8001c9e:	607b      	str	r3, [r7, #4]
 8001ca0:	687b      	ldr	r3, [r7, #4]
  __HAL_RCC_PWR_CLK_ENABLE();
 8001ca2:	2300      	movs	r3, #0
 8001ca4:	603b      	str	r3, [r7, #0]
 8001ca6:	4b09      	ldr	r3, [pc, #36]	; (8001ccc <HAL_MspInit+0x4c>)
 8001ca8:	6c1b      	ldr	r3, [r3, #64]	; 0x40
 8001caa:	4a08      	ldr	r2, [pc, #32]	; (8001ccc <HAL_MspInit+0x4c>)
 8001cac:	f043 5380 	orr.w	r3, r3, #268435456	; 0x10000000
 8001cb0:	6413      	str	r3, [r2, #64]	; 0x40
 8001cb2:	4b06      	ldr	r3, [pc, #24]	; (8001ccc <HAL_MspInit+0x4c>)
 8001cb4:	6c1b      	ldr	r3, [r3, #64]	; 0x40
 8001cb6:	f003 5380 	and.w	r3, r3, #268435456	; 0x10000000
 8001cba:	603b      	str	r3, [r7, #0]
 8001cbc:	683b      	ldr	r3, [r7, #0]

  HAL_NVIC_SetPriorityGrouping(NVIC_PRIORITYGROUP_0);
 8001cbe:	2007      	movs	r0, #7
 8001cc0:	f000 ffc6 	bl	8002c50 <HAL_NVIC_SetPriorityGrouping>
  /* System interrupt init*/

  /* USER CODE BEGIN MspInit 1 */

  /* USER CODE END MspInit 1 */
}
 8001cc4:	bf00      	nop
 8001cc6:	3708      	adds	r7, #8
 8001cc8:	46bd      	mov	sp, r7
 8001cca:	bd80      	pop	{r7, pc}
 8001ccc:	40023800 	.word	0x40023800

08001cd0 <HAL_ADC_MspInit>:
* This function configures the hardware resources used in this example
* @param hadc: ADC handle pointer
* @retval None
*/
void HAL_ADC_MspInit(ADC_HandleTypeDef* hadc)
{
 8001cd0:	b580      	push	{r7, lr}
 8001cd2:	b08a      	sub	sp, #40	; 0x28
 8001cd4:	af00      	add	r7, sp, #0
 8001cd6:	6078      	str	r0, [r7, #4]
  GPIO_InitTypeDef GPIO_InitStruct = {0};
 8001cd8:	f107 0314 	add.w	r3, r7, #20
 8001cdc:	2200      	movs	r2, #0
 8001cde:	601a      	str	r2, [r3, #0]
 8001ce0:	605a      	str	r2, [r3, #4]
 8001ce2:	609a      	str	r2, [r3, #8]
 8001ce4:	60da      	str	r2, [r3, #12]
 8001ce6:	611a      	str	r2, [r3, #16]
  if(hadc->Instance==ADC1)
 8001ce8:	687b      	ldr	r3, [r7, #4]
 8001cea:	681b      	ldr	r3, [r3, #0]
 8001cec:	4a17      	ldr	r2, [pc, #92]	; (8001d4c <HAL_ADC_MspInit+0x7c>)
 8001cee:	4293      	cmp	r3, r2
 8001cf0:	d127      	bne.n	8001d42 <HAL_ADC_MspInit+0x72>
  {
  /* USER CODE BEGIN ADC1_MspInit 0 */

  /* USER CODE END ADC1_MspInit 0 */
    /* Peripheral clock enable */
    __HAL_RCC_ADC1_CLK_ENABLE();
 8001cf2:	2300      	movs	r3, #0
 8001cf4:	613b      	str	r3, [r7, #16]
 8001cf6:	4b16      	ldr	r3, [pc, #88]	; (8001d50 <HAL_ADC_MspInit+0x80>)
 8001cf8:	6c5b      	ldr	r3, [r3, #68]	; 0x44
 8001cfa:	4a15      	ldr	r2, [pc, #84]	; (8001d50 <HAL_ADC_MspInit+0x80>)
 8001cfc:	f443 7380 	orr.w	r3, r3, #256	; 0x100
 8001d00:	6453      	str	r3, [r2, #68]	; 0x44
 8001d02:	4b13      	ldr	r3, [pc, #76]	; (8001d50 <HAL_ADC_MspInit+0x80>)
 8001d04:	6c5b      	ldr	r3, [r3, #68]	; 0x44
 8001d06:	f403 7380 	and.w	r3, r3, #256	; 0x100
 8001d0a:	613b      	str	r3, [r7, #16]
 8001d0c:	693b      	ldr	r3, [r7, #16]

    __HAL_RCC_GPIOA_CLK_ENABLE();
 8001d0e:	2300      	movs	r3, #0
 8001d10:	60fb      	str	r3, [r7, #12]
 8001d12:	4b0f      	ldr	r3, [pc, #60]	; (8001d50 <HAL_ADC_MspInit+0x80>)
 8001d14:	6b1b      	ldr	r3, [r3, #48]	; 0x30
 8001d16:	4a0e      	ldr	r2, [pc, #56]	; (8001d50 <HAL_ADC_MspInit+0x80>)
 8001d18:	f043 0301 	orr.w	r3, r3, #1
 8001d1c:	6313      	str	r3, [r2, #48]	; 0x30
 8001d1e:	4b0c      	ldr	r3, [pc, #48]	; (8001d50 <HAL_ADC_MspInit+0x80>)
 8001d20:	6b1b      	ldr	r3, [r3, #48]	; 0x30
 8001d22:	f003 0301 	and.w	r3, r3, #1
 8001d26:	60fb      	str	r3, [r7, #12]
 8001d28:	68fb      	ldr	r3, [r7, #12]
    /**ADC1 GPIO Configuration
    PA0/WKUP     ------> ADC1_IN0
    */
    GPIO_InitStruct.Pin = GPIO_PIN_0;
 8001d2a:	2301      	movs	r3, #1
 8001d2c:	617b      	str	r3, [r7, #20]
    GPIO_InitStruct.Mode = GPIO_MODE_ANALOG;
 8001d2e:	2303      	movs	r3, #3
 8001d30:	61bb      	str	r3, [r7, #24]
    GPIO_InitStruct.Pull = GPIO_NOPULL;
 8001d32:	2300      	movs	r3, #0
 8001d34:	61fb      	str	r3, [r7, #28]
    HAL_GPIO_Init(GPIOA, &GPIO_InitStruct);
 8001d36:	f107 0314 	add.w	r3, r7, #20
 8001d3a:	4619      	mov	r1, r3
 8001d3c:	4805      	ldr	r0, [pc, #20]	; (8001d54 <HAL_ADC_MspInit+0x84>)
 8001d3e:	f001 fb39 	bl	80033b4 <HAL_GPIO_Init>
  /* USER CODE BEGIN ADC1_MspInit 1 */

  /* USER CODE END ADC1_MspInit 1 */
  }

}
 8001d42:	bf00      	nop
 8001d44:	3728      	adds	r7, #40	; 0x28
 8001d46:	46bd      	mov	sp, r7
 8001d48:	bd80      	pop	{r7, pc}
 8001d4a:	bf00      	nop
 8001d4c:	40012000 	.word	0x40012000
 8001d50:	40023800 	.word	0x40023800
 8001d54:	40020000 	.word	0x40020000

08001d58 <HAL_SPI_MspInit>:
* This function configures the hardware resources used in this example
* @param hspi: SPI handle pointer
* @retval None
*/
void HAL_SPI_MspInit(SPI_HandleTypeDef* hspi)
{
 8001d58:	b580      	push	{r7, lr}
 8001d5a:	b08a      	sub	sp, #40	; 0x28
 8001d5c:	af00      	add	r7, sp, #0
 8001d5e:	6078      	str	r0, [r7, #4]
  GPIO_InitTypeDef GPIO_InitStruct = {0};
 8001d60:	f107 0314 	add.w	r3, r7, #20
 8001d64:	2200      	movs	r2, #0
 8001d66:	601a      	str	r2, [r3, #0]
 8001d68:	605a      	str	r2, [r3, #4]
 8001d6a:	609a      	str	r2, [r3, #8]
 8001d6c:	60da      	str	r2, [r3, #12]
 8001d6e:	611a      	str	r2, [r3, #16]
  if(hspi->Instance==SPI1)
 8001d70:	687b      	ldr	r3, [r7, #4]
 8001d72:	681b      	ldr	r3, [r3, #0]
 8001d74:	4a19      	ldr	r2, [pc, #100]	; (8001ddc <HAL_SPI_MspInit+0x84>)
 8001d76:	4293      	cmp	r3, r2
 8001d78:	d12b      	bne.n	8001dd2 <HAL_SPI_MspInit+0x7a>
  {
  /* USER CODE BEGIN SPI1_MspInit 0 */

  /* USER CODE END SPI1_MspInit 0 */
    /* Peripheral clock enable */
    __HAL_RCC_SPI1_CLK_ENABLE();
 8001d7a:	2300      	movs	r3, #0
 8001d7c:	613b      	str	r3, [r7, #16]
 8001d7e:	4b18      	ldr	r3, [pc, #96]	; (8001de0 <HAL_SPI_MspInit+0x88>)
 8001d80:	6c5b      	ldr	r3, [r3, #68]	; 0x44
 8001d82:	4a17      	ldr	r2, [pc, #92]	; (8001de0 <HAL_SPI_MspInit+0x88>)
 8001d84:	f443 5380 	orr.w	r3, r3, #4096	; 0x1000
 8001d88:	6453      	str	r3, [r2, #68]	; 0x44
 8001d8a:	4b15      	ldr	r3, [pc, #84]	; (8001de0 <HAL_SPI_MspInit+0x88>)
 8001d8c:	6c5b      	ldr	r3, [r3, #68]	; 0x44
 8001d8e:	f403 5380 	and.w	r3, r3, #4096	; 0x1000
 8001d92:	613b      	str	r3, [r7, #16]
 8001d94:	693b      	ldr	r3, [r7, #16]

    __HAL_RCC_GPIOA_CLK_ENABLE();
 8001d96:	2300      	movs	r3, #0
 8001d98:	60fb      	str	r3, [r7, #12]
 8001d9a:	4b11      	ldr	r3, [pc, #68]	; (8001de0 <HAL_SPI_MspInit+0x88>)
 8001d9c:	6b1b      	ldr	r3, [r3, #48]	; 0x30
 8001d9e:	4a10      	ldr	r2, [pc, #64]	; (8001de0 <HAL_SPI_MspInit+0x88>)
 8001da0:	f043 0301 	orr.w	r3, r3, #1
 8001da4:	6313      	str	r3, [r2, #48]	; 0x30
 8001da6:	4b0e      	ldr	r3, [pc, #56]	; (8001de0 <HAL_SPI_MspInit+0x88>)
 8001da8:	6b1b      	ldr	r3, [r3, #48]	; 0x30
 8001daa:	f003 0301 	and.w	r3, r3, #1
 8001dae:	60fb      	str	r3, [r7, #12]
 8001db0:	68fb      	ldr	r3, [r7, #12]
    /**SPI1 GPIO Configuration
    PA5     ------> SPI1_SCK
    PA6     ------> SPI1_MISO
    PA7     ------> SPI1_MOSI
    */
    GPIO_InitStruct.Pin = GPIO_PIN_5|GPIO_PIN_6|GPIO_PIN_7;
 8001db2:	23e0      	movs	r3, #224	; 0xe0
 8001db4:	617b      	str	r3, [r7, #20]
    GPIO_InitStruct.Mode = GPIO_MODE_AF_PP;
 8001db6:	2302      	movs	r3, #2
 8001db8:	61bb      	str	r3, [r7, #24]
    GPIO_InitStruct.Pull = GPIO_NOPULL;
 8001dba:	2300      	movs	r3, #0
 8001dbc:	61fb      	str	r3, [r7, #28]
    GPIO_InitStruct.Speed = GPIO_SPEED_FREQ_VERY_HIGH;
 8001dbe:	2303      	movs	r3, #3
 8001dc0:	623b      	str	r3, [r7, #32]
    GPIO_InitStruct.Alternate = GPIO_AF5_SPI1;
 8001dc2:	2305      	movs	r3, #5
 8001dc4:	627b      	str	r3, [r7, #36]	; 0x24
    HAL_GPIO_Init(GPIOA, &GPIO_InitStruct);
 8001dc6:	f107 0314 	add.w	r3, r7, #20
 8001dca:	4619      	mov	r1, r3
 8001dcc:	4805      	ldr	r0, [pc, #20]	; (8001de4 <HAL_SPI_MspInit+0x8c>)
 8001dce:	f001 faf1 	bl	80033b4 <HAL_GPIO_Init>
  /* USER CODE BEGIN SPI1_MspInit 1 */

  /* USER CODE END SPI1_MspInit 1 */
  }

}
 8001dd2:	bf00      	nop
 8001dd4:	3728      	adds	r7, #40	; 0x28
 8001dd6:	46bd      	mov	sp, r7
 8001dd8:	bd80      	pop	{r7, pc}
 8001dda:	bf00      	nop
 8001ddc:	40013000 	.word	0x40013000
 8001de0:	40023800 	.word	0x40023800
 8001de4:	40020000 	.word	0x40020000

08001de8 <HAL_TIM_PWM_MspInit>:
* This function configures the hardware resources used in this example
* @param htim_pwm: TIM_PWM handle pointer
* @retval None
*/
void HAL_TIM_PWM_MspInit(TIM_HandleTypeDef* htim_pwm)
{
 8001de8:	b580      	push	{r7, lr}
 8001dea:	b084      	sub	sp, #16
 8001dec:	af00      	add	r7, sp, #0
 8001dee:	6078      	str	r0, [r7, #4]
  if(htim_pwm->Instance==TIM1)
 8001df0:	687b      	ldr	r3, [r7, #4]
 8001df2:	681b      	ldr	r3, [r3, #0]
 8001df4:	4a23      	ldr	r2, [pc, #140]	; (8001e84 <HAL_TIM_PWM_MspInit+0x9c>)
 8001df6:	4293      	cmp	r3, r2
 8001df8:	d13f      	bne.n	8001e7a <HAL_TIM_PWM_MspInit+0x92>
  {
  /* USER CODE BEGIN TIM1_MspInit 0 */

  /* USER CODE END TIM1_MspInit 0 */
    /* Peripheral clock enable */
    __HAL_RCC_TIM1_CLK_ENABLE();
 8001dfa:	2300      	movs	r3, #0
 8001dfc:	60fb      	str	r3, [r7, #12]
 8001dfe:	4b22      	ldr	r3, [pc, #136]	; (8001e88 <HAL_TIM_PWM_MspInit+0xa0>)
 8001e00:	6c5b      	ldr	r3, [r3, #68]	; 0x44
 8001e02:	4a21      	ldr	r2, [pc, #132]	; (8001e88 <HAL_TIM_PWM_MspInit+0xa0>)
 8001e04:	f043 0301 	orr.w	r3, r3, #1
 8001e08:	6453      	str	r3, [r2, #68]	; 0x44
 8001e0a:	4b1f      	ldr	r3, [pc, #124]	; (8001e88 <HAL_TIM_PWM_MspInit+0xa0>)
 8001e0c:	6c5b      	ldr	r3, [r3, #68]	; 0x44
 8001e0e:	f003 0301 	and.w	r3, r3, #1
 8001e12:	60fb      	str	r3, [r7, #12]
 8001e14:	68fb      	ldr	r3, [r7, #12]

    /* TIM1 DMA Init */
    /* TIM1_CH1 Init */
    hdma_tim1_ch1.Instance = DMA2_Stream1;
 8001e16:	4b1d      	ldr	r3, [pc, #116]	; (8001e8c <HAL_TIM_PWM_MspInit+0xa4>)
 8001e18:	4a1d      	ldr	r2, [pc, #116]	; (8001e90 <HAL_TIM_PWM_MspInit+0xa8>)
 8001e1a:	601a      	str	r2, [r3, #0]
    hdma_tim1_ch1.Init.Channel = DMA_CHANNEL_6;
 8001e1c:	4b1b      	ldr	r3, [pc, #108]	; (8001e8c <HAL_TIM_PWM_MspInit+0xa4>)
 8001e1e:	f04f 6240 	mov.w	r2, #201326592	; 0xc000000
 8001e22:	605a      	str	r2, [r3, #4]
    hdma_tim1_ch1.Init.Direction = DMA_MEMORY_TO_PERIPH;
 8001e24:	4b19      	ldr	r3, [pc, #100]	; (8001e8c <HAL_TIM_PWM_MspInit+0xa4>)
 8001e26:	2240      	movs	r2, #64	; 0x40
 8001e28:	609a      	str	r2, [r3, #8]
    hdma_tim1_ch1.Init.PeriphInc = DMA_PINC_DISABLE;
 8001e2a:	4b18      	ldr	r3, [pc, #96]	; (8001e8c <HAL_TIM_PWM_MspInit+0xa4>)
 8001e2c:	2200      	movs	r2, #0
 8001e2e:	60da      	str	r2, [r3, #12]
    hdma_tim1_ch1.Init.MemInc = DMA_MINC_ENABLE;
 8001e30:	4b16      	ldr	r3, [pc, #88]	; (8001e8c <HAL_TIM_PWM_MspInit+0xa4>)
 8001e32:	f44f 6280 	mov.w	r2, #1024	; 0x400
 8001e36:	611a      	str	r2, [r3, #16]
    hdma_tim1_ch1.Init.PeriphDataAlignment = DMA_PDATAALIGN_HALFWORD;
 8001e38:	4b14      	ldr	r3, [pc, #80]	; (8001e8c <HAL_TIM_PWM_MspInit+0xa4>)
 8001e3a:	f44f 6200 	mov.w	r2, #2048	; 0x800
 8001e3e:	615a      	str	r2, [r3, #20]
    hdma_tim1_ch1.Init.MemDataAlignment = DMA_MDATAALIGN_HALFWORD;
 8001e40:	4b12      	ldr	r3, [pc, #72]	; (8001e8c <HAL_TIM_PWM_MspInit+0xa4>)
 8001e42:	f44f 5200 	mov.w	r2, #8192	; 0x2000
 8001e46:	619a      	str	r2, [r3, #24]
    hdma_tim1_ch1.Init.Mode = DMA_CIRCULAR;
 8001e48:	4b10      	ldr	r3, [pc, #64]	; (8001e8c <HAL_TIM_PWM_MspInit+0xa4>)
 8001e4a:	f44f 7280 	mov.w	r2, #256	; 0x100
 8001e4e:	61da      	str	r2, [r3, #28]
    hdma_tim1_ch1.Init.Priority = DMA_PRIORITY_MEDIUM;
 8001e50:	4b0e      	ldr	r3, [pc, #56]	; (8001e8c <HAL_TIM_PWM_MspInit+0xa4>)
 8001e52:	f44f 3280 	mov.w	r2, #65536	; 0x10000
 8001e56:	621a      	str	r2, [r3, #32]
    hdma_tim1_ch1.Init.FIFOMode = DMA_FIFOMODE_DISABLE;
 8001e58:	4b0c      	ldr	r3, [pc, #48]	; (8001e8c <HAL_TIM_PWM_MspInit+0xa4>)
 8001e5a:	2200      	movs	r2, #0
 8001e5c:	625a      	str	r2, [r3, #36]	; 0x24
    if (HAL_DMA_Init(&hdma_tim1_ch1) != HAL_OK)
 8001e5e:	480b      	ldr	r0, [pc, #44]	; (8001e8c <HAL_TIM_PWM_MspInit+0xa4>)
 8001e60:	f000 ff38 	bl	8002cd4 <HAL_DMA_Init>
 8001e64:	4603      	mov	r3, r0
 8001e66:	2b00      	cmp	r3, #0
 8001e68:	d001      	beq.n	8001e6e <HAL_TIM_PWM_MspInit+0x86>
    {
      Error_Handler();
 8001e6a:	f7ff ff03 	bl	8001c74 <Error_Handler>
    }

    __HAL_LINKDMA(htim_pwm,hdma[TIM_DMA_ID_CC1],hdma_tim1_ch1);
 8001e6e:	687b      	ldr	r3, [r7, #4]
 8001e70:	4a06      	ldr	r2, [pc, #24]	; (8001e8c <HAL_TIM_PWM_MspInit+0xa4>)
 8001e72:	625a      	str	r2, [r3, #36]	; 0x24
 8001e74:	4a05      	ldr	r2, [pc, #20]	; (8001e8c <HAL_TIM_PWM_MspInit+0xa4>)
 8001e76:	687b      	ldr	r3, [r7, #4]
 8001e78:	6393      	str	r3, [r2, #56]	; 0x38
  /* USER CODE BEGIN TIM1_MspInit 1 */

  /* USER CODE END TIM1_MspInit 1 */
  }

}
 8001e7a:	bf00      	nop
 8001e7c:	3710      	adds	r7, #16
 8001e7e:	46bd      	mov	sp, r7
 8001e80:	bd80      	pop	{r7, pc}
 8001e82:	bf00      	nop
 8001e84:	40010000 	.word	0x40010000
 8001e88:	40023800 	.word	0x40023800
 8001e8c:	200002e0 	.word	0x200002e0
 8001e90:	40026428 	.word	0x40026428

08001e94 <HAL_TIM_MspPostInit>:

void HAL_TIM_MspPostInit(TIM_HandleTypeDef* htim)
{
 8001e94:	b580      	push	{r7, lr}
 8001e96:	b088      	sub	sp, #32
 8001e98:	af00      	add	r7, sp, #0
 8001e9a:	6078      	str	r0, [r7, #4]
  GPIO_InitTypeDef GPIO_InitStruct = {0};
 8001e9c:	f107 030c 	add.w	r3, r7, #12
 8001ea0:	2200      	movs	r2, #0
 8001ea2:	601a      	str	r2, [r3, #0]
 8001ea4:	605a      	str	r2, [r3, #4]
 8001ea6:	609a      	str	r2, [r3, #8]
 8001ea8:	60da      	str	r2, [r3, #12]
 8001eaa:	611a      	str	r2, [r3, #16]
  if(htim->Instance==TIM1)
 8001eac:	687b      	ldr	r3, [r7, #4]
 8001eae:	681b      	ldr	r3, [r3, #0]
 8001eb0:	4a12      	ldr	r2, [pc, #72]	; (8001efc <HAL_TIM_MspPostInit+0x68>)
 8001eb2:	4293      	cmp	r3, r2
 8001eb4:	d11e      	bne.n	8001ef4 <HAL_TIM_MspPostInit+0x60>
  {
  /* USER CODE BEGIN TIM1_MspPostInit 0 */

  /* USER CODE END TIM1_MspPostInit 0 */

    __HAL_RCC_GPIOE_CLK_ENABLE();
 8001eb6:	2300      	movs	r3, #0
 8001eb8:	60bb      	str	r3, [r7, #8]
 8001eba:	4b11      	ldr	r3, [pc, #68]	; (8001f00 <HAL_TIM_MspPostInit+0x6c>)
 8001ebc:	6b1b      	ldr	r3, [r3, #48]	; 0x30
 8001ebe:	4a10      	ldr	r2, [pc, #64]	; (8001f00 <HAL_TIM_MspPostInit+0x6c>)
 8001ec0:	f043 0310 	orr.w	r3, r3, #16
 8001ec4:	6313      	str	r3, [r2, #48]	; 0x30
 8001ec6:	4b0e      	ldr	r3, [pc, #56]	; (8001f00 <HAL_TIM_MspPostInit+0x6c>)
 8001ec8:	6b1b      	ldr	r3, [r3, #48]	; 0x30
 8001eca:	f003 0310 	and.w	r3, r3, #16
 8001ece:	60bb      	str	r3, [r7, #8]
 8001ed0:	68bb      	ldr	r3, [r7, #8]
    /**TIM1 GPIO Configuration
    PE9     ------> TIM1_CH1
    */
    GPIO_InitStruct.Pin = GPIO_PIN_9;
 8001ed2:	f44f 7300 	mov.w	r3, #512	; 0x200
 8001ed6:	60fb      	str	r3, [r7, #12]
    GPIO_InitStruct.Mode = GPIO_MODE_AF_PP;
 8001ed8:	2302      	movs	r3, #2
 8001eda:	613b      	str	r3, [r7, #16]
    GPIO_InitStruct.Pull = GPIO_NOPULL;
 8001edc:	2300      	movs	r3, #0
 8001ede:	617b      	str	r3, [r7, #20]
    GPIO_InitStruct.Speed = GPIO_SPEED_FREQ_LOW;
 8001ee0:	2300      	movs	r3, #0
 8001ee2:	61bb      	str	r3, [r7, #24]
    GPIO_InitStruct.Alternate = GPIO_AF1_TIM1;
 8001ee4:	2301      	movs	r3, #1
 8001ee6:	61fb      	str	r3, [r7, #28]
    HAL_GPIO_Init(GPIOE, &GPIO_InitStruct);
 8001ee8:	f107 030c 	add.w	r3, r7, #12
 8001eec:	4619      	mov	r1, r3
 8001eee:	4805      	ldr	r0, [pc, #20]	; (8001f04 <HAL_TIM_MspPostInit+0x70>)
 8001ef0:	f001 fa60 	bl	80033b4 <HAL_GPIO_Init>
  /* USER CODE BEGIN TIM1_MspPostInit 1 */

  /* USER CODE END TIM1_MspPostInit 1 */
  }

}
 8001ef4:	bf00      	nop
 8001ef6:	3720      	adds	r7, #32
 8001ef8:	46bd      	mov	sp, r7
 8001efa:	bd80      	pop	{r7, pc}
 8001efc:	40010000 	.word	0x40010000
 8001f00:	40023800 	.word	0x40023800
 8001f04:	40021000 	.word	0x40021000

08001f08 <HAL_UART_MspInit>:
* This function configures the hardware resources used in this example
* @param huart: UART handle pointer
* @retval None
*/
void HAL_UART_MspInit(UART_HandleTypeDef* huart)
{
 8001f08:	b580      	push	{r7, lr}
 8001f0a:	b08a      	sub	sp, #40	; 0x28
 8001f0c:	af00      	add	r7, sp, #0
 8001f0e:	6078      	str	r0, [r7, #4]
  GPIO_InitTypeDef GPIO_InitStruct = {0};
 8001f10:	f107 0314 	add.w	r3, r7, #20
 8001f14:	2200      	movs	r2, #0
 8001f16:	601a      	str	r2, [r3, #0]
 8001f18:	605a      	str	r2, [r3, #4]
 8001f1a:	609a      	str	r2, [r3, #8]
 8001f1c:	60da      	str	r2, [r3, #12]
 8001f1e:	611a      	str	r2, [r3, #16]
  if(huart->Instance==USART1)
 8001f20:	687b      	ldr	r3, [r7, #4]
 8001f22:	681b      	ldr	r3, [r3, #0]
 8001f24:	4a19      	ldr	r2, [pc, #100]	; (8001f8c <HAL_UART_MspInit+0x84>)
 8001f26:	4293      	cmp	r3, r2
 8001f28:	d12c      	bne.n	8001f84 <HAL_UART_MspInit+0x7c>
  {
  /* USER CODE BEGIN USART1_MspInit 0 */

  /* USER CODE END USART1_MspInit 0 */
    /* Peripheral clock enable */
    __HAL_RCC_USART1_CLK_ENABLE();
 8001f2a:	2300      	movs	r3, #0
 8001f2c:	613b      	str	r3, [r7, #16]
 8001f2e:	4b18      	ldr	r3, [pc, #96]	; (8001f90 <HAL_UART_MspInit+0x88>)
 8001f30:	6c5b      	ldr	r3, [r3, #68]	; 0x44
 8001f32:	4a17      	ldr	r2, [pc, #92]	; (8001f90 <HAL_UART_MspInit+0x88>)
 8001f34:	f043 0310 	orr.w	r3, r3, #16
 8001f38:	6453      	str	r3, [r2, #68]	; 0x44
 8001f3a:	4b15      	ldr	r3, [pc, #84]	; (8001f90 <HAL_UART_MspInit+0x88>)
 8001f3c:	6c5b      	ldr	r3, [r3, #68]	; 0x44
 8001f3e:	f003 0310 	and.w	r3, r3, #16
 8001f42:	613b      	str	r3, [r7, #16]
 8001f44:	693b      	ldr	r3, [r7, #16]

    __HAL_RCC_GPIOA_CLK_ENABLE();
 8001f46:	2300      	movs	r3, #0
 8001f48:	60fb      	str	r3, [r7, #12]
 8001f4a:	4b11      	ldr	r3, [pc, #68]	; (8001f90 <HAL_UART_MspInit+0x88>)
 8001f4c:	6b1b      	ldr	r3, [r3, #48]	; 0x30
 8001f4e:	4a10      	ldr	r2, [pc, #64]	; (8001f90 <HAL_UART_MspInit+0x88>)
 8001f50:	f043 0301 	orr.w	r3, r3, #1
 8001f54:	6313      	str	r3, [r2, #48]	; 0x30
 8001f56:	4b0e      	ldr	r3, [pc, #56]	; (8001f90 <HAL_UART_MspInit+0x88>)
 8001f58:	6b1b      	ldr	r3, [r3, #48]	; 0x30
 8001f5a:	f003 0301 	and.w	r3, r3, #1
 8001f5e:	60fb      	str	r3, [r7, #12]
 8001f60:	68fb      	ldr	r3, [r7, #12]
    /**USART1 GPIO Configuration
    PA9     ------> USART1_TX
    PA10     ------> USART1_RX
    */
    GPIO_InitStruct.Pin = GPIO_PIN_9|GPIO_PIN_10;
 8001f62:	f44f 63c0 	mov.w	r3, #1536	; 0x600
 8001f66:	617b      	str	r3, [r7, #20]
    GPIO_InitStruct.Mode = GPIO_MODE_AF_PP;
 8001f68:	2302      	movs	r3, #2
 8001f6a:	61bb      	str	r3, [r7, #24]
    GPIO_InitStruct.Pull = GPIO_NOPULL;
 8001f6c:	2300      	movs	r3, #0
 8001f6e:	61fb      	str	r3, [r7, #28]
    GPIO_InitStruct.Speed = GPIO_SPEED_FREQ_VERY_HIGH;
 8001f70:	2303      	movs	r3, #3
 8001f72:	623b      	str	r3, [r7, #32]
    GPIO_InitStruct.Alternate = GPIO_AF7_USART1;
 8001f74:	2307      	movs	r3, #7
 8001f76:	627b      	str	r3, [r7, #36]	; 0x24
    HAL_GPIO_Init(GPIOA, &GPIO_InitStruct);
 8001f78:	f107 0314 	add.w	r3, r7, #20
 8001f7c:	4619      	mov	r1, r3
 8001f7e:	4805      	ldr	r0, [pc, #20]	; (8001f94 <HAL_UART_MspInit+0x8c>)
 8001f80:	f001 fa18 	bl	80033b4 <HAL_GPIO_Init>
  /* USER CODE BEGIN USART1_MspInit 1 */

  /* USER CODE END USART1_MspInit 1 */
  }

}
 8001f84:	bf00      	nop
 8001f86:	3728      	adds	r7, #40	; 0x28
 8001f88:	46bd      	mov	sp, r7
 8001f8a:	bd80      	pop	{r7, pc}
 8001f8c:	40011000 	.word	0x40011000
 8001f90:	40023800 	.word	0x40023800
 8001f94:	40020000 	.word	0x40020000

08001f98 <NMI_Handler>:
/******************************************************************************/
/**
  * @brief This function handles Non maskable interrupt.
  */
void NMI_Handler(void)
{
 8001f98:	b480      	push	{r7}
 8001f9a:	af00      	add	r7, sp, #0
  /* USER CODE BEGIN NonMaskableInt_IRQn 0 */

  /* USER CODE END NonMaskableInt_IRQn 0 */
  /* USER CODE BEGIN NonMaskableInt_IRQn 1 */
  while (1)
 8001f9c:	e7fe      	b.n	8001f9c <NMI_Handler+0x4>

08001f9e <HardFault_Handler>:

/**
  * @brief This function handles Hard fault interrupt.
  */
void HardFault_Handler(void)
{
 8001f9e:	b480      	push	{r7}
 8001fa0:	af00      	add	r7, sp, #0
  /* USER CODE BEGIN HardFault_IRQn 0 */

  /* USER CODE END HardFault_IRQn 0 */
  while (1)
 8001fa2:	e7fe      	b.n	8001fa2 <HardFault_Handler+0x4>

08001fa4 <MemManage_Handler>:

/**
  * @brief This function handles Memory management fault.
  */
void MemManage_Handler(void)
{
 8001fa4:	b480      	push	{r7}
 8001fa6:	af00      	add	r7, sp, #0
  /* USER CODE BEGIN MemoryManagement_IRQn 0 */

  /* USER CODE END MemoryManagement_IRQn 0 */
  while (1)
 8001fa8:	e7fe      	b.n	8001fa8 <MemManage_Handler+0x4>

08001faa <BusFault_Handler>:

/**
  * @brief This function handles Pre-fetch fault, memory access fault.
  */
void BusFault_Handler(void)
{
 8001faa:	b480      	push	{r7}
 8001fac:	af00      	add	r7, sp, #0
  /* USER CODE BEGIN BusFault_IRQn 0 */

  /* USER CODE END BusFault_IRQn 0 */
  while (1)
 8001fae:	e7fe      	b.n	8001fae <BusFault_Handler+0x4>

08001fb0 <UsageFault_Handler>:

/**
  * @brief This function handles Undefined instruction or illegal state.
  */
void UsageFault_Handler(void)
{
 8001fb0:	b480      	push	{r7}
 8001fb2:	af00      	add	r7, sp, #0
  /* USER CODE BEGIN UsageFault_IRQn 0 */

  /* USER CODE END UsageFault_IRQn 0 */
  while (1)
 8001fb4:	e7fe      	b.n	8001fb4 <UsageFault_Handler+0x4>

08001fb6 <SVC_Handler>:

/**
  * @brief This function handles System service call via SWI instruction.
  */
void SVC_Handler(void)
{
 8001fb6:	b480      	push	{r7}
 8001fb8:	af00      	add	r7, sp, #0

  /* USER CODE END SVCall_IRQn 0 */
  /* USER CODE BEGIN SVCall_IRQn 1 */

  /* USER CODE END SVCall_IRQn 1 */
}
 8001fba:	bf00      	nop
 8001fbc:	46bd      	mov	sp, r7
 8001fbe:	f85d 7b04 	ldr.w	r7, [sp], #4
 8001fc2:	4770      	bx	lr

08001fc4 <DebugMon_Handler>:

/**
  * @brief This function handles Debug monitor.
  */
void DebugMon_Handler(void)
{
 8001fc4:	b480      	push	{r7}
 8001fc6:	af00      	add	r7, sp, #0

  /* USER CODE END DebugMonitor_IRQn 0 */
  /* USER CODE BEGIN DebugMonitor_IRQn 1 */

  /* USER CODE END DebugMonitor_IRQn 1 */
}
 8001fc8:	bf00      	nop
 8001fca:	46bd      	mov	sp, r7
 8001fcc:	f85d 7b04 	ldr.w	r7, [sp], #4
 8001fd0:	4770      	bx	lr

08001fd2 <PendSV_Handler>:

/**
  * @brief This function handles Pendable request for system service.
  */
void PendSV_Handler(void)
{
 8001fd2:	b480      	push	{r7}
 8001fd4:	af00      	add	r7, sp, #0

  /* USER CODE END PendSV_IRQn 0 */
  /* USER CODE BEGIN PendSV_IRQn 1 */

  /* USER CODE END PendSV_IRQn 1 */
}
 8001fd6:	bf00      	nop
 8001fd8:	46bd      	mov	sp, r7
 8001fda:	f85d 7b04 	ldr.w	r7, [sp], #4
 8001fde:	4770      	bx	lr

08001fe0 <SysTick_Handler>:

/**
  * @brief This function handles System tick timer.
  */
void SysTick_Handler(void)
{
 8001fe0:	b580      	push	{r7, lr}
 8001fe2:	af00      	add	r7, sp, #0
  /* USER CODE BEGIN SysTick_IRQn 0 */

  /* USER CODE END SysTick_IRQn 0 */
  HAL_IncTick();
 8001fe4:	f000 f944 	bl	8002270 <HAL_IncTick>
  /* USER CODE BEGIN SysTick_IRQn 1 */

  /* USER CODE END SysTick_IRQn 1 */
}
 8001fe8:	bf00      	nop
 8001fea:	bd80      	pop	{r7, pc}

08001fec <DMA2_Stream1_IRQHandler>:

/**
  * @brief This function handles DMA2 stream1 global interrupt.
  */
void DMA2_Stream1_IRQHandler(void)
{
 8001fec:	b580      	push	{r7, lr}
 8001fee:	af00      	add	r7, sp, #0
  /* USER CODE BEGIN DMA2_Stream1_IRQn 0 */

  /* USER CODE END DMA2_Stream1_IRQn 0 */
  HAL_DMA_IRQHandler(&hdma_tim1_ch1);
 8001ff0:	4802      	ldr	r0, [pc, #8]	; (8001ffc <DMA2_Stream1_IRQHandler+0x10>)
 8001ff2:	f000 ff75 	bl	8002ee0 <HAL_DMA_IRQHandler>
  /* USER CODE BEGIN DMA2_Stream1_IRQn 1 */

  /* USER CODE END DMA2_Stream1_IRQn 1 */
}
 8001ff6:	bf00      	nop
 8001ff8:	bd80      	pop	{r7, pc}
 8001ffa:	bf00      	nop
 8001ffc:	200002e0 	.word	0x200002e0

08002000 <_getpid>:
void initialise_monitor_handles()
{
}

int _getpid(void)
{
 8002000:	b480      	push	{r7}
 8002002:	af00      	add	r7, sp, #0
	return 1;
 8002004:	2301      	movs	r3, #1
}
 8002006:	4618      	mov	r0, r3
 8002008:	46bd      	mov	sp, r7
 800200a:	f85d 7b04 	ldr.w	r7, [sp], #4
 800200e:	4770      	bx	lr

08002010 <_kill>:

int _kill(int pid, int sig)
{
 8002010:	b580      	push	{r7, lr}
 8002012:	b082      	sub	sp, #8
 8002014:	af00      	add	r7, sp, #0
 8002016:	6078      	str	r0, [r7, #4]
 8002018:	6039      	str	r1, [r7, #0]
	errno = EINVAL;
 800201a:	f004 f8bb 	bl	8006194 <__errno>
 800201e:	4603      	mov	r3, r0
 8002020:	2216      	movs	r2, #22
 8002022:	601a      	str	r2, [r3, #0]
	return -1;
 8002024:	f04f 33ff 	mov.w	r3, #4294967295
}
 8002028:	4618      	mov	r0, r3
 800202a:	3708      	adds	r7, #8
 800202c:	46bd      	mov	sp, r7
 800202e:	bd80      	pop	{r7, pc}

08002030 <_exit>:

void _exit (int status)
{
 8002030:	b580      	push	{r7, lr}
 8002032:	b082      	sub	sp, #8
 8002034:	af00      	add	r7, sp, #0
 8002036:	6078      	str	r0, [r7, #4]
	_kill(status, -1);
 8002038:	f04f 31ff 	mov.w	r1, #4294967295
 800203c:	6878      	ldr	r0, [r7, #4]
 800203e:	f7ff ffe7 	bl	8002010 <_kill>
	while (1) {}		/* Make sure we hang here */
 8002042:	e7fe      	b.n	8002042 <_exit+0x12>

08002044 <_read>:
}

__attribute__((weak)) int _read(int file, char *ptr, int len)
{
 8002044:	b580      	push	{r7, lr}
 8002046:	b086      	sub	sp, #24
 8002048:	af00      	add	r7, sp, #0
 800204a:	60f8      	str	r0, [r7, #12]
 800204c:	60b9      	str	r1, [r7, #8]
 800204e:	607a      	str	r2, [r7, #4]
	int DataIdx;

	for (DataIdx = 0; DataIdx < len; DataIdx++)
 8002050:	2300      	movs	r3, #0
 8002052:	617b      	str	r3, [r7, #20]
 8002054:	e00a      	b.n	800206c <_read+0x28>
	{
		*ptr++ = __io_getchar();
 8002056:	f3af 8000 	nop.w
 800205a:	4601      	mov	r1, r0
 800205c:	68bb      	ldr	r3, [r7, #8]
 800205e:	1c5a      	adds	r2, r3, #1
 8002060:	60ba      	str	r2, [r7, #8]
 8002062:	b2ca      	uxtb	r2, r1
 8002064:	701a      	strb	r2, [r3, #0]
	for (DataIdx = 0; DataIdx < len; DataIdx++)
 8002066:	697b      	ldr	r3, [r7, #20]
 8002068:	3301      	adds	r3, #1
 800206a:	617b      	str	r3, [r7, #20]
 800206c:	697a      	ldr	r2, [r7, #20]
 800206e:	687b      	ldr	r3, [r7, #4]
 8002070:	429a      	cmp	r2, r3
 8002072:	dbf0      	blt.n	8002056 <_read+0x12>
	}

return len;
 8002074:	687b      	ldr	r3, [r7, #4]
}
 8002076:	4618      	mov	r0, r3
 8002078:	3718      	adds	r7, #24
 800207a:	46bd      	mov	sp, r7
 800207c:	bd80      	pop	{r7, pc}

0800207e <_close>:
	}
	return len;
}

int _close(int file)
{
 800207e:	b480      	push	{r7}
 8002080:	b083      	sub	sp, #12
 8002082:	af00      	add	r7, sp, #0
 8002084:	6078      	str	r0, [r7, #4]
	return -1;
 8002086:	f04f 33ff 	mov.w	r3, #4294967295
}
 800208a:	4618      	mov	r0, r3
 800208c:	370c      	adds	r7, #12
 800208e:	46bd      	mov	sp, r7
 8002090:	f85d 7b04 	ldr.w	r7, [sp], #4
 8002094:	4770      	bx	lr

08002096 <_fstat>:


int _fstat(int file, struct stat *st)
{
 8002096:	b480      	push	{r7}
 8002098:	b083      	sub	sp, #12
 800209a:	af00      	add	r7, sp, #0
 800209c:	6078      	str	r0, [r7, #4]
 800209e:	6039      	str	r1, [r7, #0]
	st->st_mode = S_IFCHR;
 80020a0:	683b      	ldr	r3, [r7, #0]
 80020a2:	f44f 5200 	mov.w	r2, #8192	; 0x2000
 80020a6:	605a      	str	r2, [r3, #4]
	return 0;
 80020a8:	2300      	movs	r3, #0
}
 80020aa:	4618      	mov	r0, r3
 80020ac:	370c      	adds	r7, #12
 80020ae:	46bd      	mov	sp, r7
 80020b0:	f85d 7b04 	ldr.w	r7, [sp], #4
 80020b4:	4770      	bx	lr

080020b6 <_isatty>:

int _isatty(int file)
{
 80020b6:	b480      	push	{r7}
 80020b8:	b083      	sub	sp, #12
 80020ba:	af00      	add	r7, sp, #0
 80020bc:	6078      	str	r0, [r7, #4]
	return 1;
 80020be:	2301      	movs	r3, #1
}
 80020c0:	4618      	mov	r0, r3
 80020c2:	370c      	adds	r7, #12
 80020c4:	46bd      	mov	sp, r7
 80020c6:	f85d 7b04 	ldr.w	r7, [sp], #4
 80020ca:	4770      	bx	lr

080020cc <_lseek>:

int _lseek(int file, int ptr, int dir)
{
 80020cc:	b480      	push	{r7}
 80020ce:	b085      	sub	sp, #20
 80020d0:	af00      	add	r7, sp, #0
 80020d2:	60f8      	str	r0, [r7, #12]
 80020d4:	60b9      	str	r1, [r7, #8]
 80020d6:	607a      	str	r2, [r7, #4]
	return 0;
 80020d8:	2300      	movs	r3, #0
}
 80020da:	4618      	mov	r0, r3
 80020dc:	3714      	adds	r7, #20
 80020de:	46bd      	mov	sp, r7
 80020e0:	f85d 7b04 	ldr.w	r7, [sp], #4
 80020e4:	4770      	bx	lr
	...

080020e8 <_sbrk>:
 *
 * @param incr Memory size
 * @return Pointer to allocated memory
 */
void *_sbrk(ptrdiff_t incr)
{
 80020e8:	b580      	push	{r7, lr}
 80020ea:	b086      	sub	sp, #24
 80020ec:	af00      	add	r7, sp, #0
 80020ee:	6078      	str	r0, [r7, #4]
  extern uint8_t _end; /* Symbol defined in the linker script */
  extern uint8_t _estack; /* Symbol defined in the linker script */
  extern uint32_t _Min_Stack_Size; /* Symbol defined in the linker script */
  const uint32_t stack_limit = (uint32_t)&_estack - (uint32_t)&_Min_Stack_Size;
 80020f0:	4a14      	ldr	r2, [pc, #80]	; (8002144 <_sbrk+0x5c>)
 80020f2:	4b15      	ldr	r3, [pc, #84]	; (8002148 <_sbrk+0x60>)
 80020f4:	1ad3      	subs	r3, r2, r3
 80020f6:	617b      	str	r3, [r7, #20]
  const uint8_t *max_heap = (uint8_t *)stack_limit;
 80020f8:	697b      	ldr	r3, [r7, #20]
 80020fa:	613b      	str	r3, [r7, #16]
  uint8_t *prev_heap_end;

  /* Initialize heap end at first call */
  if (NULL == __sbrk_heap_end)
 80020fc:	4b13      	ldr	r3, [pc, #76]	; (800214c <_sbrk+0x64>)
 80020fe:	681b      	ldr	r3, [r3, #0]
 8002100:	2b00      	cmp	r3, #0
 8002102:	d102      	bne.n	800210a <_sbrk+0x22>
  {
    __sbrk_heap_end = &_end;
 8002104:	4b11      	ldr	r3, [pc, #68]	; (800214c <_sbrk+0x64>)
 8002106:	4a12      	ldr	r2, [pc, #72]	; (8002150 <_sbrk+0x68>)
 8002108:	601a      	str	r2, [r3, #0]
  }

  /* Protect heap from growing into the reserved MSP stack */
  if (__sbrk_heap_end + incr > max_heap)
 800210a:	4b10      	ldr	r3, [pc, #64]	; (800214c <_sbrk+0x64>)
 800210c:	681a      	ldr	r2, [r3, #0]
 800210e:	687b      	ldr	r3, [r7, #4]
 8002110:	4413      	add	r3, r2
 8002112:	693a      	ldr	r2, [r7, #16]
 8002114:	429a      	cmp	r2, r3
 8002116:	d207      	bcs.n	8002128 <_sbrk+0x40>
  {
    errno = ENOMEM;
 8002118:	f004 f83c 	bl	8006194 <__errno>
 800211c:	4603      	mov	r3, r0
 800211e:	220c      	movs	r2, #12
 8002120:	601a      	str	r2, [r3, #0]
    return (void *)-1;
 8002122:	f04f 33ff 	mov.w	r3, #4294967295
 8002126:	e009      	b.n	800213c <_sbrk+0x54>
  }

  prev_heap_end = __sbrk_heap_end;
 8002128:	4b08      	ldr	r3, [pc, #32]	; (800214c <_sbrk+0x64>)
 800212a:	681b      	ldr	r3, [r3, #0]
 800212c:	60fb      	str	r3, [r7, #12]
  __sbrk_heap_end += incr;
 800212e:	4b07      	ldr	r3, [pc, #28]	; (800214c <_sbrk+0x64>)
 8002130:	681a      	ldr	r2, [r3, #0]
 8002132:	687b      	ldr	r3, [r7, #4]
 8002134:	4413      	add	r3, r2
 8002136:	4a05      	ldr	r2, [pc, #20]	; (800214c <_sbrk+0x64>)
 8002138:	6013      	str	r3, [r2, #0]

  return (void *)prev_heap_end;
 800213a:	68fb      	ldr	r3, [r7, #12]
}
 800213c:	4618      	mov	r0, r3
 800213e:	3718      	adds	r7, #24
 8002140:	46bd      	mov	sp, r7
 8002142:	bd80      	pop	{r7, pc}
 8002144:	20030000 	.word	0x20030000
 8002148:	00000400 	.word	0x00000400
 800214c:	20000388 	.word	0x20000388
 8002150:	200003a0 	.word	0x200003a0

08002154 <SystemInit>:
  *         configuration.
  * @param  None
  * @retval None
  */
void SystemInit(void)
{
 8002154:	b480      	push	{r7}
 8002156:	af00      	add	r7, sp, #0
  /* FPU settings ------------------------------------------------------------*/
  #if (__FPU_PRESENT == 1) && (__FPU_USED == 1)
    SCB->CPACR |= ((3UL << 10*2)|(3UL << 11*2));  /* set CP10 and CP11 Full Access */
 8002158:	4b06      	ldr	r3, [pc, #24]	; (8002174 <SystemInit+0x20>)
 800215a:	f8d3 3088 	ldr.w	r3, [r3, #136]	; 0x88
 800215e:	4a05      	ldr	r2, [pc, #20]	; (8002174 <SystemInit+0x20>)
 8002160:	f443 0370 	orr.w	r3, r3, #15728640	; 0xf00000
 8002164:	f8c2 3088 	str.w	r3, [r2, #136]	; 0x88

  /* Configure the Vector Table location -------------------------------------*/
#if defined(USER_VECT_TAB_ADDRESS)
  SCB->VTOR = VECT_TAB_BASE_ADDRESS | VECT_TAB_OFFSET; /* Vector Table Relocation in Internal SRAM */
#endif /* USER_VECT_TAB_ADDRESS */
}
 8002168:	bf00      	nop
 800216a:	46bd      	mov	sp, r7
 800216c:	f85d 7b04 	ldr.w	r7, [sp], #4
 8002170:	4770      	bx	lr
 8002172:	bf00      	nop
 8002174:	e000ed00 	.word	0xe000ed00

08002178 <Reset_Handler>:

    .section  .text.Reset_Handler
  .weak  Reset_Handler
  .type  Reset_Handler, %function
Reset_Handler: 
  ldr   sp, =_estack       /* set stack pointer */
 8002178:	f8df d034 	ldr.w	sp, [pc, #52]	; 80021b0 <LoopFillZerobss+0x12>
 
/* Copy the data segment initializers from flash to SRAM */  
  ldr r0, =_sdata
 800217c:	480d      	ldr	r0, [pc, #52]	; (80021b4 <LoopFillZerobss+0x16>)
  ldr r1, =_edata
 800217e:	490e      	ldr	r1, [pc, #56]	; (80021b8 <LoopFillZerobss+0x1a>)
  ldr r2, =_sidata
 8002180:	4a0e      	ldr	r2, [pc, #56]	; (80021bc <LoopFillZerobss+0x1e>)
  movs r3, #0
 8002182:	2300      	movs	r3, #0
  b LoopCopyDataInit
 8002184:	e002      	b.n	800218c <LoopCopyDataInit>

08002186 <CopyDataInit>:

CopyDataInit:
  ldr r4, [r2, r3]
 8002186:	58d4      	ldr	r4, [r2, r3]
  str r4, [r0, r3]
 8002188:	50c4      	str	r4, [r0, r3]
  adds r3, r3, #4
 800218a:	3304      	adds	r3, #4

0800218c <LoopCopyDataInit>:

LoopCopyDataInit:
  adds r4, r0, r3
 800218c:	18c4      	adds	r4, r0, r3
  cmp r4, r1
 800218e:	428c      	cmp	r4, r1
  bcc CopyDataInit
 8002190:	d3f9      	bcc.n	8002186 <CopyDataInit>
  
/* Zero fill the bss segment. */
  ldr r2, =_sbss
 8002192:	4a0b      	ldr	r2, [pc, #44]	; (80021c0 <LoopFillZerobss+0x22>)
  ldr r4, =_ebss
 8002194:	4c0b      	ldr	r4, [pc, #44]	; (80021c4 <LoopFillZerobss+0x26>)
  movs r3, #0
 8002196:	2300      	movs	r3, #0
  b LoopFillZerobss
 8002198:	e001      	b.n	800219e <LoopFillZerobss>

0800219a <FillZerobss>:

FillZerobss:
  str  r3, [r2]
 800219a:	6013      	str	r3, [r2, #0]
  adds r2, r2, #4
 800219c:	3204      	adds	r2, #4

0800219e <LoopFillZerobss>:

LoopFillZerobss:
  cmp r2, r4
 800219e:	42a2      	cmp	r2, r4
  bcc FillZerobss
 80021a0:	d3fb      	bcc.n	800219a <FillZerobss>

/* Call the clock system initialization function.*/
  bl  SystemInit   
 80021a2:	f7ff ffd7 	bl	8002154 <SystemInit>
/* Call static constructors */
    bl __libc_init_array
 80021a6:	f003 fffb 	bl	80061a0 <__libc_init_array>
/* Call the application's entry point.*/
  bl  main
 80021aa:	f7ff f903 	bl	80013b4 <main>
  bx  lr    
 80021ae:	4770      	bx	lr
  ldr   sp, =_estack       /* set stack pointer */
 80021b0:	20030000 	.word	0x20030000
  ldr r0, =_sdata
 80021b4:	20000000 	.word	0x20000000
  ldr r1, =_edata
 80021b8:	200001dc 	.word	0x200001dc
  ldr r2, =_sidata
 80021bc:	08009274 	.word	0x08009274
  ldr r2, =_sbss
 80021c0:	200001dc 	.word	0x200001dc
  ldr r4, =_ebss
 80021c4:	200003a0 	.word	0x200003a0

080021c8 <ADC_IRQHandler>:
 * @retval None       
*/
    .section  .text.Default_Handler,"ax",%progbits
Default_Handler:
Infinite_Loop:
  b  Infinite_Loop
 80021c8:	e7fe      	b.n	80021c8 <ADC_IRQHandler>
	...

080021cc <HAL_Init>:
  *         need to ensure that the SysTick time base is always set to 1 millisecond
  *         to have correct HAL operation.
  * @retval HAL status
  */
HAL_StatusTypeDef HAL_Init(void)
{
 80021cc:	b580      	push	{r7, lr}
 80021ce:	af00      	add	r7, sp, #0
  /* Configure Flash prefetch, Instruction cache, Data cache */ 
#if (INSTRUCTION_CACHE_ENABLE != 0U)
  __HAL_FLASH_INSTRUCTION_CACHE_ENABLE();
 80021d0:	4b0e      	ldr	r3, [pc, #56]	; (800220c <HAL_Init+0x40>)
 80021d2:	681b      	ldr	r3, [r3, #0]
 80021d4:	4a0d      	ldr	r2, [pc, #52]	; (800220c <HAL_Init+0x40>)
 80021d6:	f443 7300 	orr.w	r3, r3, #512	; 0x200
 80021da:	6013      	str	r3, [r2, #0]
#endif /* INSTRUCTION_CACHE_ENABLE */

#if (DATA_CACHE_ENABLE != 0U)
  __HAL_FLASH_DATA_CACHE_ENABLE();
 80021dc:	4b0b      	ldr	r3, [pc, #44]	; (800220c <HAL_Init+0x40>)
 80021de:	681b      	ldr	r3, [r3, #0]
 80021e0:	4a0a      	ldr	r2, [pc, #40]	; (800220c <HAL_Init+0x40>)
 80021e2:	f443 6380 	orr.w	r3, r3, #1024	; 0x400
 80021e6:	6013      	str	r3, [r2, #0]
#endif /* DATA_CACHE_ENABLE */

#if (PREFETCH_ENABLE != 0U)
  __HAL_FLASH_PREFETCH_BUFFER_ENABLE();
 80021e8:	4b08      	ldr	r3, [pc, #32]	; (800220c <HAL_Init+0x40>)
 80021ea:	681b      	ldr	r3, [r3, #0]
 80021ec:	4a07      	ldr	r2, [pc, #28]	; (800220c <HAL_Init+0x40>)
 80021ee:	f443 7380 	orr.w	r3, r3, #256	; 0x100
 80021f2:	6013      	str	r3, [r2, #0]
#endif /* PREFETCH_ENABLE */

  /* Set Interrupt Group Priority */
  HAL_NVIC_SetPriorityGrouping(NVIC_PRIORITYGROUP_4);
 80021f4:	2003      	movs	r0, #3
 80021f6:	f000 fd2b 	bl	8002c50 <HAL_NVIC_SetPriorityGrouping>

  /* Use systick as time base source and configure 1ms tick (default clock after Reset is HSI) */
  HAL_InitTick(TICK_INT_PRIORITY);
 80021fa:	2000      	movs	r0, #0
 80021fc:	f000 f808 	bl	8002210 <HAL_InitTick>

  /* Init the low level hardware */
  HAL_MspInit();
 8002200:	f7ff fd3e 	bl	8001c80 <HAL_MspInit>

  /* Return function status */
  return HAL_OK;
 8002204:	2300      	movs	r3, #0
}
 8002206:	4618      	mov	r0, r3
 8002208:	bd80      	pop	{r7, pc}
 800220a:	bf00      	nop
 800220c:	40023c00 	.word	0x40023c00

08002210 <HAL_InitTick>:
  *       implementation  in user file.
  * @param TickPriority Tick interrupt priority.
  * @retval HAL status
  */
__weak HAL_StatusTypeDef HAL_InitTick(uint32_t TickPriority)
{
 8002210:	b580      	push	{r7, lr}
 8002212:	b082      	sub	sp, #8
 8002214:	af00      	add	r7, sp, #0
 8002216:	6078      	str	r0, [r7, #4]
  /* Configure the SysTick to have interrupt in 1ms time basis*/
  if (HAL_SYSTICK_Config(SystemCoreClock / (1000U / uwTickFreq)) > 0U)
 8002218:	4b12      	ldr	r3, [pc, #72]	; (8002264 <HAL_InitTick+0x54>)
 800221a:	681a      	ldr	r2, [r3, #0]
 800221c:	4b12      	ldr	r3, [pc, #72]	; (8002268 <HAL_InitTick+0x58>)
 800221e:	781b      	ldrb	r3, [r3, #0]
 8002220:	4619      	mov	r1, r3
 8002222:	f44f 737a 	mov.w	r3, #1000	; 0x3e8
 8002226:	fbb3 f3f1 	udiv	r3, r3, r1
 800222a:	fbb2 f3f3 	udiv	r3, r2, r3
 800222e:	4618      	mov	r0, r3
 8002230:	f000 fd43 	bl	8002cba <HAL_SYSTICK_Config>
 8002234:	4603      	mov	r3, r0
 8002236:	2b00      	cmp	r3, #0
 8002238:	d001      	beq.n	800223e <HAL_InitTick+0x2e>
  {
    return HAL_ERROR;
 800223a:	2301      	movs	r3, #1
 800223c:	e00e      	b.n	800225c <HAL_InitTick+0x4c>
  }

  /* Configure the SysTick IRQ priority */
  if (TickPriority < (1UL << __NVIC_PRIO_BITS))
 800223e:	687b      	ldr	r3, [r7, #4]
 8002240:	2b0f      	cmp	r3, #15
 8002242:	d80a      	bhi.n	800225a <HAL_InitTick+0x4a>
  {
    HAL_NVIC_SetPriority(SysTick_IRQn, TickPriority, 0U);
 8002244:	2200      	movs	r2, #0
 8002246:	6879      	ldr	r1, [r7, #4]
 8002248:	f04f 30ff 	mov.w	r0, #4294967295
 800224c:	f000 fd0b 	bl	8002c66 <HAL_NVIC_SetPriority>
    uwTickPrio = TickPriority;
 8002250:	4a06      	ldr	r2, [pc, #24]	; (800226c <HAL_InitTick+0x5c>)
 8002252:	687b      	ldr	r3, [r7, #4]
 8002254:	6013      	str	r3, [r2, #0]
  {
    return HAL_ERROR;
  }

  /* Return function status */
  return HAL_OK;
 8002256:	2300      	movs	r3, #0
 8002258:	e000      	b.n	800225c <HAL_InitTick+0x4c>
    return HAL_ERROR;
 800225a:	2301      	movs	r3, #1
}
 800225c:	4618      	mov	r0, r3
 800225e:	3708      	adds	r7, #8
 8002260:	46bd      	mov	sp, r7
 8002262:	bd80      	pop	{r7, pc}
 8002264:	20000000 	.word	0x20000000
 8002268:	20000008 	.word	0x20000008
 800226c:	20000004 	.word	0x20000004

08002270 <HAL_IncTick>:
 * @note This function is declared as __weak to be overwritten in case of other 
  *      implementations in user file.
  * @retval None
  */
__weak void HAL_IncTick(void)
{
 8002270:	b480      	push	{r7}
 8002272:	af00      	add	r7, sp, #0
  uwTick += uwTickFreq;
 8002274:	4b06      	ldr	r3, [pc, #24]	; (8002290 <HAL_IncTick+0x20>)
 8002276:	781b      	ldrb	r3, [r3, #0]
 8002278:	461a      	mov	r2, r3
 800227a:	4b06      	ldr	r3, [pc, #24]	; (8002294 <HAL_IncTick+0x24>)
 800227c:	681b      	ldr	r3, [r3, #0]
 800227e:	4413      	add	r3, r2
 8002280:	4a04      	ldr	r2, [pc, #16]	; (8002294 <HAL_IncTick+0x24>)
 8002282:	6013      	str	r3, [r2, #0]
}
 8002284:	bf00      	nop
 8002286:	46bd      	mov	sp, r7
 8002288:	f85d 7b04 	ldr.w	r7, [sp], #4
 800228c:	4770      	bx	lr
 800228e:	bf00      	nop
 8002290:	20000008 	.word	0x20000008
 8002294:	2000038c 	.word	0x2000038c

08002298 <HAL_GetTick>:
  * @note This function is declared as __weak to be overwritten in case of other 
  *       implementations in user file.
  * @retval tick value
  */
__weak uint32_t HAL_GetTick(void)
{
 8002298:	b480      	push	{r7}
 800229a:	af00      	add	r7, sp, #0
  return uwTick;
 800229c:	4b03      	ldr	r3, [pc, #12]	; (80022ac <HAL_GetTick+0x14>)
 800229e:	681b      	ldr	r3, [r3, #0]
}
 80022a0:	4618      	mov	r0, r3
 80022a2:	46bd      	mov	sp, r7
 80022a4:	f85d 7b04 	ldr.w	r7, [sp], #4
 80022a8:	4770      	bx	lr
 80022aa:	bf00      	nop
 80022ac:	2000038c 	.word	0x2000038c

080022b0 <HAL_Delay>:
  *       implementations in user file.
  * @param Delay specifies the delay time length, in milliseconds.
  * @retval None
  */
__weak void HAL_Delay(uint32_t Delay)
{
 80022b0:	b580      	push	{r7, lr}
 80022b2:	b084      	sub	sp, #16
 80022b4:	af00      	add	r7, sp, #0
 80022b6:	6078      	str	r0, [r7, #4]
  uint32_t tickstart = HAL_GetTick();
 80022b8:	f7ff ffee 	bl	8002298 <HAL_GetTick>
 80022bc:	60b8      	str	r0, [r7, #8]
  uint32_t wait = Delay;
 80022be:	687b      	ldr	r3, [r7, #4]
 80022c0:	60fb      	str	r3, [r7, #12]

  /* Add a freq to guarantee minimum wait */
  if (wait < HAL_MAX_DELAY)
 80022c2:	68fb      	ldr	r3, [r7, #12]
 80022c4:	f1b3 3fff 	cmp.w	r3, #4294967295
 80022c8:	d005      	beq.n	80022d6 <HAL_Delay+0x26>
  {
    wait += (uint32_t)(uwTickFreq);
 80022ca:	4b0a      	ldr	r3, [pc, #40]	; (80022f4 <HAL_Delay+0x44>)
 80022cc:	781b      	ldrb	r3, [r3, #0]
 80022ce:	461a      	mov	r2, r3
 80022d0:	68fb      	ldr	r3, [r7, #12]
 80022d2:	4413      	add	r3, r2
 80022d4:	60fb      	str	r3, [r7, #12]
  }

  while((HAL_GetTick() - tickstart) < wait)
 80022d6:	bf00      	nop
 80022d8:	f7ff ffde 	bl	8002298 <HAL_GetTick>
 80022dc:	4602      	mov	r2, r0
 80022de:	68bb      	ldr	r3, [r7, #8]
 80022e0:	1ad3      	subs	r3, r2, r3
 80022e2:	68fa      	ldr	r2, [r7, #12]
 80022e4:	429a      	cmp	r2, r3
 80022e6:	d8f7      	bhi.n	80022d8 <HAL_Delay+0x28>
  {
  }
}
 80022e8:	bf00      	nop
 80022ea:	bf00      	nop
 80022ec:	3710      	adds	r7, #16
 80022ee:	46bd      	mov	sp, r7
 80022f0:	bd80      	pop	{r7, pc}
 80022f2:	bf00      	nop
 80022f4:	20000008 	.word	0x20000008

080022f8 <HAL_ADC_Init>:
  * @param  hadc pointer to a ADC_HandleTypeDef structure that contains
  *         the configuration information for the specified ADC.  
  * @retval HAL status
  */
HAL_StatusTypeDef HAL_ADC_Init(ADC_HandleTypeDef* hadc)
{
 80022f8:	b580      	push	{r7, lr}
 80022fa:	b084      	sub	sp, #16
 80022fc:	af00      	add	r7, sp, #0
 80022fe:	6078      	str	r0, [r7, #4]
  HAL_StatusTypeDef tmp_hal_status = HAL_OK;
 8002300:	2300      	movs	r3, #0
 8002302:	73fb      	strb	r3, [r7, #15]
  
  /* Check ADC handle */
  if(hadc == NULL)
 8002304:	687b      	ldr	r3, [r7, #4]
 8002306:	2b00      	cmp	r3, #0
 8002308:	d101      	bne.n	800230e <HAL_ADC_Init+0x16>
  {
    return HAL_ERROR;
 800230a:	2301      	movs	r3, #1
 800230c:	e033      	b.n	8002376 <HAL_ADC_Init+0x7e>
  if(hadc->Init.ExternalTrigConv != ADC_SOFTWARE_START)
  {
    assert_param(IS_ADC_EXT_TRIG_EDGE(hadc->Init.ExternalTrigConvEdge));
  }
  
  if(hadc->State == HAL_ADC_STATE_RESET)
 800230e:	687b      	ldr	r3, [r7, #4]
 8002310:	6c1b      	ldr	r3, [r3, #64]	; 0x40
 8002312:	2b00      	cmp	r3, #0
 8002314:	d109      	bne.n	800232a <HAL_ADC_Init+0x32>

    /* Init the low level hardware */
    hadc->MspInitCallback(hadc);
#else
    /* Init the low level hardware */
    HAL_ADC_MspInit(hadc);
 8002316:	6878      	ldr	r0, [r7, #4]
 8002318:	f7ff fcda 	bl	8001cd0 <HAL_ADC_MspInit>
#endif /* USE_HAL_ADC_REGISTER_CALLBACKS */

    /* Initialize ADC error code */
    ADC_CLEAR_ERRORCODE(hadc);
 800231c:	687b      	ldr	r3, [r7, #4]
 800231e:	2200      	movs	r2, #0
 8002320:	645a      	str	r2, [r3, #68]	; 0x44
    
    /* Allocate lock resource and initialize it */
    hadc->Lock = HAL_UNLOCKED;
 8002322:	687b      	ldr	r3, [r7, #4]
 8002324:	2200      	movs	r2, #0
 8002326:	f883 203c 	strb.w	r2, [r3, #60]	; 0x3c
  }
  
  /* Configuration of ADC parameters if previous preliminary actions are      */ 
  /* correctly completed.                                                     */
  if (HAL_IS_BIT_CLR(hadc->State, HAL_ADC_STATE_ERROR_INTERNAL))
 800232a:	687b      	ldr	r3, [r7, #4]
 800232c:	6c1b      	ldr	r3, [r3, #64]	; 0x40
 800232e:	f003 0310 	and.w	r3, r3, #16
 8002332:	2b00      	cmp	r3, #0
 8002334:	d118      	bne.n	8002368 <HAL_ADC_Init+0x70>
  {
    /* Set ADC state */
    ADC_STATE_CLR_SET(hadc->State,
 8002336:	687b      	ldr	r3, [r7, #4]
 8002338:	6c1b      	ldr	r3, [r3, #64]	; 0x40
 800233a:	f423 5388 	bic.w	r3, r3, #4352	; 0x1100
 800233e:	f023 0302 	bic.w	r3, r3, #2
 8002342:	f043 0202 	orr.w	r2, r3, #2
 8002346:	687b      	ldr	r3, [r7, #4]
 8002348:	641a      	str	r2, [r3, #64]	; 0x40
                      HAL_ADC_STATE_REG_BUSY | HAL_ADC_STATE_INJ_BUSY,
                      HAL_ADC_STATE_BUSY_INTERNAL);
    
    /* Set ADC parameters */
    ADC_Init(hadc);
 800234a:	6878      	ldr	r0, [r7, #4]
 800234c:	f000 fab4 	bl	80028b8 <ADC_Init>
    
    /* Set ADC error code to none */
    ADC_CLEAR_ERRORCODE(hadc);
 8002350:	687b      	ldr	r3, [r7, #4]
 8002352:	2200      	movs	r2, #0
 8002354:	645a      	str	r2, [r3, #68]	; 0x44
    
    /* Set the ADC state */
    ADC_STATE_CLR_SET(hadc->State,
 8002356:	687b      	ldr	r3, [r7, #4]
 8002358:	6c1b      	ldr	r3, [r3, #64]	; 0x40
 800235a:	f023 0303 	bic.w	r3, r3, #3
 800235e:	f043 0201 	orr.w	r2, r3, #1
 8002362:	687b      	ldr	r3, [r7, #4]
 8002364:	641a      	str	r2, [r3, #64]	; 0x40
 8002366:	e001      	b.n	800236c <HAL_ADC_Init+0x74>
                      HAL_ADC_STATE_BUSY_INTERNAL,
                      HAL_ADC_STATE_READY);
  }
  else
  {
    tmp_hal_status = HAL_ERROR;
 8002368:	2301      	movs	r3, #1
 800236a:	73fb      	strb	r3, [r7, #15]
  }
  
  /* Release Lock */
  __HAL_UNLOCK(hadc);
 800236c:	687b      	ldr	r3, [r7, #4]
 800236e:	2200      	movs	r2, #0
 8002370:	f883 203c 	strb.w	r2, [r3, #60]	; 0x3c

  /* Return function status */
  return tmp_hal_status;
 8002374:	7bfb      	ldrb	r3, [r7, #15]
}
 8002376:	4618      	mov	r0, r3
 8002378:	3710      	adds	r7, #16
 800237a:	46bd      	mov	sp, r7
 800237c:	bd80      	pop	{r7, pc}
	...

08002380 <HAL_ADC_Start>:
  * @param  hadc pointer to a ADC_HandleTypeDef structure that contains
  *         the configuration information for the specified ADC.
  * @retval HAL status
  */
HAL_StatusTypeDef HAL_ADC_Start(ADC_HandleTypeDef* hadc)
{
 8002380:	b480      	push	{r7}
 8002382:	b085      	sub	sp, #20
 8002384:	af00      	add	r7, sp, #0
 8002386:	6078      	str	r0, [r7, #4]
  __IO uint32_t counter = 0U;
 8002388:	2300      	movs	r3, #0
 800238a:	60bb      	str	r3, [r7, #8]
  /* Check the parameters */
  assert_param(IS_FUNCTIONAL_STATE(hadc->Init.ContinuousConvMode));
  assert_param(IS_ADC_EXT_TRIG_EDGE(hadc->Init.ExternalTrigConvEdge)); 
  
  /* Process locked */
  __HAL_LOCK(hadc);
 800238c:	687b      	ldr	r3, [r7, #4]
 800238e:	f893 303c 	ldrb.w	r3, [r3, #60]	; 0x3c
 8002392:	2b01      	cmp	r3, #1
 8002394:	d101      	bne.n	800239a <HAL_ADC_Start+0x1a>
 8002396:	2302      	movs	r3, #2
 8002398:	e0b2      	b.n	8002500 <HAL_ADC_Start+0x180>
 800239a:	687b      	ldr	r3, [r7, #4]
 800239c:	2201      	movs	r2, #1
 800239e:	f883 203c 	strb.w	r2, [r3, #60]	; 0x3c
  
  /* Enable the ADC peripheral */
  /* Check if ADC peripheral is disabled in order to enable it and wait during 
  Tstab time the ADC's stabilization */
  if((hadc->Instance->CR2 & ADC_CR2_ADON) != ADC_CR2_ADON)
 80023a2:	687b      	ldr	r3, [r7, #4]
 80023a4:	681b      	ldr	r3, [r3, #0]
 80023a6:	689b      	ldr	r3, [r3, #8]
 80023a8:	f003 0301 	and.w	r3, r3, #1
 80023ac:	2b01      	cmp	r3, #1
 80023ae:	d018      	beq.n	80023e2 <HAL_ADC_Start+0x62>
  {  
    /* Enable the Peripheral */
    __HAL_ADC_ENABLE(hadc);
 80023b0:	687b      	ldr	r3, [r7, #4]
 80023b2:	681b      	ldr	r3, [r3, #0]
 80023b4:	689a      	ldr	r2, [r3, #8]
 80023b6:	687b      	ldr	r3, [r7, #4]
 80023b8:	681b      	ldr	r3, [r3, #0]
 80023ba:	f042 0201 	orr.w	r2, r2, #1
 80023be:	609a      	str	r2, [r3, #8]
    
    /* Delay for ADC stabilization time */
    /* Compute number of CPU cycles to wait for */
    counter = (ADC_STAB_DELAY_US * (SystemCoreClock / 1000000U));
 80023c0:	4b52      	ldr	r3, [pc, #328]	; (800250c <HAL_ADC_Start+0x18c>)
 80023c2:	681b      	ldr	r3, [r3, #0]
 80023c4:	4a52      	ldr	r2, [pc, #328]	; (8002510 <HAL_ADC_Start+0x190>)
 80023c6:	fba2 2303 	umull	r2, r3, r2, r3
 80023ca:	0c9a      	lsrs	r2, r3, #18
 80023cc:	4613      	mov	r3, r2
 80023ce:	005b      	lsls	r3, r3, #1
 80023d0:	4413      	add	r3, r2
 80023d2:	60bb      	str	r3, [r7, #8]
    while(counter != 0U)
 80023d4:	e002      	b.n	80023dc <HAL_ADC_Start+0x5c>
    {
      counter--;
 80023d6:	68bb      	ldr	r3, [r7, #8]
 80023d8:	3b01      	subs	r3, #1
 80023da:	60bb      	str	r3, [r7, #8]
    while(counter != 0U)
 80023dc:	68bb      	ldr	r3, [r7, #8]
 80023de:	2b00      	cmp	r3, #0
 80023e0:	d1f9      	bne.n	80023d6 <HAL_ADC_Start+0x56>
    }
  }
  
  /* Start conversion if ADC is effectively enabled */
  if(HAL_IS_BIT_SET(hadc->Instance->CR2, ADC_CR2_ADON))
 80023e2:	687b      	ldr	r3, [r7, #4]
 80023e4:	681b      	ldr	r3, [r3, #0]
 80023e6:	689b      	ldr	r3, [r3, #8]
 80023e8:	f003 0301 	and.w	r3, r3, #1
 80023ec:	2b01      	cmp	r3, #1
 80023ee:	d17a      	bne.n	80024e6 <HAL_ADC_Start+0x166>
  {
    /* Set ADC state                                                          */
    /* - Clear state bitfield related to regular group conversion results     */
    /* - Set state bitfield related to regular group operation                */
    ADC_STATE_CLR_SET(hadc->State,
 80023f0:	687b      	ldr	r3, [r7, #4]
 80023f2:	6c1b      	ldr	r3, [r3, #64]	; 0x40
 80023f4:	f423 63e0 	bic.w	r3, r3, #1792	; 0x700
 80023f8:	f023 0301 	bic.w	r3, r3, #1
 80023fc:	f443 7280 	orr.w	r2, r3, #256	; 0x100
 8002400:	687b      	ldr	r3, [r7, #4]
 8002402:	641a      	str	r2, [r3, #64]	; 0x40
                      HAL_ADC_STATE_READY | HAL_ADC_STATE_REG_EOC | HAL_ADC_STATE_REG_OVR,
                      HAL_ADC_STATE_REG_BUSY);
    
    /* If conversions on group regular are also triggering group injected,    */
    /* update ADC state.                                                      */
    if (READ_BIT(hadc->Instance->CR1, ADC_CR1_JAUTO) != RESET)
 8002404:	687b      	ldr	r3, [r7, #4]
 8002406:	681b      	ldr	r3, [r3, #0]
 8002408:	685b      	ldr	r3, [r3, #4]
 800240a:	f403 6380 	and.w	r3, r3, #1024	; 0x400
 800240e:	2b00      	cmp	r3, #0
 8002410:	d007      	beq.n	8002422 <HAL_ADC_Start+0xa2>
    {
      ADC_STATE_CLR_SET(hadc->State, HAL_ADC_STATE_INJ_EOC, HAL_ADC_STATE_INJ_BUSY);  
 8002412:	687b      	ldr	r3, [r7, #4]
 8002414:	6c1b      	ldr	r3, [r3, #64]	; 0x40
 8002416:	f423 5340 	bic.w	r3, r3, #12288	; 0x3000
 800241a:	f443 5280 	orr.w	r2, r3, #4096	; 0x1000
 800241e:	687b      	ldr	r3, [r7, #4]
 8002420:	641a      	str	r2, [r3, #64]	; 0x40
    }
    
    /* State machine update: Check if an injected conversion is ongoing */
    if (HAL_IS_BIT_SET(hadc->State, HAL_ADC_STATE_INJ_BUSY))
 8002422:	687b      	ldr	r3, [r7, #4]
 8002424:	6c1b      	ldr	r3, [r3, #64]	; 0x40
 8002426:	f403 5380 	and.w	r3, r3, #4096	; 0x1000
 800242a:	f5b3 5f80 	cmp.w	r3, #4096	; 0x1000
 800242e:	d106      	bne.n	800243e <HAL_ADC_Start+0xbe>
    {
      /* Reset ADC error code fields related to conversions on group regular */
      CLEAR_BIT(hadc->ErrorCode, (HAL_ADC_ERROR_OVR | HAL_ADC_ERROR_DMA));         
 8002430:	687b      	ldr	r3, [r7, #4]
 8002432:	6c5b      	ldr	r3, [r3, #68]	; 0x44
 8002434:	f023 0206 	bic.w	r2, r3, #6
 8002438:	687b      	ldr	r3, [r7, #4]
 800243a:	645a      	str	r2, [r3, #68]	; 0x44
 800243c:	e002      	b.n	8002444 <HAL_ADC_Start+0xc4>
    }
    else
    {
      /* Reset ADC all error code fields */
      ADC_CLEAR_ERRORCODE(hadc);
 800243e:	687b      	ldr	r3, [r7, #4]
 8002440:	2200      	movs	r2, #0
 8002442:	645a      	str	r2, [r3, #68]	; 0x44
    } 

    /* Process unlocked */
    /* Unlock before starting ADC conversions: in case of potential           */
    /* interruption, to let the process to ADC IRQ Handler.                   */
    __HAL_UNLOCK(hadc);
 8002444:	687b      	ldr	r3, [r7, #4]
 8002446:	2200      	movs	r2, #0
 8002448:	f883 203c 	strb.w	r2, [r3, #60]	; 0x3c

    /* Pointer to the common control register to which is belonging hadc    */
    /* (Depending on STM32F4 product, there may be up to 3 ADCs and 1 common */
    /* control register)                                                    */
    tmpADC_Common = ADC_COMMON_REGISTER(hadc);
 800244c:	4b31      	ldr	r3, [pc, #196]	; (8002514 <HAL_ADC_Start+0x194>)
 800244e:	60fb      	str	r3, [r7, #12]

    /* Clear regular group conversion flag and overrun flag */
    /* (To ensure of no unknown state from potential previous ADC operations) */
    __HAL_ADC_CLEAR_FLAG(hadc, ADC_FLAG_EOC | ADC_FLAG_OVR);
 8002450:	687b      	ldr	r3, [r7, #4]
 8002452:	681b      	ldr	r3, [r3, #0]
 8002454:	f06f 0222 	mvn.w	r2, #34	; 0x22
 8002458:	601a      	str	r2, [r3, #0]
    
    /* Check if Multimode enabled */
    if(HAL_IS_BIT_CLR(tmpADC_Common->CCR, ADC_CCR_MULTI))
 800245a:	68fb      	ldr	r3, [r7, #12]
 800245c:	685b      	ldr	r3, [r3, #4]
 800245e:	f003 031f 	and.w	r3, r3, #31
 8002462:	2b00      	cmp	r3, #0
 8002464:	d12a      	bne.n	80024bc <HAL_ADC_Start+0x13c>
    {
#if defined(ADC2) && defined(ADC3)
      if((hadc->Instance == ADC1) || ((hadc->Instance == ADC2) && ((ADC->CCR & ADC_CCR_MULTI_Msk) < ADC_CCR_MULTI_0)) \
 8002466:	687b      	ldr	r3, [r7, #4]
 8002468:	681b      	ldr	r3, [r3, #0]
 800246a:	4a2b      	ldr	r2, [pc, #172]	; (8002518 <HAL_ADC_Start+0x198>)
 800246c:	4293      	cmp	r3, r2
 800246e:	d015      	beq.n	800249c <HAL_ADC_Start+0x11c>
 8002470:	687b      	ldr	r3, [r7, #4]
 8002472:	681b      	ldr	r3, [r3, #0]
 8002474:	4a29      	ldr	r2, [pc, #164]	; (800251c <HAL_ADC_Start+0x19c>)
 8002476:	4293      	cmp	r3, r2
 8002478:	d105      	bne.n	8002486 <HAL_ADC_Start+0x106>
 800247a:	4b26      	ldr	r3, [pc, #152]	; (8002514 <HAL_ADC_Start+0x194>)
 800247c:	685b      	ldr	r3, [r3, #4]
 800247e:	f003 031f 	and.w	r3, r3, #31
 8002482:	2b00      	cmp	r3, #0
 8002484:	d00a      	beq.n	800249c <HAL_ADC_Start+0x11c>
                                  || ((hadc->Instance == ADC3) && ((ADC->CCR & ADC_CCR_MULTI_Msk) < ADC_CCR_MULTI_4)))
 8002486:	687b      	ldr	r3, [r7, #4]
 8002488:	681b      	ldr	r3, [r3, #0]
 800248a:	4a25      	ldr	r2, [pc, #148]	; (8002520 <HAL_ADC_Start+0x1a0>)
 800248c:	4293      	cmp	r3, r2
 800248e:	d136      	bne.n	80024fe <HAL_ADC_Start+0x17e>
 8002490:	4b20      	ldr	r3, [pc, #128]	; (8002514 <HAL_ADC_Start+0x194>)
 8002492:	685b      	ldr	r3, [r3, #4]
 8002494:	f003 0310 	and.w	r3, r3, #16
 8002498:	2b00      	cmp	r3, #0
 800249a:	d130      	bne.n	80024fe <HAL_ADC_Start+0x17e>
      {
#endif /* ADC2 || ADC3 */
        /* if no external trigger present enable software conversion of regular channels */
        if((hadc->Instance->CR2 & ADC_CR2_EXTEN) == RESET) 
 800249c:	687b      	ldr	r3, [r7, #4]
 800249e:	681b      	ldr	r3, [r3, #0]
 80024a0:	689b      	ldr	r3, [r3, #8]
 80024a2:	f003 5340 	and.w	r3, r3, #805306368	; 0x30000000
 80024a6:	2b00      	cmp	r3, #0
 80024a8:	d129      	bne.n	80024fe <HAL_ADC_Start+0x17e>
        {
          /* Enable the selected ADC software conversion for regular group */
          hadc->Instance->CR2 |= (uint32_t)ADC_CR2_SWSTART;
 80024aa:	687b      	ldr	r3, [r7, #4]
 80024ac:	681b      	ldr	r3, [r3, #0]
 80024ae:	689a      	ldr	r2, [r3, #8]
 80024b0:	687b      	ldr	r3, [r7, #4]
 80024b2:	681b      	ldr	r3, [r3, #0]
 80024b4:	f042 4280 	orr.w	r2, r2, #1073741824	; 0x40000000
 80024b8:	609a      	str	r2, [r3, #8]
 80024ba:	e020      	b.n	80024fe <HAL_ADC_Start+0x17e>
#endif /* ADC2 || ADC3 */
    }
    else
    {
      /* if instance of handle correspond to ADC1 and  no external trigger present enable software conversion of regular channels */
      if((hadc->Instance == ADC1) && ((hadc->Instance->CR2 & ADC_CR2_EXTEN) == RESET))
 80024bc:	687b      	ldr	r3, [r7, #4]
 80024be:	681b      	ldr	r3, [r3, #0]
 80024c0:	4a15      	ldr	r2, [pc, #84]	; (8002518 <HAL_ADC_Start+0x198>)
 80024c2:	4293      	cmp	r3, r2
 80024c4:	d11b      	bne.n	80024fe <HAL_ADC_Start+0x17e>
 80024c6:	687b      	ldr	r3, [r7, #4]
 80024c8:	681b      	ldr	r3, [r3, #0]
 80024ca:	689b      	ldr	r3, [r3, #8]
 80024cc:	f003 5340 	and.w	r3, r3, #805306368	; 0x30000000
 80024d0:	2b00      	cmp	r3, #0
 80024d2:	d114      	bne.n	80024fe <HAL_ADC_Start+0x17e>
      {
        /* Enable the selected ADC software conversion for regular group */
          hadc->Instance->CR2 |= (uint32_t)ADC_CR2_SWSTART;
 80024d4:	687b      	ldr	r3, [r7, #4]
 80024d6:	681b      	ldr	r3, [r3, #0]
 80024d8:	689a      	ldr	r2, [r3, #8]
 80024da:	687b      	ldr	r3, [r7, #4]
 80024dc:	681b      	ldr	r3, [r3, #0]
 80024de:	f042 4280 	orr.w	r2, r2, #1073741824	; 0x40000000
 80024e2:	609a      	str	r2, [r3, #8]
 80024e4:	e00b      	b.n	80024fe <HAL_ADC_Start+0x17e>
    }
  }
  else
  {
    /* Update ADC state machine to error */
    SET_BIT(hadc->State, HAL_ADC_STATE_ERROR_INTERNAL);
 80024e6:	687b      	ldr	r3, [r7, #4]
 80024e8:	6c1b      	ldr	r3, [r3, #64]	; 0x40
 80024ea:	f043 0210 	orr.w	r2, r3, #16
 80024ee:	687b      	ldr	r3, [r7, #4]
 80024f0:	641a      	str	r2, [r3, #64]	; 0x40

    /* Set ADC error code to ADC IP internal error */
    SET_BIT(hadc->ErrorCode, HAL_ADC_ERROR_INTERNAL);
 80024f2:	687b      	ldr	r3, [r7, #4]
 80024f4:	6c5b      	ldr	r3, [r3, #68]	; 0x44
 80024f6:	f043 0201 	orr.w	r2, r3, #1
 80024fa:	687b      	ldr	r3, [r7, #4]
 80024fc:	645a      	str	r2, [r3, #68]	; 0x44
  }
  
  /* Return function status */
  return HAL_OK;
 80024fe:	2300      	movs	r3, #0
}
 8002500:	4618      	mov	r0, r3
 8002502:	3714      	adds	r7, #20
 8002504:	46bd      	mov	sp, r7
 8002506:	f85d 7b04 	ldr.w	r7, [sp], #4
 800250a:	4770      	bx	lr
 800250c:	20000000 	.word	0x20000000
 8002510:	431bde83 	.word	0x431bde83
 8002514:	40012300 	.word	0x40012300
 8002518:	40012000 	.word	0x40012000
 800251c:	40012100 	.word	0x40012100
 8002520:	40012200 	.word	0x40012200

08002524 <HAL_ADC_PollForConversion>:
  *         the configuration information for the specified ADC.
  * @param  Timeout Timeout value in millisecond.  
  * @retval HAL status
  */
HAL_StatusTypeDef HAL_ADC_PollForConversion(ADC_HandleTypeDef* hadc, uint32_t Timeout)
{
 8002524:	b580      	push	{r7, lr}
 8002526:	b084      	sub	sp, #16
 8002528:	af00      	add	r7, sp, #0
 800252a:	6078      	str	r0, [r7, #4]
 800252c:	6039      	str	r1, [r7, #0]
  uint32_t tickstart = 0U;
 800252e:	2300      	movs	r3, #0
 8002530:	60fb      	str	r3, [r7, #12]
  /* each conversion:                                                       */
  /* Particular case is ADC configured in DMA mode and ADC sequencer with   */
  /* several ranks and polling for end of each conversion.                  */
  /* For code simplicity sake, this particular case is generalized to       */
  /* ADC configured in DMA mode and polling for end of each conversion.     */
  if (HAL_IS_BIT_SET(hadc->Instance->CR2, ADC_CR2_EOCS) &&
 8002532:	687b      	ldr	r3, [r7, #4]
 8002534:	681b      	ldr	r3, [r3, #0]
 8002536:	689b      	ldr	r3, [r3, #8]
 8002538:	f403 6380 	and.w	r3, r3, #1024	; 0x400
 800253c:	f5b3 6f80 	cmp.w	r3, #1024	; 0x400
 8002540:	d113      	bne.n	800256a <HAL_ADC_PollForConversion+0x46>
      HAL_IS_BIT_SET(hadc->Instance->CR2, ADC_CR2_DMA)    )
 8002542:	687b      	ldr	r3, [r7, #4]
 8002544:	681b      	ldr	r3, [r3, #0]
 8002546:	689b      	ldr	r3, [r3, #8]
 8002548:	f403 7380 	and.w	r3, r3, #256	; 0x100
  if (HAL_IS_BIT_SET(hadc->Instance->CR2, ADC_CR2_EOCS) &&
 800254c:	f5b3 7f80 	cmp.w	r3, #256	; 0x100
 8002550:	d10b      	bne.n	800256a <HAL_ADC_PollForConversion+0x46>
  {
    /* Update ADC state machine to error */
    SET_BIT(hadc->State, HAL_ADC_STATE_ERROR_CONFIG);
 8002552:	687b      	ldr	r3, [r7, #4]
 8002554:	6c1b      	ldr	r3, [r3, #64]	; 0x40
 8002556:	f043 0220 	orr.w	r2, r3, #32
 800255a:	687b      	ldr	r3, [r7, #4]
 800255c:	641a      	str	r2, [r3, #64]	; 0x40
    
    /* Process unlocked */
    __HAL_UNLOCK(hadc);
 800255e:	687b      	ldr	r3, [r7, #4]
 8002560:	2200      	movs	r2, #0
 8002562:	f883 203c 	strb.w	r2, [r3, #60]	; 0x3c
    
    return HAL_ERROR;
 8002566:	2301      	movs	r3, #1
 8002568:	e063      	b.n	8002632 <HAL_ADC_PollForConversion+0x10e>
  }

  /* Get tick */ 
  tickstart = HAL_GetTick();
 800256a:	f7ff fe95 	bl	8002298 <HAL_GetTick>
 800256e:	60f8      	str	r0, [r7, #12]

  /* Check End of conversion flag */
  while(!(__HAL_ADC_GET_FLAG(hadc, ADC_FLAG_EOC)))
 8002570:	e021      	b.n	80025b6 <HAL_ADC_PollForConversion+0x92>
  {
    /* Check if timeout is disabled (set to infinite wait) */
    if(Timeout != HAL_MAX_DELAY)
 8002572:	683b      	ldr	r3, [r7, #0]
 8002574:	f1b3 3fff 	cmp.w	r3, #4294967295
 8002578:	d01d      	beq.n	80025b6 <HAL_ADC_PollForConversion+0x92>
    {
      if((Timeout == 0U) || ((HAL_GetTick() - tickstart ) > Timeout))
 800257a:	683b      	ldr	r3, [r7, #0]
 800257c:	2b00      	cmp	r3, #0
 800257e:	d007      	beq.n	8002590 <HAL_ADC_PollForConversion+0x6c>
 8002580:	f7ff fe8a 	bl	8002298 <HAL_GetTick>
 8002584:	4602      	mov	r2, r0
 8002586:	68fb      	ldr	r3, [r7, #12]
 8002588:	1ad3      	subs	r3, r2, r3
 800258a:	683a      	ldr	r2, [r7, #0]
 800258c:	429a      	cmp	r2, r3
 800258e:	d212      	bcs.n	80025b6 <HAL_ADC_PollForConversion+0x92>
      {
        /* New check to avoid false timeout detection in case of preemption */
        if(!(__HAL_ADC_GET_FLAG(hadc, ADC_FLAG_EOC)))
 8002590:	687b      	ldr	r3, [r7, #4]
 8002592:	681b      	ldr	r3, [r3, #0]
 8002594:	681b      	ldr	r3, [r3, #0]
 8002596:	f003 0302 	and.w	r3, r3, #2
 800259a:	2b02      	cmp	r3, #2
 800259c:	d00b      	beq.n	80025b6 <HAL_ADC_PollForConversion+0x92>
        {
          /* Update ADC state machine to timeout */
          SET_BIT(hadc->State, HAL_ADC_STATE_TIMEOUT);
 800259e:	687b      	ldr	r3, [r7, #4]
 80025a0:	6c1b      	ldr	r3, [r3, #64]	; 0x40
 80025a2:	f043 0204 	orr.w	r2, r3, #4
 80025a6:	687b      	ldr	r3, [r7, #4]
 80025a8:	641a      	str	r2, [r3, #64]	; 0x40
          
          /* Process unlocked */
          __HAL_UNLOCK(hadc);
 80025aa:	687b      	ldr	r3, [r7, #4]
 80025ac:	2200      	movs	r2, #0
 80025ae:	f883 203c 	strb.w	r2, [r3, #60]	; 0x3c
          
          return HAL_TIMEOUT;
 80025b2:	2303      	movs	r3, #3
 80025b4:	e03d      	b.n	8002632 <HAL_ADC_PollForConversion+0x10e>
  while(!(__HAL_ADC_GET_FLAG(hadc, ADC_FLAG_EOC)))
 80025b6:	687b      	ldr	r3, [r7, #4]
 80025b8:	681b      	ldr	r3, [r3, #0]
 80025ba:	681b      	ldr	r3, [r3, #0]
 80025bc:	f003 0302 	and.w	r3, r3, #2
 80025c0:	2b02      	cmp	r3, #2
 80025c2:	d1d6      	bne.n	8002572 <HAL_ADC_PollForConversion+0x4e>
      }
    }
  }
  
  /* Clear regular group conversion flag */
  __HAL_ADC_CLEAR_FLAG(hadc, ADC_FLAG_STRT | ADC_FLAG_EOC);
 80025c4:	687b      	ldr	r3, [r7, #4]
 80025c6:	681b      	ldr	r3, [r3, #0]
 80025c8:	f06f 0212 	mvn.w	r2, #18
 80025cc:	601a      	str	r2, [r3, #0]
  
  /* Update ADC state machine */
  SET_BIT(hadc->State, HAL_ADC_STATE_REG_EOC);
 80025ce:	687b      	ldr	r3, [r7, #4]
 80025d0:	6c1b      	ldr	r3, [r3, #64]	; 0x40
 80025d2:	f443 7200 	orr.w	r2, r3, #512	; 0x200
 80025d6:	687b      	ldr	r3, [r7, #4]
 80025d8:	641a      	str	r2, [r3, #64]	; 0x40
  /* by external trigger, continuous mode or scan sequence on going.          */
  /* Note: On STM32F4, there is no independent flag of end of sequence.       */
  /*       The test of scan sequence on going is done either with scan        */
  /*       sequence disabled or with end of conversion flag set to            */
  /*       of end of sequence.                                                */
  if(ADC_IS_SOFTWARE_START_REGULAR(hadc)                   &&
 80025da:	687b      	ldr	r3, [r7, #4]
 80025dc:	681b      	ldr	r3, [r3, #0]
 80025de:	689b      	ldr	r3, [r3, #8]
 80025e0:	f003 5340 	and.w	r3, r3, #805306368	; 0x30000000
 80025e4:	2b00      	cmp	r3, #0
 80025e6:	d123      	bne.n	8002630 <HAL_ADC_PollForConversion+0x10c>
     (hadc->Init.ContinuousConvMode == DISABLE)            &&
 80025e8:	687b      	ldr	r3, [r7, #4]
 80025ea:	7e1b      	ldrb	r3, [r3, #24]
  if(ADC_IS_SOFTWARE_START_REGULAR(hadc)                   &&
 80025ec:	2b00      	cmp	r3, #0
 80025ee:	d11f      	bne.n	8002630 <HAL_ADC_PollForConversion+0x10c>
     (HAL_IS_BIT_CLR(hadc->Instance->SQR1, ADC_SQR1_L) ||
 80025f0:	687b      	ldr	r3, [r7, #4]
 80025f2:	681b      	ldr	r3, [r3, #0]
 80025f4:	6adb      	ldr	r3, [r3, #44]	; 0x2c
 80025f6:	f403 0370 	and.w	r3, r3, #15728640	; 0xf00000
     (hadc->Init.ContinuousConvMode == DISABLE)            &&
 80025fa:	2b00      	cmp	r3, #0
 80025fc:	d006      	beq.n	800260c <HAL_ADC_PollForConversion+0xe8>
      HAL_IS_BIT_CLR(hadc->Instance->CR2, ADC_CR2_EOCS)  )   )
 80025fe:	687b      	ldr	r3, [r7, #4]
 8002600:	681b      	ldr	r3, [r3, #0]
 8002602:	689b      	ldr	r3, [r3, #8]
 8002604:	f403 6380 	and.w	r3, r3, #1024	; 0x400
     (HAL_IS_BIT_CLR(hadc->Instance->SQR1, ADC_SQR1_L) ||
 8002608:	2b00      	cmp	r3, #0
 800260a:	d111      	bne.n	8002630 <HAL_ADC_PollForConversion+0x10c>
  {
    /* Set ADC state */
    CLEAR_BIT(hadc->State, HAL_ADC_STATE_REG_BUSY);   
 800260c:	687b      	ldr	r3, [r7, #4]
 800260e:	6c1b      	ldr	r3, [r3, #64]	; 0x40
 8002610:	f423 7280 	bic.w	r2, r3, #256	; 0x100
 8002614:	687b      	ldr	r3, [r7, #4]
 8002616:	641a      	str	r2, [r3, #64]	; 0x40
    
    if (HAL_IS_BIT_CLR(hadc->State, HAL_ADC_STATE_INJ_BUSY))
 8002618:	687b      	ldr	r3, [r7, #4]
 800261a:	6c1b      	ldr	r3, [r3, #64]	; 0x40
 800261c:	f403 5380 	and.w	r3, r3, #4096	; 0x1000
 8002620:	2b00      	cmp	r3, #0
 8002622:	d105      	bne.n	8002630 <HAL_ADC_PollForConversion+0x10c>
    { 
      SET_BIT(hadc->State, HAL_ADC_STATE_READY);
 8002624:	687b      	ldr	r3, [r7, #4]
 8002626:	6c1b      	ldr	r3, [r3, #64]	; 0x40
 8002628:	f043 0201 	orr.w	r2, r3, #1
 800262c:	687b      	ldr	r3, [r7, #4]
 800262e:	641a      	str	r2, [r3, #64]	; 0x40
    }
  }
  
  /* Return ADC state */
  return HAL_OK;
 8002630:	2300      	movs	r3, #0
}
 8002632:	4618      	mov	r0, r3
 8002634:	3710      	adds	r7, #16
 8002636:	46bd      	mov	sp, r7
 8002638:	bd80      	pop	{r7, pc}

0800263a <HAL_ADC_GetValue>:
  * @param  hadc pointer to a ADC_HandleTypeDef structure that contains
  *         the configuration information for the specified ADC.
  * @retval Converted value
  */
uint32_t HAL_ADC_GetValue(ADC_HandleTypeDef* hadc)
{       
 800263a:	b480      	push	{r7}
 800263c:	b083      	sub	sp, #12
 800263e:	af00      	add	r7, sp, #0
 8002640:	6078      	str	r0, [r7, #4]
  /* Return the selected ADC converted value */ 
  return hadc->Instance->DR;
 8002642:	687b      	ldr	r3, [r7, #4]
 8002644:	681b      	ldr	r3, [r3, #0]
 8002646:	6cdb      	ldr	r3, [r3, #76]	; 0x4c
}
 8002648:	4618      	mov	r0, r3
 800264a:	370c      	adds	r7, #12
 800264c:	46bd      	mov	sp, r7
 800264e:	f85d 7b04 	ldr.w	r7, [sp], #4
 8002652:	4770      	bx	lr

08002654 <HAL_ADC_ConfigChannel>:
  *         the configuration information for the specified ADC.
  * @param  sConfig ADC configuration structure. 
  * @retval HAL status
  */
HAL_StatusTypeDef HAL_ADC_ConfigChannel(ADC_HandleTypeDef* hadc, ADC_ChannelConfTypeDef* sConfig)
{
 8002654:	b480      	push	{r7}
 8002656:	b085      	sub	sp, #20
 8002658:	af00      	add	r7, sp, #0
 800265a:	6078      	str	r0, [r7, #4]
 800265c:	6039      	str	r1, [r7, #0]
  __IO uint32_t counter = 0U;
 800265e:	2300      	movs	r3, #0
 8002660:	60bb      	str	r3, [r7, #8]
  assert_param(IS_ADC_CHANNEL(sConfig->Channel));
  assert_param(IS_ADC_REGULAR_RANK(sConfig->Rank));
  assert_param(IS_ADC_SAMPLE_TIME(sConfig->SamplingTime));
  
  /* Process locked */
  __HAL_LOCK(hadc);
 8002662:	687b      	ldr	r3, [r7, #4]
 8002664:	f893 303c 	ldrb.w	r3, [r3, #60]	; 0x3c
 8002668:	2b01      	cmp	r3, #1
 800266a:	d101      	bne.n	8002670 <HAL_ADC_ConfigChannel+0x1c>
 800266c:	2302      	movs	r3, #2
 800266e:	e113      	b.n	8002898 <HAL_ADC_ConfigChannel+0x244>
 8002670:	687b      	ldr	r3, [r7, #4]
 8002672:	2201      	movs	r2, #1
 8002674:	f883 203c 	strb.w	r2, [r3, #60]	; 0x3c
    
  /* if ADC_Channel_10 ... ADC_Channel_18 is selected */
  if (sConfig->Channel > ADC_CHANNEL_9)
 8002678:	683b      	ldr	r3, [r7, #0]
 800267a:	681b      	ldr	r3, [r3, #0]
 800267c:	2b09      	cmp	r3, #9
 800267e:	d925      	bls.n	80026cc <HAL_ADC_ConfigChannel+0x78>
  {
    /* Clear the old sample time */
    hadc->Instance->SMPR1 &= ~ADC_SMPR1(ADC_SMPR1_SMP10, sConfig->Channel);
 8002680:	687b      	ldr	r3, [r7, #4]
 8002682:	681b      	ldr	r3, [r3, #0]
 8002684:	68d9      	ldr	r1, [r3, #12]
 8002686:	683b      	ldr	r3, [r7, #0]
 8002688:	681b      	ldr	r3, [r3, #0]
 800268a:	b29b      	uxth	r3, r3
 800268c:	461a      	mov	r2, r3
 800268e:	4613      	mov	r3, r2
 8002690:	005b      	lsls	r3, r3, #1
 8002692:	4413      	add	r3, r2
 8002694:	3b1e      	subs	r3, #30
 8002696:	2207      	movs	r2, #7
 8002698:	fa02 f303 	lsl.w	r3, r2, r3
 800269c:	43da      	mvns	r2, r3
 800269e:	687b      	ldr	r3, [r7, #4]
 80026a0:	681b      	ldr	r3, [r3, #0]
 80026a2:	400a      	ands	r2, r1
 80026a4:	60da      	str	r2, [r3, #12]
    
    /* Set the new sample time */
    hadc->Instance->SMPR1 |= ADC_SMPR1(sConfig->SamplingTime, sConfig->Channel);
 80026a6:	687b      	ldr	r3, [r7, #4]
 80026a8:	681b      	ldr	r3, [r3, #0]
 80026aa:	68d9      	ldr	r1, [r3, #12]
 80026ac:	683b      	ldr	r3, [r7, #0]
 80026ae:	689a      	ldr	r2, [r3, #8]
 80026b0:	683b      	ldr	r3, [r7, #0]
 80026b2:	681b      	ldr	r3, [r3, #0]
 80026b4:	b29b      	uxth	r3, r3
 80026b6:	4618      	mov	r0, r3
 80026b8:	4603      	mov	r3, r0
 80026ba:	005b      	lsls	r3, r3, #1
 80026bc:	4403      	add	r3, r0
 80026be:	3b1e      	subs	r3, #30
 80026c0:	409a      	lsls	r2, r3
 80026c2:	687b      	ldr	r3, [r7, #4]
 80026c4:	681b      	ldr	r3, [r3, #0]
 80026c6:	430a      	orrs	r2, r1
 80026c8:	60da      	str	r2, [r3, #12]
 80026ca:	e022      	b.n	8002712 <HAL_ADC_ConfigChannel+0xbe>
  }
  else /* ADC_Channel include in ADC_Channel_[0..9] */
  {
    /* Clear the old sample time */
    hadc->Instance->SMPR2 &= ~ADC_SMPR2(ADC_SMPR2_SMP0, sConfig->Channel);
 80026cc:	687b      	ldr	r3, [r7, #4]
 80026ce:	681b      	ldr	r3, [r3, #0]
 80026d0:	6919      	ldr	r1, [r3, #16]
 80026d2:	683b      	ldr	r3, [r7, #0]
 80026d4:	681b      	ldr	r3, [r3, #0]
 80026d6:	b29b      	uxth	r3, r3
 80026d8:	461a      	mov	r2, r3
 80026da:	4613      	mov	r3, r2
 80026dc:	005b      	lsls	r3, r3, #1
 80026de:	4413      	add	r3, r2
 80026e0:	2207      	movs	r2, #7
 80026e2:	fa02 f303 	lsl.w	r3, r2, r3
 80026e6:	43da      	mvns	r2, r3
 80026e8:	687b      	ldr	r3, [r7, #4]
 80026ea:	681b      	ldr	r3, [r3, #0]
 80026ec:	400a      	ands	r2, r1
 80026ee:	611a      	str	r2, [r3, #16]
    
    /* Set the new sample time */
    hadc->Instance->SMPR2 |= ADC_SMPR2(sConfig->SamplingTime, sConfig->Channel);
 80026f0:	687b      	ldr	r3, [r7, #4]
 80026f2:	681b      	ldr	r3, [r3, #0]
 80026f4:	6919      	ldr	r1, [r3, #16]
 80026f6:	683b      	ldr	r3, [r7, #0]
 80026f8:	689a      	ldr	r2, [r3, #8]
 80026fa:	683b      	ldr	r3, [r7, #0]
 80026fc:	681b      	ldr	r3, [r3, #0]
 80026fe:	b29b      	uxth	r3, r3
 8002700:	4618      	mov	r0, r3
 8002702:	4603      	mov	r3, r0
 8002704:	005b      	lsls	r3, r3, #1
 8002706:	4403      	add	r3, r0
 8002708:	409a      	lsls	r2, r3
 800270a:	687b      	ldr	r3, [r7, #4]
 800270c:	681b      	ldr	r3, [r3, #0]
 800270e:	430a      	orrs	r2, r1
 8002710:	611a      	str	r2, [r3, #16]
  }
  
  /* For Rank 1 to 6 */
  if (sConfig->Rank < 7U)
 8002712:	683b      	ldr	r3, [r7, #0]
 8002714:	685b      	ldr	r3, [r3, #4]
 8002716:	2b06      	cmp	r3, #6
 8002718:	d824      	bhi.n	8002764 <HAL_ADC_ConfigChannel+0x110>
  {
    /* Clear the old SQx bits for the selected rank */
    hadc->Instance->SQR3 &= ~ADC_SQR3_RK(ADC_SQR3_SQ1, sConfig->Rank);
 800271a:	687b      	ldr	r3, [r7, #4]
 800271c:	681b      	ldr	r3, [r3, #0]
 800271e:	6b59      	ldr	r1, [r3, #52]	; 0x34
 8002720:	683b      	ldr	r3, [r7, #0]
 8002722:	685a      	ldr	r2, [r3, #4]
 8002724:	4613      	mov	r3, r2
 8002726:	009b      	lsls	r3, r3, #2
 8002728:	4413      	add	r3, r2
 800272a:	3b05      	subs	r3, #5
 800272c:	221f      	movs	r2, #31
 800272e:	fa02 f303 	lsl.w	r3, r2, r3
 8002732:	43da      	mvns	r2, r3
 8002734:	687b      	ldr	r3, [r7, #4]
 8002736:	681b      	ldr	r3, [r3, #0]
 8002738:	400a      	ands	r2, r1
 800273a:	635a      	str	r2, [r3, #52]	; 0x34
    
    /* Set the SQx bits for the selected rank */
    hadc->Instance->SQR3 |= ADC_SQR3_RK(sConfig->Channel, sConfig->Rank);
 800273c:	687b      	ldr	r3, [r7, #4]
 800273e:	681b      	ldr	r3, [r3, #0]
 8002740:	6b59      	ldr	r1, [r3, #52]	; 0x34
 8002742:	683b      	ldr	r3, [r7, #0]
 8002744:	681b      	ldr	r3, [r3, #0]
 8002746:	b29b      	uxth	r3, r3
 8002748:	4618      	mov	r0, r3
 800274a:	683b      	ldr	r3, [r7, #0]
 800274c:	685a      	ldr	r2, [r3, #4]
 800274e:	4613      	mov	r3, r2
 8002750:	009b      	lsls	r3, r3, #2
 8002752:	4413      	add	r3, r2
 8002754:	3b05      	subs	r3, #5
 8002756:	fa00 f203 	lsl.w	r2, r0, r3
 800275a:	687b      	ldr	r3, [r7, #4]
 800275c:	681b      	ldr	r3, [r3, #0]
 800275e:	430a      	orrs	r2, r1
 8002760:	635a      	str	r2, [r3, #52]	; 0x34
 8002762:	e04c      	b.n	80027fe <HAL_ADC_ConfigChannel+0x1aa>
  }
  /* For Rank 7 to 12 */
  else if (sConfig->Rank < 13U)
 8002764:	683b      	ldr	r3, [r7, #0]
 8002766:	685b      	ldr	r3, [r3, #4]
 8002768:	2b0c      	cmp	r3, #12
 800276a:	d824      	bhi.n	80027b6 <HAL_ADC_ConfigChannel+0x162>
  {
    /* Clear the old SQx bits for the selected rank */
    hadc->Instance->SQR2 &= ~ADC_SQR2_RK(ADC_SQR2_SQ7, sConfig->Rank);
 800276c:	687b      	ldr	r3, [r7, #4]
 800276e:	681b      	ldr	r3, [r3, #0]
 8002770:	6b19      	ldr	r1, [r3, #48]	; 0x30
 8002772:	683b      	ldr	r3, [r7, #0]
 8002774:	685a      	ldr	r2, [r3, #4]
 8002776:	4613      	mov	r3, r2
 8002778:	009b      	lsls	r3, r3, #2
 800277a:	4413      	add	r3, r2
 800277c:	3b23      	subs	r3, #35	; 0x23
 800277e:	221f      	movs	r2, #31
 8002780:	fa02 f303 	lsl.w	r3, r2, r3
 8002784:	43da      	mvns	r2, r3
 8002786:	687b      	ldr	r3, [r7, #4]
 8002788:	681b      	ldr	r3, [r3, #0]
 800278a:	400a      	ands	r2, r1
 800278c:	631a      	str	r2, [r3, #48]	; 0x30
    
    /* Set the SQx bits for the selected rank */
    hadc->Instance->SQR2 |= ADC_SQR2_RK(sConfig->Channel, sConfig->Rank);
 800278e:	687b      	ldr	r3, [r7, #4]
 8002790:	681b      	ldr	r3, [r3, #0]
 8002792:	6b19      	ldr	r1, [r3, #48]	; 0x30
 8002794:	683b      	ldr	r3, [r7, #0]
 8002796:	681b      	ldr	r3, [r3, #0]
 8002798:	b29b      	uxth	r3, r3
 800279a:	4618      	mov	r0, r3
 800279c:	683b      	ldr	r3, [r7, #0]
 800279e:	685a      	ldr	r2, [r3, #4]
 80027a0:	4613      	mov	r3, r2
 80027a2:	009b      	lsls	r3, r3, #2
 80027a4:	4413      	add	r3, r2
 80027a6:	3b23      	subs	r3, #35	; 0x23
 80027a8:	fa00 f203 	lsl.w	r2, r0, r3
 80027ac:	687b      	ldr	r3, [r7, #4]
 80027ae:	681b      	ldr	r3, [r3, #0]
 80027b0:	430a      	orrs	r2, r1
 80027b2:	631a      	str	r2, [r3, #48]	; 0x30
 80027b4:	e023      	b.n	80027fe <HAL_ADC_ConfigChannel+0x1aa>
  }
  /* For Rank 13 to 16 */
  else
  {
    /* Clear the old SQx bits for the selected rank */
    hadc->Instance->SQR1 &= ~ADC_SQR1_RK(ADC_SQR1_SQ13, sConfig->Rank);
 80027b6:	687b      	ldr	r3, [r7, #4]
 80027b8:	681b      	ldr	r3, [r3, #0]
 80027ba:	6ad9      	ldr	r1, [r3, #44]	; 0x2c
 80027bc:	683b      	ldr	r3, [r7, #0]
 80027be:	685a      	ldr	r2, [r3, #4]
 80027c0:	4613      	mov	r3, r2
 80027c2:	009b      	lsls	r3, r3, #2
 80027c4:	4413      	add	r3, r2
 80027c6:	3b41      	subs	r3, #65	; 0x41
 80027c8:	221f      	movs	r2, #31
 80027ca:	fa02 f303 	lsl.w	r3, r2, r3
 80027ce:	43da      	mvns	r2, r3
 80027d0:	687b      	ldr	r3, [r7, #4]
